:020000040000FA
:040000006FD00400B9
:101000006F00907E00000000000000009020002093
:10101000AA220020A9BDF9F56C23002000000000E1
:10102000000000006C230020902000200000000041
:101030000000000090200020000000009020002010
:101040000000000090200020902000209020002030
:101050009020002090200020582F00209424002071
:101060000000000090200020902000201E2400207E
:1010700090200020D22300209020002090200020EB
:101080009020002090200020902000209020002020
:101090009020002001A04111B7170040985F3AC688
:1010A000945F3247E39CE6FE3245410182800111A4
:1010B00013078008F337078093F787083EC20100C3
:1010C0000100B7170040930570052380B70413068D
:1010D00080FA2380C7040100010083C6B70493F699
:1010E000F60DA385D704238007049246F3A6068055
:1010F0000100010093760502D5CEF336078093F602
:10110000860836C4010001002380B7042380C70489
:1011100001000100B70614007D89558D88C70100C4
:1011200001000100010023800704A246F3A6068007
:101130000100010073370780137787083AC6010062
:1011400001002380B7042380C704010001000100CF
:1011500001003727004093061005A303D7802380A2
:101160000704B247F3A70780010001009307800836
:10117000F3B7078093F787083ECE01000100B71749
:101180000040130770052380E704130780FA2380CB
:10119000E7040100010003C7B70413670708A3852C
:1011A000E70423800704F247F3A70780010001004A
:1011B0000561828093760504BDC6F336078093F6F9
:1011C000860836C8010001002380B7042380C704C5
:1011D00001000100B7061400938606047D89558D31
:1011E00088C7010001000100010023800704C246F6
:1011F000F3A6068001000100733707801377870884
:101200003ACA010001002380B7042380C70401000B
:1012100001003727004093062005A303D7802380D1
:101220000704D24781B773370780137787083ACC12
:10123000010001002380B7042380C70401000100DE
:1012400098471367070C98C723800704E24719BF24
:101250000111814601468145114506CE97000000E7
:10126000E780605893078008F3B7078093F78708F3
:101270003EC601000100B717004013077005238028
:10128000E704130780FA2380E7040100010003C785
:101290006704136717002383E70423800704B2471A
:1012A000F3A7078001000100F2400561828041112F
:1012B000814601468145114597000000E780A05214
:1012C00013078008F337078093F787083EC40100AF
:1012D0000100B7170040130670052380C70493066A
:1012E00080FA2380D70401000100FD552396B70240
:1012F00023800704A245F3A5058001000100733790
:101300000780137787083AC6010001002380C704CD
:101310002380D7040100010003C767041367170087
:101320002383E70423800704B247F3A70780010063
:10133000010001A0B1473305F50201007D1575FDDF
:101340008280411122C426C206C6AA8401446317C2
:101350009400B24022449244410182800504130566
:10136000803E420497000000E78000FD4180C5B741
:101370009305000273A04580824573901534924016
:101380002242B2424243D2436244F2440255925551
:101390002256B2564257D2576258F25806499649D9
:1013A000264AB64A464BD64B664CF64C065D965DD1
:1013B000265EB65E465FD65F09617300203041113C
:1013C000B7170040985F3AC6945F3247E39CE6FE49
:1013D000324541018280B71700401307000323887C
:1013E000E702854717170000232AF74873002030CB
:1013F000411122C42D6426C24AC006C637190040D6
:101400001304A4AAB704002023208900976000E0F9
:10141000E780206F9C408297976000E0E780606ED5
:10142000E5B737370040834747009146BD8B639E41
:10143000D702B73600401306F00F973500009385AA
:1014400025209737000083D7A72F03C7A60013775F
:10145000F70F1DE3B7E70400BC4F09468945171590
:1014600000000345A5F8829731A099466394D70000
:10147000834757007300203003C786001377F70FA8
:10148000E365F6FC13851700AE97173800002319A3
:10149000A82A2380E70075B7B787004003C7670015
:1014A000098B6309071003C77700930600031377BE
:1014B0000703630DD708173800000348387817363C
:1014C00000001306A6740547B30606012380E60054
:1014D00083C577001737000013074775429793F5C8
:1014E000F50F2300B70003C58700973500009385EB
:1014F000E572C2951375F50F2380A5000347070019
:1015000089451377F703630CB70C63E7E50A6306B5
:10151000071A8545630CB7129737000083C7177207
:101520003307F600034707001377F70F19CB85073A
:1015300093F7F70F3D476363F71A17370000A30FC0
:10154000F76EB787004009472383E700B78700405D
:1015500083C77700E207E18763DE0704973700005F
:1015600083C7D76D173700001307476A3E97854634
:101570002300D700173700001307476B3E979306E9
:1015800000032300D70017370000130727693E9791
:10159000A14685072300D70093F7F70F3D47636403
:1015A000F71417370000A30BF768B7870040094707
:1015B0002383E70073002030930610026300D70EE8
:1015C000930620026305D70693060002E316D7F4BC
:1015D00003C727021377C70F13672700D5A803C7D0
:1015E00067001377070465CB03C7A702173800000D
:1015F00013084843173500001305853A13470708B9
:101600002385E70203C7A7021377370F1367870005
:101610002385E702814713070004B305F5008C41D9
:10162000B306F80091078CC2E399E7FEF5B503C74E
:10163000A702134707042385E70203C7A70213770E
:10164000C70F136727002385E702F9B503C76700B3
:101650001377070449C303C767021738000013084C
:101660002830173500001305652713470708238323
:10167000E70203C767021377370F136787002383D7
:10168000E702814713070004B305F5008C41B30658
:10169000F80091078CC2E399E7FEBDBD03C767025E
:1016A000134707042383E70203C767021377C70FB3
:1016B000136727002383E70285B503C76700137705
:1016C000070411CB03C727021377370F136787006F
:1016D0002381E70291B5238006003DBD97370000C6
:1016E000A38E0754B9BD97370000A389075475BD71
:1016F0002303048015472303E48001002302A48010
:10170000828083076480E3CE07FE23030480828007
:1017100083076480E3CE07FE03454480828083070D
:101720006480E3CE07FE2302A4808280411126C498
:101730004AC24EC006C61377F50BAD47AA892E895B
:101740009544630CF700194597000000E78080FA84
:1017500097000000E78020FB8D444E859700000035
:10176000E78040F9FD59FD1463983401B240A2446A
:101770001249824941018280135509011375F50F01
:1017800097000000E780E0F92209F1BF011126CCA3
:1017900006CEB704080097000000E780C0F61545A4
:1017A00097000000E78000F597000000E78080F6D2
:1017B00097000000E78000F62AC697000000E78047
:1017C00080F432459377150089EB13651500137586
:1017D000F50FF240E24405618280FD14E9F0014515
:1017E000CDBF397126DC4ADA4ED852D656D45AD2F9
:1017F0005ED006DE62CE66CCB7E700E07D5783AAF6
:10180000070022C603AA470023A0E71823A2E7186F
:10181000B7170040130770052380E704130780FA09
:101820002380E70483C74704930B75FFB684E20760
:1018300093FBFB0F8546AA892E8B32893724004003
:10184000E187015763FA76016308D50089461307DB
:1018500000026313D5000157D98F93F7F70FB71C18
:1018600000402382FC0411472303E4801305F00F9A
:1018700097000000E78000E8094C97000000E7802F
:1018800080E863657C15B7050700DA9537870700A0
:10189000795563FEE504B3879500636AF704370B57
:1018A0000800A94733EB65016395F90881E8814495
:1018B00097000000E78020E5268515A8DA85094510
:1018C00097000000E780C0E605090345F9FFFD1415
:1018D000050B97000000E780C0E481C49377FB0FFD
:1018E000E5F797000000E780A0EA69F17D55B7179A
:1018F0000040130770052380E704130780FA238054
:10190000E70403C74704418B2382E704F250B7E79B
:1019100000E023A0571123A24711E2543244525948
:10192000C259325AA25A125B825B724CE24C21615C
:101930008280A547639BF90685691309F00FB306FA
:101940009900B3742B01B6941349F9FFB37499004D
:10195000856B33796901416B9387F9FFB3F72701F1
:1019600099E363FC340193D94900C147E3E637FFAB
:101970003DBF0569C1697D19D9B71305800D63881D
:101980006901130500026384790113051008CA85F3
:1019900097000000E780C0D997000000E78040DF93
:1019A00031D54E99B38434416DBFDA852D4597000A
:1019B0000000E780E0D7CA94E30B99EE0509970091
:1019C0000000E78020D5A30FA9FEFDB79387F9FF9C
:1019D00093F7F70F636DFC0C83C71C0413073008E3
:1019E0006315F706370708006361EB06B3079B0032
:1019F000B706100063FBD704334BEB0089476399AC
:101A0000F9068980D549E38404EADA850945970017
:101A10000000E780E0D111090327C9FF9147232087
:101A2000E48003076480E34E07FE23033481FD173F
:101A3000EDFBFD14110B81C49377FB0FE9FF9700B9
:101A40000000E780E0D461F155B5B717004003C747
:101A50005704B70708001377070219E3B787070091
:101A60007955E376FBE833079B00E3F9E7F841B5E6
:101A70008547E380F9F0DA852D4597000000E7807F
:101A800020CB9389F4FFE38404E297000000E78011
:101A900060C893F7390091EB83260480032709007F
:101AA00093074900E396E6E03E89CE84D9BFB54767
:101AB0006399F9001305900B97000000E78080C33D
:101AC000FDB3B1471305B00AE388F9FE9947639760
:101AD000F904B7050800B365BB002D459700000069
:101AE000E78000C581448D4BA14997000000E78045
:101AF00060C263967401832704802320F900850463
:101B0000E39534FF8327048013172B0163550700E7
:101B10002312F90069BB2322F90051BB9D47639F43
:101B2000F90281451305B00497000000E78040C02A
:101B3000BD442320090023220900FD59970000001D
:101B4000E78040BD93F77400CA9703C70700FD14F0
:101B5000398D2380A700E39334FF91BBA14763979E
:101B6000F90697000000E780A0C28144630D0B00D6
:101B70008D479304C0036308FB00930400056304CE
:101B80008B01930440041375C507E30295D21945F0
:101B900097000000E78000B697000000E780A0B63D
:101BA000054597000000E780E0B426859700000017
:101BB000E78020B7094597000000E78080B69700CE
:101BC0000000E780E0BCE31405CE0DB39147639FAE
:101BD000F9001305600697000000E780A0B19700A8
:101BE0000000E78040B213059009F9B5E38109CC04
:101BF000F1547DB9BD6601471736000013068621F2
:101C0000938606A685458347060093F7F70F91C391
:101C100082800507E3F9E6FE97370000238CB71EA4
:101C2000DDB77D166206618693178601E18763D46E
:101C3000070001458280931726003307F500AE9711
:101C400018439C4363E7E7007D16E37FF7FC7D556F
:101C5000828005458280FD15E205E18513978501A7
:101C6000618793F7F50F63480700FD15139725006B
:101C70002A97584365D713851700620561858280CE
:101C80003308B5021C4283A80600B335B502C297DB
:101C900033B50701AE98469585486367B5006394F0
:101CA000A50063E3070181480C43C6950CC388C2B5
:101CB0001CC2828081471397870161876343B70005
:101CC0008280139727002A97232007008507E5B70E
:101CD0008147014793968701E18663C5B6001335B6
:101CE0001700828093962700AA9694428507558F05
:101CF000D5B793D755408A07AA979C430545331516
:101D0000B5007D8D828017F3FFDFE702833D2A84D3
:101D100097000000E78060F405C5931725003E9406
:101D20000327C4FF814711EB7D1516053E9542053B
:101D3000418517F3FFDF6700033D05838507E5B79E
:101D40000145C5BF81471397870161876343C7007A
:101D5000828013972700B386E50094422A9785076F
:101D600014C3D5B77D1662066186014793178601B5
:101D7000E18763D50700133517008280931726008B
:101D8000B306F500AE9794429C437D16B58F5D8FE8
:101D9000F1BF8A05AA9501476363B500828083A6D7
:101DA000C5FFF11593D71600D98F9CC11397F60183
:101DB000E5B72A830148014701456343D700828084
:101DC000B387050183A80700B30706019C43C697A4
:101DD000AA976384F80033B517010507B308030118
:101DE000620723A0F80061871108C1BF2A83014759
:101DF0008147014563C3D70082803388E50083288B
:101E00000800330EE600032E0E003388A840330886
:101E1000C8416384080133B508018507B308E300AE
:101E2000E20723A00801E1871107E9B717F3FFDFF5
:101E3000E702232B0111B286B2842E86AA850A8579
:101E400097000000E780C0FA2A84A6850A859700DB
:101E50000000E78020E833348000060413351500C5
:101E6000018D056117F3FFDF6700E32917F3FFDF3B
:101E7000E702A3244111AA89AE8A328BB68402C23A
:101E800002C402C60144131C8401135C8C416349E3
:101E90009C02939B1400FD1B0549138CF4FFF15C1D
:101EA00033048901620461846340740792478E049D
:101EB000CE9423AEF4FE410117F3FFDF67006323E6
:101EC00013192400B30B2B01014A93172A00D6974C
:101ED00083A50B0088437800340050009700000071
:101EE000E78040DA050A93178A01E187F11BE35E78
:101EF000FCFC92474E9905042320F900A2473EC2FC
:101F0000B24702C63EC441B7131A8901135A8A4127
:101F1000131D240093178A01E18763CF970092472E
:101F20000A044E941CC0A24705091379F90F3EC25A
:101F3000B24702C63EC4ADB7B3079A0313152A00D1
:101F400056950841780034005000050AEA97DA9760
:101F50008C4397000000E780E0D26DBF197106C284
:101F600012C416C61AC81ECA22CC26CE2AD02ED219
:101F700032D436D63AD83EDA42DC46DECAC0CEC2C9
:101F8000D2C4D6C6DAC8DECAE2CCE6CEEAD0EED2F9
:101F9000F2D4F6D6FAD8FEDA971500009385858D2F
:101FA0008841E700050092402242B2424243D243B8
:101FB0006244F244025592552256B2564257D257C5
:101FC0006258F25806499649264AB64A464BD64BBD
:101FD000664CF64C065D965D265EB65E465FD65F45
:101FE0000961730020300000972100209381810156
:101FF000175100201301018117F5FFFF1305C500DC
:102000009705002093850500171600201306C6FDCE
:1020100063FAC5008322050023A055001105910530
:10202000E3EAC5FE17050200130545439715002096
:102030009385C5FB171600201306466763FAC50093
:102040008322050023A0550011059105E3EAC5FE92
:102050001715002013058565974500209385852772
:102060006377B500232005001105E36DB5FEFD4241
:10207000739002BC8D4273904280B722000093821D
:10208000828873900230970200209382A2F793E235
:10209000320073905230975200009382A2A6739040
:1020A00012346FB0F47573002030397101436EC67D
:1020B00019A0397141536AC866CA62CC5ECE19A0B4
:1020C000397101535AD056D252D44ED64AD826DA54
:1020D00022DC06DE33016140828241114AC026C201
:1020E00022C406C68282B24D4101024D924C224C5E
:1020F000B24B4101024B924A224AB2494101024984
:1021000092442244B240410182803D432A87637356
:10211000C3029377F700BDEFADE5937606FF3D8AE6
:10212000BA960CC34CC30CC74CC74107E36BD7FE30
:1021300011E28280B306C3408A0697020000969699
:102140006780A6002307B700A306B7002306B700E1
:10215000A305B7002305B700A304B7002304B70005
:10216000A303B7002303B700A302B7002302B700FD
:10217000A301B7002301B700A300B7002300B700F5
:10218000828093F5F50F93968500D58D9396050182
:10219000D58D61B7939627009702000096968682A8
:1021A000E78086FA9680C1171D8F3E96E374C3F8C8
:1021B000A5B73367B500FD530D8B79E7B7877F7FF0
:1021C0009387F7F710419441B372F6003363F6003A
:1021D000BE92B3E262006397720C6318D606504158
:1021E000D441B372F6003363F600BE92B3E26200EC
:1021F0006398720A631BD60410459445B372F600C7
:102200003363F600BE92B3E262006391720A631E0A
:10221000D6025045D445B372F6003363F600BE9241
:10222000B3E26200639A72086311D60210499449BE
:10223000B372F6003363F600BE92B3E262006393BA
:1022400072085105D105E30FD6F6131706019397CF
:102250000601631CF7001357060193D706013305E7
:10226000F7409375F50F91E982804183C18333056F
:10227000F7409375F50F91E182801377F70F93F78D
:10228000F70F3305F74082800346050083C605003B
:10229000050585056313D60065FA3305D6408280AF
:1022A00011059105E312D6FE014582802105A105A5
:1022B000E31CD6FC014582803105B105E316D6FC4E
:1022C000014582804105C105E310D6FC01458280AD
:1022D000B717004003C777051377E70FA38BE70411
:1022E000130700F8A38DE7043D47238CE704130789
:1022F0005003A38CE70403C7A7051377D70F238DDB
:10230000E7048280B717004003C7E7020D89411137
:102310001377C70F498F93068008F3B6068093F6AC
:10232000860836C601000100930670052380D70495
:10233000930680FA2380D704010001002387E70277
:1023400023800704B247F3A7078001000100410181
:10235000828041112A83014E930E407E130F001993
:10236000930F400663E56E129308001913034006AD
:10237000B3781503854E0D4FA14F337365020D8958
:102380001335150063EFBE121308F6FF79467298F5
:102390004208135808013307C70213D61700BE07B7
:1023A00032976146B3F6C60213068070B386C60242
:1023B0003697A166F58F42075D8FB716004083C739
:1023C000F60293F70708A303F1000346710083C7E1
:1023D000F60293F70708E394C7FE83477100B71628
:1023E000004093F7F70F6388071293078008F3B74D
:1023F000078093F787083EC401000100B71700402B
:10240000930670052380D704930680FA2380D704AF
:102410000100010023AA070383C6170393E60608F9
:10242000A388D70223800704A247F3A707800100EF
:1024300001001166B71700407D16D45BC85F938515
:102440004703A98EF18EF5FA93068008F3B606804D
:1024500093F6860836C601000100930670052380B6
:10246000D704930680FA2380D7040100010098C1A5
:1024700003C7170313670704A388E7022380070431
:10248000B247F3A7078001000100410182807D135C
:102490003368E3039308E016630E08003368F30320
:1024A0009308D016630808009378330093B8180097
:1024B0009388D81633081E01131E0801135E0E01FF
:1024C00055B56393E5030548638608000148630337
:1024D00003002A8871087298FD15131E0801C205B1
:1024E000135E0E01C18179BD13F8150063F4BF00BE
:1024F0007908D5B713381800E5BF83C7F60293F7FC
:102500000708A303F1000346710083C7F60293F79F
:102510000708E394C7FE8347710093F7F70FF1DFD5
:10252000E9B531714AD966CB06DF22DD26DB4ED70D
:1025300052D556D35AD15ECF62CD6AC96EC7AA8C26
:1025400002D897100000E78020B12A8993078008FD
:10255000F3B7078093F787083EDA01000100B71749
:102560000040130770052380E704130780FA2380D7
:10257000E7040100010003C7F7021377770FA38771
:10258000E70203C7F70213678700A387E7022380E8
:102590000704D257F3A70780010001000545970003
:1025A0000000E78060D6130780C13347E902116A53
:1025B00093070AE893065002BD69930BA004814A71
:1025C000014B13048008930470057D1AB347F90288
:1025D0003307D7023EC0FD873ECC938709A69309F7
:1025E000803E3347F7023AC27D873AC43347390306
:1025F0008549B399990193D93940B306D702B30BF2
:102600007703B3C6F602B3CBFB0236C6FD8636C8E7
:1026100093D6FB4136CEB7460F0093860624334946
:10262000D9028566938606FAB3969601B389E902C4
:10263000130760553309D90293060010B389E902E4
:102640003349D902B3C9F9029316390036CA37198A
:102650000040FD8636D0930D090493D7F9413ED250
:10266000F336048093F6860836DC010001009307F8
:1026700070052380FD00930680FA2380DD000100B1
:1026800001008346390593F6860FA309D9048346D2
:10269000390593E61600A309D90423800D00E256FC
:1026A000F3A6068001000100130C80FA116DF336C9
:1026B000048093F6860836DE01000100930770055A
:1026C0002380FD0023808D01010001008346390530
:1026D000216693E60602A309D90483560905B3E6E9
:1026E000A6012318D90483560905D18E2318D904CD
:1026F00023800D00F256F3A60680010001008346F8
:10270000390593F606026381061A03463905218AC4
:102710006DDE081897100000E7800098733604807B
:1027200013768608B2C20100010023809D00238039
:102730008D0101000100B717004003C6370513766D
:10274000F60DA389C70403C6370513660602A389DD
:10275000C704835609052166B3E6A6012318D904E8
:1027600083560905D18E2318D90423800D0096467F
:10277000F3A60680010001008346390593F60602A0
:10278000638B061483463905A18AEDFE970000206D
:10279000E7806090AA8636D497000020E780A08F5B
:1027A000A256E30AD5FE835609054255B3E6A601B3
:1027B0002318D90497100000E780C08F834639059D
:1027C000A18AEDDE03560905834629058247337643
:1027D000CA00B306DA0293D5F641B296B388F64042
:1027E000E24733B8C6002E983308F840A247B3B684
:1027F00016013308D84063C70701631DF8009247EC
:1028000063FA1701C247634FF80E63950701B24799
:1028100063EAF80E894663E9660FF24693151800DD
:1028200013D3F8015E8613951800B365B30042D642
:1028300046D497C00100E780A0143258050B137BE3
:10284000FB0F63470001631A0838A25863870838F2
:1028500013081500B336A800B69513D6F5013298C3
:10286000B336C800AE9613581800FE06B3E606014C
:102870007336048013768608B2C6010001002380F7
:102880009D0023808D01010001000356C902B2960C
:10289000C206C1822316D90223800D00B646F3A6D4
:1028A00006800100010021B5F336048093F6860806
:1028B000B6C00100010023809D0023808D0101002E
:1028C00001008346390593E60602A309D904238053
:1028D0000D0086460DB5F336048093F68608B6C41F
:1028E0000100010023809D0023808D010100010073
:1028F0008346390593E60602A309D90423800D0017
:10290000A646BDB5E30B0BF0F336048093F68608BC
:10291000B6C801000100930680FA23809D00238041
:10292000DD00010001008346390593F5FC0F93F6A5
:10293000860FA309D90483463905CD8EA309D9048E
:1029400023800D00C646F3A6068001000100130592
:1029500080FA03463905930639051D8A631C9629BA
:102960007336048013768608B2CC0100010013068A
:1029700080FA23809D002380CD000100010003C662
:1029800006001376F60D2380C60003C60600136604
:1029900006022380C600835609051166D18E2318CE
:1029A000D904835609052166D18E2318D9042380C2
:1029B0000D00E646F3A6068001000100130680FA2A
:1029C0008346390593F60602638006268346390559
:1029D000130C3905A18AFDDA081897000000E7807A
:1029E000A06BF336048093F68608B6D00100010090
:1029F000930680FA23809D002380DD000100010002
:102A000083460C00116693F6F60D2300DC00834626
:102A10000C0093E606022300DC0083560905D18EE4
:102A20002318D904835609052166D18E2318D904A9
:102A300023800D008656F3A60680010001001306D0
:102A400080FA8346390593F60602638A0620834698
:102A50003905A18AEDFE97F0FF1FE780C0632A8C3D
:102A600097F0FF1FE7802063E30C85FF835609057D
:102A700011664255D18E2318D90497000000E780D3
:102A800060638346390513063905A18AFDDAF336FA
:102A9000048093F68608B6D401000100930680FAFC
:102AA00023809D002380DD00010001008346060095
:102AB00093F6F60D2300D60023800D00A656F3A64C
:102AC0000680010001008356090503462905D24707
:102AD000B376DA003306CA021305800C9355F6412B
:102AE0003696330DF6408257333CD6002E9C333653
:102AF000A601330CFC40330CCC40330885039256BE
:102B00004E86B335A5033305A503C29597C00100D2
:102B1000E78000E763468001631E0C16630C0D1608
:102B2000130615003335A6002E959356F5013696FB
:102B3000B335D600AA959396F50105828585D18E89
:102B40006346B000639D051A638B061A0356C902DB
:102B500015823305D6003336C500B2956348B00000
:102B6000639105241306F00F637DA622894663F363
:102B7000561593078008F3B7078093F78708BED6EA
:102B80000100010037170040930770052300F70488
:102B9000930780FA2300F704010001008356C7025F
:102BA00089678117D58FC207C1832316F7022300D7
:102BB0000704B657F3A7078001000100FA506A54D2
:102BC000DA544A59BA592A5A9A5A0A5BFA4B6A4C49
:102BD000DA4C4A4DBA4D296182801308F5FF33352E
:102BE000A800FD152E951356F5013298B336C8008E
:102BF000AA9695B9F336048093F68608B6CA010002
:102C0000010023809D002380AD0001000100834668
:102C10003905CD8EA309D90423800D00D646F3A62D
:102C200006800100010035B3F336048093F6860870
:102C3000B6CE0100010023809D002380CD0001005D
:102C400001008346390593E60602A309D9042380CF
:102C50000D00F646F3A606800100010095B3F33699
:102C6000048093F68608B6D20100010023809D00FF
:102C70002380CD00010001008346390593E606025A
:102C8000A309D90423800D009656F3A606800100FF
:102C9000010045BB9306F5FF33B5A600FD152E9543
:102CA0009355F501AE96B3B5B600AA951396F50106
:102CB000858269B5F336048093F68608B6D801009C
:102CC0000100930680FA23809D002380DD0001002F
:102CD00001008356C9020566011693F6F60FD18EE0
:102CE000C206C1822316D90223800D00C656F3A660
:102CF000068001000100850A93FAFA0F95B233E6C7
:102D0000B60045C20356C9023305D0403338A0008F
:102D1000B305B040B385054115826345B000D1E1EC
:102D20006371A608894663F0560593078008F3B7D8
:102D3000078093F78708BEDA01000100B71700404B
:102D4000130770052380E704130780FA2380E70444
:102D50000100010003D7C7027D8B2396E702238081
:102D60000704D65781BDF336048093F68608B6DC97
:102D700001000100930680FA23809D002380DD007E
:102D8000010001008356C9020566011693F6F60F8D
:102D9000D18EC206C1822316D90223800D00E656C9
:102DA000B9B793078008F3B7078093F78708BEDEAB
:102DB0000100010037170040930770052300F70456
:102DC000930780FA2300F704010001000356C702AD
:102DD00093975600B297C207C1832316F7022300C8
:102DE0000704F657C1BB914763EEB70217D701003E
:102DF000130747568A05BA959C41BA978287B71739
:102E0000004003A7470B1345F5FF698F23AAE70A84
:102E100003A7070B698F23A8E70A03A7070A798D81
:102E200023A0A70A8280B717004083A6470B134749
:102E3000F5FFF98E23AAD70A83A6070B558D23A881
:102E4000A70A83A6070A758F23A0E70A8280B7170F
:102E5000004003A7470B498F23AAE70A03A7070BE4
:102E60001345F5FF45BFB717004083A6470B13472F
:102E7000F5FF758F23AAE70A03A7070A598D4DB7F7
:102E8000B717004003A7470B498FEDB7914763EE93
:102E9000B70217D701001307274D8A05BA959C4141
:102EA000BA978287B717004003A7470D1345F5FF70
:102EB000698F23AAE70C03A7070D698F23A8E70CE6
:102EC00003A7070C798D23A0A70C8280B7170040B9
:102ED00083A6470D1347F5FFF98E23AAD70C83A6C7
:102EE000070D558D23A8A70C83A6070C758F23A06B
:102EF000E70C8280B717004003A7470D498F23AA2C
:102F0000E70C03A7070D1345F5FF45BFB7170040B2
:102F100083A6470D1347F5FF758F23AAE70C03A778
:102F2000070C598D4DB7B717004003A7470D498FC0
:102F3000EDB7797122D43714004026D24AD0035914
:102F400024028354040206D64209C2044ECE52CC57
:102F500056CA13590901C1802DE11379F9F793F489
:102F6000F49F4209C20413590901C18093078008E4
:102F7000F3B7078093F787083EC401000100930769
:102F800070052300F404930780FA2300F404010081
:102F90000100231124032310940223000404A247F8
:102FA000F3A7078001000100B25022549254025945
:102FB000F249624AD24A45618280B7F507008146EC
:102FC0003000B105194597000020E7808081A247B5
:102FD00013972701E34A07FC1369090893E40440A7
:102FE00093098008F3B7098093F787083EC0010072
:102FF0000100930A700523005405130A80FA230088
:10300000440501000100231124032310940223002E
:1030100004048247F3A7078001000100294597F0C7
:10302000FF1FE7802031F3B9098093F989084EC268
:1030300001000100230054052300440501000100A4
:103040008357040293E707202310F40223000404AB
:103050009247B9B7B7170040884742054181937737
:10306000050491EB9377F5013755E80113050580C9
:103070003345F50282809377050C130700046397AC
:10308000E7009377F50137459C1CCDB72165130503
:1030900005D0828037E700E01C435443A183E20659
:1030A000D58F1CC1FD572320F7182322F7188280E3
:1030B00013178500B7E700E023A0E710618123A282
:1030C000A7108280B7F700E08847CC47828081470D
:1030D00037370040A14663C4C7003285828003456C
:1030E000B740E38EA6FE3385F5000345050085074E
:1030F0002304A740CDB797070020938727EF9C4371
:10310000173700201307071D3E95636EE50017373C
:1031100000201307274F6368A70017070020232705
:10312000A7EC3E858280FD57EDBF8280411122C40D
:1031300006C62A8497000000E78000F22947B307FB
:10314000E502B2408D83B3D7870222449507B3D7F7
:10315000E70237370040C207C1832316F700410159
:103160008280411137150E0006C697000000E780E7
:1031700020FCB7370040130770F82381E7000D47A4
:10318000A381E70013070004A380E7000547238716
:10319000E700B24041018280373700408347270073
:1031A0001A0593F7F703C98F93F7F70F2301F70079
:1031B0008280B737004003C7170019C9D98DA38093
:1031C000B70003C70700136787002380E7008280EA
:1031D00093C5F5FFF98DA380B7008280AE872A875B
:1031E000B736004021463738004089E71703000012
:1031F0006700E3F383C8B600E30916FF05078348B9
:10320000F7FFFD17C20723041801C183F9BF41115D
:1032100022C406C62A8497000000E780E0E329471D
:10322000B307E502B2408D83B3D7870222449507E6
:10323000B3D7E70237370040C207C1832316F740F0
:1032400041018280716541111305052006C6970072
:103250000000E78000FCB7370040130770F82381B7
:10326000E7400D47A381E74013070004A380E74030
:1032700005472387E740B24041018280CC4141119C
:1032800006C6328503C6150083C5050022064D8E8D
:1032900042068D654186138875A2630C0611634B47
:1032A000C804138845A26300060D634AC8009385CD
:1032B00035A26301B6082390060029464DA0138865
:1032C00055A26305060D938565A2E316B6FE8D45EE
:1032D0001D4663E6E5081146198E63F3C7003E8676
:1032E000B7E704002390C600FC4797D501009385FB
:1032F000E5099DA0138895A263030611634E060D90
:103300001388A5A263000613938505A5E315B6FAF5
:1033100099451D4663E5E504198E63F3C7003E86B3
:10332000B7E704002390C600FC479705002093856B
:1033300025D61DA09D451D4663E3E5022146198E55
:1033400063F3C7003E86B7E70400FC472390C6003E
:103350009705002093850536BA9582970146B240BD
:10336000328541018280AD451D46E3EAE5FE3146E6
:10337000198E63F3C7003E86B7E704002390C600AA
:10338000FC4797D501009385E502F9B7B1451D4685
:10339000E3E7E5FC3546198E63F3C7003E86B7E7E1
:1033A00004002390C600FC4797D501009385850152
:1033B00065B78D451D46E3E4E5FA1146198E63F3C2
:1033C000C7003E86B7E704002390C600FC4797D5A8
:1033D0000100938565FC49B78D451D46E3E1E5F89D
:1033E0001146198E63F3C7003E86B7E704002390A9
:1033F000C600FC4797D50100938585FEB1BFA54562
:103400001D46E3EEE5F42946198E63F3C7003E86B8
:10341000B7E704002390C600FC4797D501009385C9
:1034200065F81DBFB5451D46E3EBE5F23946198E3B
:1034300063F3C7003E86B7E704002390C600FC474D
:1034400097D50100938585F301BFB7E7040003A377
:103450000713970600209386A6C24146A545170587
:1034600000201305E5B802832D455DE703C505007F
:103470000947631FE50803A84500411106C6034735
:10348000180032850346080022074168518F9308CF
:1034900028FE6307170563E9E800051863030703BF
:1034A00023900600294591A8130648FE630AC70425
:1034B0001518E31707FF15463E87637BF60015478F
:1034C00001A8130600023E876374F600130700028A
:1034D000B7E704002390E600FC471316070111A884
:1034E0003E8691C30546B7E70400FC472390C6001B
:1034F0004206CC45418282970145B240410182801B
:10350000130600083E87E375F6FC13070008C9B7E9
:103510002390060005458280828041677917630405
:10352000E504411122C406C685472A84639FF5003D
:10353000B7E7040022852244B24003A3871397050E
:103540000020938565314101028389476399F50025
:10355000B7E7040083A7070B8545829771D9B2406E
:103560002244410182808280797126D252CCAE847D
:103570002A8A97D501009385A5E817D50100130580
:10358000A5EA06D63AC622D44AD0368432894ECE2F
:1035900097C00100E780008AA28517D501001305B6
:1035A000A5E997C00100E780E088294597C00100A0
:1035B000E780208D83C7840093F70702F9E383C96E
:1035C00004008947054532476396F908D44083C70C
:1035D000160083C60600A207D58FC166138616FEA5
:1035E000638CC7028D16638FD7068D6693862690EF
:1035F00029456391D706B7E70400A286225403A3A6
:103600004714B250F2494A86A6850259925452850F
:10361000624A8547456102832D450DEF93070002FD
:10362000354563E98702B7E70400FC47C844130641
:103630000002CA85829781499707002093878722D5
:103640009C43014581CB9C4391C74E852286CA8508
:1036500082970145B250225492540259F249624A6B
:10366000456182802D457DF79307700F3545E3E373
:1036700087FEB7E70400FC47C8442286CA858297C4
:1036800065BF2145C1BF411122C437E4040083272F
:10369000841326C2AA84416506C697050020938537
:1036A000A51B7D1582978327C40A17050000130503
:1036B00005E78588829795C0032304132244B2400E
:1036C000924497060020938626AE4146C5451705CD
:1036D00000201305659C41010283B24022449244BC
:1036E00001454101828019C59707002023ACA71628
:1036F00001458280454582801147636AA70A97D6B3
:1037000001009386A6CE0A0536951841411106C6DA
:103710003697AE87B2850287130700026145639D25
:10372000E700B7E70400FC47130600021705002076
:103730001305C5F882970145B240410182800547D3
:103740006145E39BE7FEB7E70400FC470546170524
:1037500000201305A5F8F9BF1307700F6145E39D1D
:10376000E7FCB7E70400FC471306700F17050020BD
:10377000130505F7C1B7130700086145E39EE7FA93
:10378000B7E70400FC4713060008170500201305DF
:10379000A5044DB715476145E390E7FAB7E7040084
:1037A000FC471546170500201305450B61B7094571
:1037B0008280411126C2B7E4040083A7C41322C447
:1037C0004AC006C62E84970500209385E5082A89FD
:1037D0008297058905C5970700209387E78B83D7D4
:1037E000A70BA28503A3440D2310F4002244B2408A
:1037F00092444A850249014641010283B240224473
:103800009244024949454101828097070020238D57
:1038100007049707002023AB0704B717004003A74E
:10382000070CB706C0FFFD16758F23A0E70C03A792
:10383000070DB7064000558F23A8E70C03A7070C18
:103840003D9B23A0E70C03A7070D1367070123A8DF
:10385000E70C8280B717004003A5470C83A7470CED
:10386000598113451500C18B058999E3136525001E
:103870009707002083C747FF6380A70297070020B0
:103880002384A7FE11C997070020938727FE03A36F
:1038900007006303030002838280114517F3FFFFD3
:1038A000670063C8011122CC06CE3714004026CA37
:1038B0004AC84EC652C483447405034AB4058349BA
:1038C00084050349940597F0FFFFE780A0A0834794
:1038D000A40593F4F40F137AFA0F93E71700230D5E
:1038E000F40493F9F90F1379F90FB717004003C7E0
:1038F000A705058B6DFF03D5C705A38D4705238C51
:103900003705A38C2705A38B9704F2406244D24469
:103910004249B249224A05618280411193970501CB
:1039200022C406C626C2C1872E8463DC0700B7E422
:103930000400FC54829719C1BC5482972165218DE3
:1039400015A893F7150013C515008DE793F725000B
:103950009DC797000000E78020F0B7E70400BC4F48
:103960001306000A8945170500200345A5F0829734
:1039700013452400B240224492444101828093972F
:10398000250163D80702B7E4040083A7C41E829709
:1039900097000000E780A0F0BC4C375607001306E4
:1039A00006308965170500200345C5EC8297096537
:1039B00079B7939715010145E3DE07FA17D50100A2
:1039C000130585AF97B00100E780A05EB7E704005C
:1039D000BC4F13060064916517050020034585E977
:1039E00082971165A9BF1D71A2CC37E404005C5C0D
:1039F000485886CE494697D50100938565A782979A
:103A000011E917D501001305E5A797B00100E7807C
:103A1000405A01A0B7F600E0795798CAFD57DCCAB2
:103A20000567B7E700E023A0E7101306F00290C295
:103A300023A0E718010001003707002018471306EC
:103A4000000481459706002023A4E6E24157A38A9B
:103A5000E7403C4408088297970700209387C77D7A
:103A60003EC8856713870740938757D1231AE10023
:103A70002312F1021307B00F97F7FFFF9387C76474
:103A80002310E1023ED81547970700009387C7E14E
:103A9000B7F50700A30FE1003EDC054797070000DC
:103AA0009387E7DF81463000E10519452301E102F4
:103AB0003EDE97F0FF1FE780C0D218088147994685
:103AC00030003E960346060085070507A30BC70096
:103AD000E398D7FEC24791C70357410185676373D7
:103AE000F70001A0B7E7040083A7470A08088297F8
:103AF000AA8511C917D501001305059A97B00100D1
:103B0000E780403301A0F640664425618280411180
:103B100026C2B7E4040083A7040806C622C417051A
:103B200000001305C5DF829717040020130484D416
:103B30002300A40097000000E780800297000000A7
:103B4000E780E0CC03450400224403A38405B2408F
:103B5000924413060032896541010283797106D6C9
:103B600022D413078008F337078093F787083EC2F3
:103B700001000100B7170040930570052380B704CA
:103B8000130680FA2380C7040100010083C6F702F0
:103B900093F6A60FA387D702238007049246F3A6C5
:103BA00006800100010073370780137787083AC445
:103BB000010001002380B7042380C7040100010035
:103BC00003C7F70213672700A387E70223800704D0
:103BD000A247F3A7078001000100054597E0FFFF1A
:103BE000E780807297000000E78060CB0147814644
:103BF0008147054685451305407E97E0FFFFE78036
:103C0000807537E404003C44680051468145829742
:103C1000B707C0A83EC8B787E803938707D03ECA56
:103C200097E7FF1F9387A7793EC67C586800829765
:103C3000B250225445618280411197D5010093858D
:103C400025E817C501001305257E06C697B00100BB
:103C5000E780401E17D501001305850297B00100CB
:103C6000E780401DB2402945410117B301006700BC
:103C70004321411197D501009385C5E517C5010082
:103C80001305857A06C697B00100E780A01A17D5FC
:103C900001001305A5FD97B00100E780A019B2400F
:103CA0002945410117B301006700A31D411122C43A
:103CB00006C6834705002A849DC797D501009385D2
:103CC00065EA17C501001305257697B00100E78066
:103CD00060164C4017D501001305050F97B0010081
:103CE000E78040153DA058410DEF97D50100938521
:103CF00065E717C501001305257397B00100E7803C
:103D0000601317D501001305A50D97B00100E780DA
:103D100060122244B2402945410117B301006700F7
:103D20004316A1679386D7036313D70297D5010083
:103D3000938545E317C501001305056F97B0010092
:103D4000E780400F17D501001305850A7DBFED07F9
:103D500097D50100938505E117C501001305C56CD2
:103D6000631BF70097B00100E780C00C17D5010076
:103D70001305450959BF97B00100E780A00B4C40DF
:103D800017D501001305050A91BF411106C622C4CB
:103D9000970700209387472F054717240020130417
:103DA000049A2392A7002390B7002391E7002310E1
:103DB000B40017C501001305256797D50100938549
:103DC00025D4972700202389E78697B00100E78054
:103DD00060068355040017D501001305650F97B0E1
:103DE0000100E78020052244B2402945410117B374
:103DF000010067000309411197D501009385C5CEE5
:103E000017C501001305456206C697B00100E7809B
:103E10006002B2402945410117B301006700630603
:103E2000797122D426D24AD02E842A898145B2843F
:103E30004800714606D697E0FFFFE780402D97F7D0
:103E4000FF1F93876758DC4783D70700231421019E
:103E50002313F10097500000E78060188547A30501
:103E6000F1009307401F3EC6FD572305A100230A1A
:103E7000F10097500000E780C02A2686A2854800FE
:103E800097500000E7808018B25022549254025993
:103E900045618280972700202393078A9717002087
:103EA000238C0778B7E70400FC47411106C641465A
:103EB00097D50100938585F817F5FF1F1305054E6B
:103EC000829717070020034767279307F00A6315B7
:103ED000F7029307F0F8894517050020130505261A
:103EE00017070020230CF72497070020A388072436
:103EF00097600000E78020D497600000E78080FF93
:103F00008145370504009707002023AF0720970756
:103F10000020239907209707002023860720970772
:103F2000002023950718970700202393071697076B
:103F300000202398071E970700202399071E97301B
:103F40000000E780005D014597600000E780A0D792
:103F500097D501009385C5BB17C501001305C54C56
:103F600097B00100E78000ED17D501001305C5F7F4
:103F700097B00100E78000ECB2402945410117B33A
:103F80000100670003F04111054506C69780010056
:103F9000E78060C929E58545814617F6FF1F1306AE
:103FA000E63E97C00000E780A05A97D501009385B0
:103FB000E5B62DC917C501001305054797B00100E7
:103FC000E78040E717D50100130505DC97B0010035
:103FD000E78040E6294597B00100E78080EA97F73F
:103FE000FF1F9387673EDC47054797D50100938500
:103FF000E5B22390E70017C501001305E54297B02D
:104000000100E78020E317D50100130565DA97B0BA
:104010000100E78020E2B2402945410117B30100C9
:10402000670023E617C501001305054097B001009E
:10403000E78040E017D50100130545D641BFB7E73B
:104040000400FC474111414606C622C426C24AC0AC
:1040500097D50100938585DF17F5FF1F13050534FC
:1040600082979707002083C7E7811707002003473F
:104070007781A207A166D98F1386E6FF7D8E13078D
:10408000001001CA1387F6FF7D8FD1476313F70035
:10409000554797D501009385A5A917C501001305BC
:1040A000A53897070020239FE70697B00100E78017
:1040B00060D89705002083D5E50617D501001305C4
:1040C00025DD97B00100E780E0D62945AD6497B0C3
:1040D0000100E78000DB371900409384A4AA232065
:1040E00099009706002093862604944297D70100F2
:1040F000938707E2170700200357C702170600201F
:1041000003466602814517F5FF1F130525299770A1
:104110000000E78080622320990097F7FF1F23911A
:10412000A71A2A8431C597D50100938565A017C5C4
:1041300001001305652F97B00100E780A0CFA2858D
:1041400017D50100130505D797B00100E78080CE91
:10415000294597B00100E780C0D29707002023933C
:1041600007FC2285B24022449244024941018280E8
:1041700097000000E78060E117F5FF1F1305052297
:1041800097200000E7802042E9BF011122CC06CE33
:1041900026CA4AC84EC693F715002E84BDC393079E
:1041A00010F817070020230BF7F89707002083D794
:1041B000A7ED914517050020130545F817070020C6
:1041C000A30EF7F6A18317070020230AF7F6970737
:1041D0000020A38607F697600000E780C0A597201F
:1041E0000000E780A023054597600000E780A0ADB0
:1041F00013451400F2406244D2444249B249056179
:10420000828093F72500E9CF17070020035787F135
:1042100069C7AD64B71900409384A4AA23A099008C
:1042200097060020938646F0944297D70100938723
:1042300027CE17060020034606EF814517F5FF1F1E
:104240001305C51597700000E780204F23A0990043
:1042500097F7FF1F2396A7062A8941C197D501002A
:104260009385C59517C501001305051C97B001007E
:10427000E78040BCCA8517D501001305A5C397B0D8
:104280000100E78020BB294597B00100E78060BFAF
:1042900097070020239807E8930710F817070020D6
:1042A000230EF7E89707002083D707DE17070020C3
:1042B000A306F7E8A183170700202302F7E891453A
:1042C0008D4717050020130565E717070020A30891
:1042D000F7E697600000E78000961345240019BFB9
:1042E00093F7051095C3AD67371700409387A7AACA
:1042F00017F5FF1F0355650F1CC397200000E780CB
:10430000604513450410FDB593F7052091CFAD67C7
:10431000371700409387A7AA1CC397200000E780A7
:10432000E01A13450420F9B593F74500D1C397D59A
:1043300001009385A58817C501001305E50E97B008
:104340000100E78020AF17C501001305A52597B030
:104350000100E78020AE294597B00100E78060B2F8
:10436000930720F817070020230AF7DC970700209F
:1043700083D7C7D317070020A302F7DCA183170751
:104380000020230EF7DA854717070020A309F7DA84
:1043900097500000E780E0D817050020130505DAE4
:1043A000914597600000E78000891345440099B566
:1043B00093F78500A9C797D501009385258017C578
:1043C00001001305650697B00100E780A0A617C598
:1043D00001001305651E97B00100E780A0A52945DF
:1043E00097B00100E780E0A997070020239C07D23F
:1043F00097700000E780404413458400E5BB93F7C5
:104400000501D1C3854517050020035525CA9760CE
:104410000100E78020F797C501009385257A17C52D
:1044200001001305650097B00100E780A0A017C543
:1044300001001305A51997B00100E780A09F294549
:1044400097B00100E780E0A3930730F8170700203A
:104450002306F7CE9707002083D747C5170700200C
:10446000A30EF7CC17050020130545CDA1838D457C
:10447000170700202305F7CC97500000E780A07BAA
:104480001345040185BB93F70502D1C797C5010009
:104490009385C57217C50100130505F997B0010092
:1044A000E780409917C501001305851497B00100F6
:1044B000E7804098294597B00100E780809C9307EA
:1044C00040F817070020230BF7C69707002083D773
:1044D00027BC17070020A303F7C6A18317070020F6
:1044E000230FF7C4854717070020A30AF7C49707CF
:1044F0000020239F07B897500000E78080C217056F
:1045000000201305A5C3914597500000E780A072D5
:1045100013450402C5B193F70504FDC397C5010017
:104520009385C56917C50100130505F097B0010013
:10453000E780409017C501001305050D97B00100F5
:10454000E780408F294597B00100E7808093970767
:10455000002083C7A7BE1307700A6386E706130708
:10456000800A638CE7081307600A6393E7049307E4
:1045700060F8170700202303F7BC9707002083D7B4
:1045800047BA17070020A30BF7BAA183170700202B
:104590002307F7BA854717070020A306F7BAB145E6
:1045A00017050020130585B997500000E780A06823
:1045B00097500000E780E0B61345040497070020F9
:1045C000239107B605B9930770F817070020230752
:1045D000F7B69707002083D7C7B417070020A30FAB
:1045E000F7B4A18317070020230BF7B485471707FB
:1045F0000020A307F7B4994565B7930780F8F1B792
:1046000093F705080145E38707BE97C50100938529
:10461000E55A17C50100130525E197B00100E780B1
:10462000608117C501001305A5FF97B00100E78061
:104630006080294597B00100E780A0849307A0F827
:1046400017070020230CF7AE9707002083D707AE8B
:1046500017070020A304F7AEA1831707002023004B
:10466000F7AE854717070020A30BF7AC970700208C
:10467000239E07AA97500000E780A0AA17050020F4
:104680001305C5AB914597500000E780C05A13450C
:1046900004088DB6411122C497C501009385C54D0C
:1046A0002A8417C50100130525D806C697A0010066
:1046B000E78040784C4017C501001305656A97A054
:1046C0000100E7802077294597A00100E780607B03
:1046D000034704009307F00F631FF70297C501001B
:1046E0009385854917C50100130505D497A00100DE
:1046F000E78040744C4017C501001305656797A01B
:104700000100E78020732244B2402945410117A3EC
:10471000010067000377B240224441018280B1C1A9
:10472000411122C417C50100130505D02E8497C579
:1047300001009385253C06C697A00100E780806FA5
:10474000A28517C501001305E57397A00100E78056
:10475000606E2244B2402945410117A30100670061
:1047600043728280B7E7040003A387051306001491
:104770009305001017F5FF1F034545100283B7E7A7
:10478000040003A38705130600149305002017F502
:10479000FF1F0345A50E0283011122CC37E404005C
:1047A0005C5C06CE26CA354697C501009385854ECA
:1047B00017D5010013054530829711E917C501008F
:1047C000130545CC97A00100E780A07E01A097F7D4
:1047D000FF1F9387670B3EC4B7F507008567938774
:1047E0000780814617F6FF1F13068609E105194564
:1047F0003EC697E0FF1FE780C0FE7C44194697F550
:10480000FF1F9385E507170500201305658A82972A
:10481000340017F6FF1F1306A60697D501009385EF
:1048200065A417D50100130565A597700000E78002
:10483000C0C52A8421C197C501009385253717C5B6
:104840000100130565BE97A00100E780A05EA28568
:1048500017C501001305054597A00100E780805D9D
:10486000294597A00100E780C061F2406244D2442C
:104870000561828097E00000E780C02817C501002D
:104880001305453997600000E780E0B997A0000064
:10489000E780007D97600100E78080E117F5FF1F4A
:1048A000130505AE97600100E78020CA17C5010017
:1048B0001305453797600100E78000E22A8497607E
:1048C0000000E780202097100100E78060B9978002
:1048D0000100E780805297700000E7802079977090
:1048E0000000E780209697300100E780C07A97C5E6
:1048F00001009385A52B17C501001305E5B219C862
:1049000097A00100E7800053A28517C50100130599
:10491000A53B99B797A00100E780C05117C50100DA
:104920001305C53C97A00100E780C0502D64B71463
:1049300000401304A4AA294597A00100E780605411
:1049400080C097300100E780E05580C097F00000FC
:10495000E7808074630705108545370504009730AC
:104960000000E78000BB97C501009385252417C58B
:104970000100130565AB97A00100E780A04B17C5A8
:1049800001001305253897A00100E780A04A2945BA
:1049900097A00100E780E04E97F7FF1F93874791AC
:1049A00083D7070017170020231BF7D88547171751
:1049B00000202303F7C897200000E780E0C397F0AA
:1049C000FFFFE780805C97200000E78020BC21E5A6
:1049D00097C501009385851717C501001305C5A468
:1049E00097A00100E780004517C501001305C533F6
:1049F00097A00100E7800044294597A00100E780C7
:104A0000404880C097700000E78000E380C097F0C6
:104A1000FFFFE780006397200000E78020A01715C4
:104A200000200355C5D197500000E78020F60545CA
:104A300097500000E780202997C50100938505174E
:104A400017C501001305459E97A00100E780803E31
:104A500017C501001305852F97A00100E780803D51
:104A600001B597500000E780002697F0FFFFE78030
:104A7000405D97200000E780609A55BF411122C435
:104A800037E404008327041A06C682979750000073
:104A9000E78080F38327040817F5FFFF1305256FD0
:104AA000829797F7FF1F238BA7DC17F5FF1F1305CE
:104AB000A59197500000E78060992244B2404101DF
:104AC00017030000670083CDB7E70400FC471171AE
:104AD000A2DDCAD986DFA6DBCED72E8432892E8608
:104AE000AA8517F5FF1F13056565829717F7FF1F46
:104AF0001307C76483470700930680029387E7077D
:104B000093F7F70FE3ECF610BA898A0717C701008D
:104B10001307C79ABA979C43BA9782878D4797C560
:104B200001009385E50A17C501001305E58F630FA2
:104B3000F40097A00100E780E02F17C501001305DE
:104B4000A5C497A00100E780E02EBDA497A00100B6
:104B5000E780402E17C50100130585C497A001000A
:104B6000E780402D294597A00100E7808031930719
:104B700020F8114697F5FF1F9385455C4A8517F786
:104B8000FF1F230DF75A97F7FF1FA38A075A97F0C5
:104B9000FFFFE78020292A841DC997C5010093855E
:104BA000250317C501001305258897A00100E7809C
:104BB0006028A28517C50100130545C297A0010012
:104BC000E7804027294597A00100E780802B97C503
:104BD00001009385E5FF17C501001305E58497A043
:104BE0000100E780202517C50100130565C097A0C7
:104BF0000100E7802024294597A00100E780602874
:104C00004165930730FA054697F5FF1F93850553D5
:104C10007D1517F7FF1F2303F75297F0FFFFE7807B
:104C200060202A841DC997C50100938565FA17B5D0
:104C300001001305657F97A00100E780A01FA285F2
:104C400017C50100130585B997A00100E780801EF4
:104C5000294597A00100E780C022B7E70400BC4FB8
:104C60000566130606C8A14517F5FF1F034505C1D4
:104C70008297FE506E54DE544E59BE5911618280A7
:104C800091476303F40297C50100938565F417B556
:104C900001001305657997A00100E780A01917C5E9
:104CA0000100130525B871BDB7E70400FC4F91451D
:104CB00017F5FF1F034585BC829797C501009385B3
:104CC00025F117B501001305257697A00100E780AF
:104CD000601617C501001305A5B697A00100E7806F
:104CE0006015294597A00100E780A01997400000B2
:104CF000E7802043914535A485476303F40297C5B7
:104D000001009385E5EC17B501001305E57197A047
:104D10000100E780201217C501001305E5B315B5A2
:104D200097F7FF1F23942739B7E704000566BC4FA8
:104D3000130606C8C1450DBF8D476303F40297C52E
:104D400001009385E5E817B501001305E56D97A00F
:104D50000100E780200E17C501001305A5B1D5B3EA
:104D6000930740F8114697F5FF1F9385253D4A8527
:104D700017F7FF1F2304F73C97F7FF1FA381073C9A
:104D800097F0FFFFE780000A2A84E30405EE97C549
:104D900001009385E5E317B501001305E56897A0C9
:104DA0000100E7802009A28517C50100130505A3AE
:104DB00097A00100E7800008294597A00100E7803F
:104DC000400C45BD9147E31CF4F6B7E70400FC4FE7
:104DD0009305000217F5FF1F034545AA829797C563
:104DE00001009385E5DE17B501001305E56397A083
:104DF0000100E780200417C50100130525A9F1BDB6
:104E0000894763E3870297C50100938565DC17B581
:104E100001001305656197A00100E780A00117C597
:104E200001001305E5A731BB97F4FF1F83C42431AC
:104E300097F7FF1F83C7973097C50100938545D922
:104E4000A20417B501001305255EDD8C97A00100B3
:104E5000E78040FEA28517C501001305A5A597A010
:104E60000100E78020FDC204294597A00100E780EA
:104E70004001C1849305D4FF93960401C1824A8600
:104E800093F5F50F17F5FF1F1305752B97200000FD
:104E9000E780E06BE35F90DC930750F817F7FF1FA4
:104EA000230EF72883C73900228697F5FF1F9385C5
:104EB000E52885074A8517F7FF1FA302F72897F013
:104EC000FFFFE78020F62A84E30505DA97C5010095
:104ED000938505D017B501001305055597A001006E
:104EE000E78040F5A28517C501001305A5F8C9B5EF
:104EF000894763E3870297C50100938565CD17B5A0
:104F000001001305655297A00100E780A0F217C5C4
:104F100001001305E59B35B197400000E780602054
:104F2000A28517F5FF1F1305652197500000E78044
:104F300080D081B38D476303F40297C50100938548
:104F400025C917B501001305254E97A00100E7807C
:104F500060EE17C5010013056599E5B6B766020056
:104F60000146B7750200054597E0FF1FE78060879F
:104F7000930760F817F7FF1F2302F71C97F7FF1F2F
:104F8000A38F071A9307000617F7FF1F230AF71AC4
:104F9000894717F7FF1FA305F71A97F7FF1F23820B
:104FA000071A97F7FF1FA38E0718C14717F7FF1FB0
:104FB000230AF718930720F917F7FF1FA304F71820
:104FC000314697F7FF1FA380A71897F5FF1F93851A
:104FD000E5164A8597F7FF1F2387071697F0FFFF0F
:104FE000E78040E42A84E30605C897C5010093855D
:104FF00025BE17B501001305254397A00100E780E2
:1050000060E3A28517C501001305C58F55B3B147ED
:105010006303F40297C50100938585BB17B50100B2
:105020001305854097A00100E780C0E017C5010087
:105030001305058F39B6B7E70400FC4F930500044C
:1050400017F5FF1F03458583829797400000E7808F
:10505000400DB145F9B5914763E3870297C501005B
:10506000938505B717B501001305053C97A001000E
:10507000E78040DC17C501001305458CD9B497F4CF
:10508000FF1F83C4E40B97F7FF1F83C7570BA204CE
:10509000DD8C8E04B77702006D14BE942286A6853F
:1050A00017C501001305C58A97A00100E78080D8C5
:1050B000B7E70400FC47228697F5FF1F9385550844
:1050C0002800829793160401C1823000A685094505
:1050D00097D0FF1FE780E0702A8409C917C5010037
:1050E0001305C58897A00100E780A0EC930770F82E
:1050F000194697F5FF1F938565044A8517F7FF1F2B
:10510000230EF70297F7FF1FA38C870297F0FFFF8C
:10511000E78040D12A84E30E05B497C5010093854A
:1051200025AB17B501001305253097A00100E780D6
:1051300060D0A28517C501001305458495B999472C
:10514000630BF41297C50100938585A817B501007C
:105150001305852D97A00100E780C0CD17C501007C
:1051600013054583F9BA914763E3870297C50100A8
:10517000938505A617B501001305052B97A001001F
:10518000E78040CB17C50100130545825DBA97F44F
:10519000FF1F83C4E4FA97F7FF1F83C757FAA204DF
:1051A000DD8C8E04B77702006D14BE942286A6852E
:1051B00017C501001305C58097A00100E78080C7CF
:1051C000B7E70400FC47228697F5FF1F938555F744
:1051D0002800829793160401C1823000A6850D45F0
:1051E00097D0FF1FE780E05F2A8409C917B5010047
:1051F0001305C57E97A00100E780A0DB930780F828
:10520000194697F5FF1F938565F34A8517F7FF1F2A
:105210002306F7F297F7FF1FA38487F297F0FFFFAB
:10522000E78040C02A84E30605A497C50100938562
:10523000259A17B501001305251F97A00100E780E7
:1052400060BFA28517B501001305857A95B6994709
:105250006303F40297C501009385859717B5010094
:105260001305851C97A00100E780C0BC17B501009D
:1052700013058579F9B0B7E70400FC4F93050004E6
:1052800017E5FF1F0345855F829797400000E78081
:1052900040E9994579B18D476303F40297C5010050
:1052A0009385059317B501001305051897A0010014
:1052B000E78040B817B501001305857659B017B5DA
:1052C00001001305E57697A00100E78080CE130565
:1052D000C01297D0FF1FE780C006014597E0FFFF8F
:1052E000E78080DB0D4597100000E780E09F2945AF
:1052F00097D0FF1FE780E00497D0FF1FE78040F5BD
:105300008DBA99476303F40297C501009385458CD4
:1053100017B501001305451197A00100E78080B182
:1053200017B501001305857129B817F7FF1F03474B
:1053300037E197F7FF1F83C7A7E022075D8F9166CC
:10534000BA96C2061166C1821306F6EF8D476365F1
:10535000D60297E7FF1F938727079C4B17F6FF1F7F
:105360000346F6DD9386C7002DC203D6070069CA3F
:105370008907E39CD7FE89471307A0F8114697F5E4
:10538000FF1F9385A5DB4A8597F6FF1F2388E6DA82
:1053900017F7FF1FA305F7DA97F0FFFFE78080A854
:1053A0002A84E308058C97C501009385658217B5AB
:1053B00001001305650797A00100E780A0A7A2855B
:1053C00017B501001305C568E5B203D60700630EE3
:1053D000E60A8907E39BF6FE8D4779BF9147630490
:1053E000F40297B501009385A57E17B5010013055A
:1053F000A50397A00100E780E0A317B501001305FE
:10540000A5666FF00FF4B7E70400FC4F93050008A2
:1054100017E5FF1F034585468297C9B897B5010078
:105420009385057B17B501001305050097A00100C2
:10543000E78040A017B50100130585646FF06FF099
:105440002390E70017E5FF1F130505F897300100CB
:10545000E780C0CA97B501009385857717B501002D
:10546000130585FC97A00100E780C09C17B50100DB
:105470001305056297A00100E780C09B294597A00E
:105480000100E78000A08147C5BD2390070017E514
:10549000FF1F130565F397300100E78020C697B51D
:1054A00001009385E57217B501001305E5F797A094
:1054B0000100E780209817B501001305E55E5DBF88
:1054C000411122C406C6834705002A849DC797B5AB
:1054D00001009385A56B17B501001305E5F497A0AE
:1054E0000100E78020954C4017C50100130545A336
:1054F00097A00100E7800094E1A05841B707CF00D2
:105500009387777D631DF70697B50100938505683E
:1055100017B50100130545F197A00100E7808091C0
:105520001C448356E4008355C40003C6070017C516
:105530000100130565A097A00100E780A08F294511
:1055400097A00100E780E0930357E400970700204D
:1055500083D7E71E6309F7008355C400084497E02A
:10556000FFFFE780E0C70356E4008355C40008440A
:105570002244B240410117F3FFFF67002355B707EC
:10558000CC009387777D6315F70497B50100938569
:10559000E55F17B50100130525E997A00100E78035
:1055A00060891C448356E4008355C40003C6070089
:1055B00017C501001305459897A00100E780808773
:1055C0002244B2402945410117A301006700638BC3
:1055D000B707CE009387777D6304F70297B5010084
:1055E0009385C55A17B50100130505E497A001007E
:1055F000E78040844C4017C501001305A582CDBD4E
:10560000B240224441018280B7E70400FC474111C7
:105610002E8606C622C426C24AC02E842A89AA859E
:1056200017F5FF1F130585B1829797B50100938584
:10563000E55B17B50100130525DF97900100E780B2
:10564000607F97F5FF1F83C565AF17B50100130590
:10565000A5FE97900100E780E07D294597A0010015
:10566000E780208297F4FF1F938444AD83C7040032
:1056700041479387070693F7F70F636EF75A17B7FB
:1056800001001307E7ED8A07BA979C43BA97828710
:105690009D476307F40297B501009385255517B51B
:1056A0000100130565D897900100E780A07817B531
:1056B00001001305E5F897900100E780A0778DA41D
:1056C00097F7FF1F83C797A7DDCB17F7FF1F034788
:1056D00017A797F7FF1F83C787A622075D8F97F746
:1056E000FF1F83C7E7A5C2075D8F97F7FF1F83C71B
:1056F00037A5E207D98F17F7FF1F2327F7A283C724
:10570000640097B501009385654E17B50100130538
:10571000A5D117F7FF1F2308F7A097900100E78096
:10572000607197F7FF1F938727A08C4317F6FF1F21
:105730000346669F17B50100130545F297900100D7
:10574000E780406F294597900100E780807397F7C5
:10575000FF1FA385079E2244B2409244024993074B
:1057600000F817F7FF1F230BF79C9D4517F5FF1F48
:105770001305C59C4101174300006700C34B9760A8
:105780000000E780E01A97F7FF1F238AA79A935734
:10579000850017F7FF1FA304F79A935705012A8482
:1057A00017F7FF1F230EF79893578501014517F749
:1057B000FF1FA307F79897600000E780E01897F7AE
:1057C000FF1F2380A79897B501009385254217B541
:1057D0000100130565C597900100E780A06517F6E5
:1057E000FF1F03460696A28517B50100130585E83D
:1057F000B1B7CD476303F40297B501009385053F28
:1058000017B50100130545C297900100E78080623B
:1058100017B50100130585E779BD37E404007C4422
:10582000414697F5FF1F9385759117E5FF1F1305F7
:10583000E5B6829797F7FF1F83C7679117F7FF1F9A
:105840000347D790A20703238405D98F17F7FF1FBB
:10585000231AF78C1306000A89452244B240924469
:10586000024917E5FF1F03456501410102838D478A
:105870006303F40297B501009385453717B501001E
:10588000130585BA97900100E780C05A17B501004B
:10589000130585EF0DB517F4FF1F0344448A97F7EE
:1058A000FF1F83C7B78997B501009385253422046C
:1058B00017B50100130545B75D8C97900100E7808F
:1058C0006057A28517B501001305C5DD979001004B
:1058D000E7804056294597900100E780805A0D46A1
:1058E00097F5FF1F93858585228597E0FFFFE78069
:1058F0006053AA8421C197B501009385252F17B560
:105900000100130565B297900100E780A052A685BB
:1059100017B50100130545DA97900100E780805123
:105920002244B240924402492945410117930100A3
:105930006700235597E7FF1F239A8776B7E7040090
:10594000116603A38705130606E8914539B78D470D
:105950006303F40297B501009385452917B501004B
:10596000130585AC97900100E780C04C17B5010086
:10597000130545F089B317E4FF1F0344447C97E700
:10598000FF1F83C7B77B97B50100938525262204A7
:1059900017B50100130545A95D8C97900100E780BC
:1059A0006049A28517B50100130545D29790010003
:1059B000E7804048294597900100E780804C0D46DC
:1059C00097E5FF1F93858577228597E0FFFFE780A6
:1059D0006045AA841DC197B501009385252117B59F
:1059E0000100130565A497900100E780A044A685F7
:1059F00017B501001305C5CE05B797E7FF1F23991B
:105A00008768B7E70400116603A38705130606E855
:105A10009305000299B5894763E3870297B50100B2
:105A20009385C51C17B50100130505A097900100CB
:105A3000E780404017B50100130585E6ADB997E44E
:105A4000FF1F83C4C46F97E7FF1F83C7376F97B5E6
:105A500001009385A519A20417B501001305C59C83
:105A6000DD8C97900100E780E03CA68517B501002A
:105A7000130585C897900100E780C03B29459790A2
:105A80000100E7800040228697E5FF1F9385056BA4
:105A9000268597E0FFFFE780E0382A84630E051A29
:105AA00097B501009385851417B501001305C597B7
:105AB00097900100E7800038A28517B50100130513
:105AC000E5C499BD854763F98718834519002244C9
:105AD000B24092440249B335B00097E7FF1F2381DB
:105AE000B75E17B501001305A5C341011793010067
:105AF00067004334A2852244B24092444A85024959
:105B00004101170300006700632499476303F4020F
:105B100097B501009385850D17B501001305C59054
:105B200097900100E780003117B50100130505F1DA
:105B300059B617E4FF1F0344846097E7FF1F83C72C
:105B4000F75F97B501009385650A220417B5010038
:105B50001305858D5D8C97900100E780A02DA285AF
:105B600017B50100130545BD97900100E780802C13
:105B7000294597900100E780C030194697E5FF1F3F
:105B80009385C55B228597E0FFFFE780A029AA8463
:105B90001DC197B501009385650517B50100130573
:105BA000A58897900100E780E028A68517B5010039
:105BB000130585B995B397E7FF1F23998756B7E774
:105BC0000400116603A38705130606E89305000881
:105BD00069B1854797B501009385450117B5010067
:105BE00013058584630BF40097900100E7808024FF
:105BF00017B50100130585B67DBC97900100E780BD
:105C0000602317B501001305E5B697900100E78002
:105C10006022294597900100E780A0262244B240E7
:105C20009244024997E7FF1F239E074E41011763E5
:105C30000000670063C097B50100938525FB17A599
:105C400001001305657E97900100E780A01E17B53F
:105C500001001305E5E285B4B240224492440249B2
:105C600041018280411106C622C497E0FFFFE78010
:105C7000601B21CD97E7FF1F83D7A74485072A84A0
:105C800017E7FF1F231FF74297B50100938585F79C
:105C900097E7FF1F2398A74217A501001305C578B2
:105CA00097900100E7800019A28517B50100130540
:105CB000651C97900100E780E0172244B240294517
:105CC0004101179301006700C31B97E7FF1F83D7AC
:105CD000873FB2402244850717E7FF1F2315F73E91
:105CE00041018280411122C491462A8417E6FF1F98
:105CF0001306C6529D652D4506C697D0FF1FE78047
:105D000040AEB7F7070003C70701A5476313F700C5
:105D100001A09306001001469D65254597D0FF1F01
:105D2000E78020AC97E7FF1F238A874E2244B240CA
:105D3000914617E6FF1F1306664E9D6529454101F2
:105D400017D3FF1F6700E3A91171CED7B7E904008D
:105D500083A7C904CAD917E9FF1F1309293EA2DD89
:105D60002E8686DFA6DB2E84AA854A85829797E752
:105D7000FF1F83C7A73C1307700A6385E710636D95
:105D8000F7001307600A6385E704FE506E54DE5483
:105D90004E59BE59116182801307800A6385E71648
:105DA0001307900AE393E7FE8D476306F41C97B54B
:105DB00001009385E52317A501001305E56697907B
:105DC0000100E780200717B501001305A51F25A0D6
:105DD0008D47630CF40297B501009385652117A5E3
:105DE00001001305656497900100E780A00417B5D2
:105DF00001001305651697900100E780A00329456F
:105E000097900100E780E00749B7854717B5010083
:105E10001305451617E7FF1F2304F72A9790010083
:105E2000E7802019B7750200B766020001460545F4
:105E300097D0FF1FE780E09A930760F817E7FF1FEE
:105E4000230EF72E97E7FF1FA38B072E930700263D
:105E500017E7FF1F2326F72EE5779387072117E71C
:105E6000FF1F2311F72EB14597E7FF1F238D072C46
:105E700097E7FF1FA389A72C4A8597000000E780BA
:105E8000E01621B7914763E3870297B50100938538
:105E9000251617A501001305255997900100E780E5
:105EA00060F917B501001305E50EB1B797E4FF1FC0
:105EB00083C4042997E7FF1F83C77728A204DD8CDA
:105EC00083A7C9046D14228697E5FF1F9385552784
:105ED000280082978E0493160401B7750200C182D0
:105EE0003000A695094597D0FF1FE780808F930764
:105EF00070F817E7FF1F2303F724994597E7FF1F63
:105F0000A380A72495BF914763E3870297B501005B
:105F10009385050E17A50100130505519790010003
:105F2000E78040F117B5010013054508E9B597E48E
:105F3000FF1F83C4E42097E7FF1F83C75720A204F5
:105F4000DD8C83A7C9046D14228697E5FF1F938516
:105F5000351F280082978E0493160401B77502003E
:105F6000C1823000A6950D4597D0FF1FE78060875E
:105F7000930780F8BDBF17B501001305E50597909D
:105F80000100E7800003930790F82304F1008347A2
:105F900019008D452800A304F1008347290023053B
:105FA000F10097000000E78060041305C01297C05D
:105FB000FF1FE7800039014597D0FFFFE780C00D44
:105FC0000D4597000000E78020D2294597C0FF1FAC
:105FD000E780203797C0FF1FE78080277DB397E7D2
:105FE000FF1F23A5A724828097E7FF1F938707241D
:105FF00003A3070063030300028317430000670045
:1060000083C341114AC097F6FF1F83D64673328976
:1060100017D6FF1F0356663D22C426C206C62A8431
:10602000AE8497000000E780006A35C12DC0994713
:1060300063FF97048347140003470400A207D98F26
:1060400013978700A183D98FC2073167C1831307D4
:10605000C755639EE70297D7FF1F83D70739A30170
:10606000F400A1832302F40097F7FF1F83D7276D65
:1060700091C7A302F400A1832303F400A68517B5FA
:1060800001001305E5FA97900100E780A0DA97F781
:10609000FF1F83C7675AA5C797D5FF1F83D5E53470
:1060A00017B50100130585FA97900100E78080D8A5
:1060B0002686A28517D5FF1F0355253397000000BC
:1060C000E78080BA6306090497F7FF1F83C7C756A6
:1060D000A1E397E7FF1F83C7E7159DCB95C897E717
:1060E000FF1F83C7E7FD8DE722852244B2400249A6
:1060F000A68592444101174300006700C3B317B55A
:1061000001001305A5F597900100E78080EA5DBFC7
:10611000B2402244924402494101828083475500A3
:106120008345450017B50100130545EFA207DD8D36
:1061300017930100670003D017B50100130505EDA3
:10614000179301006700E3E68D4763FBB70A01116F
:1061500026CA06CE22CC0344350097E4FF1F83C431
:10616000740D97B50100938525F0B337800017E7CC
:10617000FF1FA301F70C09C497B50100938585EFB4
:1061800017B50100130585EF97900100E78080CADD
:1061900097E7FF1F83C7170A6386970097E0FFFF03
:1061A000E780205E97E7FF1F83C7D7088DC7854725
:1061B0002306F100B7E7040083A747177000854561
:1061C00013055030829717B50100130525EC979001
:1061D0000100E78000DE9967938757EE2316F100F0
:1061E000680085479145A30781002307F1009700C8
:1061F0000000E780A0DFF2406244D2440561828063
:106200008280894763FCB708011122CC06CE834700
:10621000250005472A846393E706914763FCB7048A
:106220008347450003473500A207D98F17D7FF1FC3
:106230000357A71B630AF70017D7FF1F2317F71A87
:1062400097E0FFFFE78040529967938767EE23143A
:10625000F10085472305F10083473400A305F100D1
:1062600083474400954528002306F100970000006D
:10627000E780C0D7F240624405618280E5FF9967FC
:10628000938767EE2314F10097D7FF1F83D7E71595
:10629000A305F10023050100A183E9B78280011164
:1062A000996722CCD51717F4FF1F1304E438231481
:1062B000F1008347040026CA97F4FF1F9384244803
:1062C0002305F10083D7040028009545A305F100BC
:1062D000A18306CE2306F10097000000E78000D1DD
:1062E00003D604008345040017B50100130585DBC0
:1062F00097900100E78000B4F2406244D244056107
:1063000082809D677971D9172316F10097F7FF1FD7
:1063100083C7873206D62307F100A9C3B7E7040075
:10632000FC47414697D5FF1F938545071305F100AC
:1063300082976800CD4597000000E78020CB97F555
:10634000FF1F83C5652F17B501001305A5D89790CA
:106350000100E78020AEB25045618280B7E70400BB
:10636000BC47414681451305F1008297D9B745C521
:10637000411106C622C4930750FA2300F500930783
:10638000A005A300F50089472301F5009147A3016B
:10639000F50093073004A302F50097F7FF1F9387DA
:1063A000A72983C70700230205002A842303F500D9
:1063B00097E7FF1F938717E883C70700414697D5E4
:1063C000FF1F9385A5FDA303F50097F7FF1F83D754
:1063D00007372304F500A183A304F50097D7FF1F17
:1063E00083D7A7002305F500A183A305F500B7E730
:1063F0000400FC47310582972285F1459700000093
:10640000E7806028230EA4002181A30EA400B240DF
:1064100022444101828082805D710A8586C6A2C4C1
:1064200097000000E780E0F437E404007C448A85AC
:106430000810794682973C441305E10309468145DB
:106440008297101093050002014597D0FFFFE78067
:10645000E02AB640264461618280011122CC2D647D
:1064600026CA4AC84EC652C456C25AC006CEB7142F
:1064700000401304A4AA80C037E900E0B709400037
:106480002A8AAE8A328B23203919010001008566E1
:10649000AA850146254597C0FF1FE7808034DA862C
:1064A0005686D285294597C0FF1FE7808033232079
:1064B000391180C0F2406244D2444249B249224A72
:1064C000924A024B056182800111B7C7A55A22CCBE
:1064D0009387C73317E4FF1F1304D4D53EC4834703
:1064E00004002C002146196506CE3EC69700000028
:1064F000E780E0F68345040017B50100130545CD9C
:1065000097900100E7800093F24062440561828029
:106510000111A146300099652D4522CC06CE97C0C9
:10652000FF1FE780002CA24737C4A55A1304C433C9
:1065300063958702B24517B501001305E5BBB33576
:10654000B00097E7FF1FA387B7CE97900100E780C1
:10655000608EF2406244056182809165A146300000
:10656000938505F02D4597C0FF1FE7808027A24740
:10657000E38287FC97E7FF1FA38E07CA814517B503
:1065800001001305A5B9D1B797E7FF1F938747CA45
:106590008843B7D7CBA99387F7FC3E9513351500F1
:1065A0008280B7C7A55A79719387F7353EC4B7E79C
:1065B0000400FC4706D6AA85414668008297B73793
:1065C0003456938717032C00614611653ECE17E7BA
:1065D000FF1F232FF7C497000000E78040E817B59E
:1065E00001001305A5C297900100E780809CB2507E
:1065F000456182807971E146300091652D4522D454
:1066000097E7FF1F23A607C206D697C0FF1FE780A4
:10661000401DA24737C4A55A1304F435639D870271
:10662000B7E70400FC476C0017D5FF1F130505D71B
:1066300041468297F24517B50100130525B497E747
:10664000FF1F23A7B7BE97800100E780A07EB2504E
:106650002254456182809165E1463000938505E8CA
:106660002D4597C0FF1FE780C017A247E38A87FA2E
:1066700017B50100130545B397900100E7806093BB
:10668000F9B7C16769768146FD17050613970601BC
:1066900041836364B7003E8582803307D50003479A
:1066A0000700B98F214713F8170085836305080099
:1066B000B18FC207C1837D171377F70F6DF785067A
:1066C000F1B741C5A547054763F2B70883471500F1
:1066D000034705003168A207D98F13978700A1836C
:1066E000D98FC207C1831308C855054763900707B0
:1066F000411106C622C426C203442500914763F017
:1067000087049307540063ECF502A301C5002182BE
:106710002302C5009304340091C6A302D500A182D0
:106720002303D5002A84A68597000000E780A0F502
:1067300026942300A4002181A300A4000147B240B5
:10674000224492443A854101828005473A858280FD
:106750000111B7C7A55A22CC9387E7342A842AC6E9
:1067600021462C00156506CE3EC497000000E78048
:1067700000CFA28517B50100130585A797800100FA
:10678000E780406B97000000E78040C9F240624418
:10679000056182800111A146300095652D4522CC0E
:1067A00006CE97C0FF1FE780C003A24737C4A55A93
:1067B0001304E43463958702B24517B5010013054D
:1067C000E59797D7FF1F2392B7C2C205C181978073
:1067D0000100E7802066F240624405618280916595
:1067E000A1463000938505EE2D4597C0FF1FE78039
:1067F00040FFA247E38287FCD14717D7FF1F23162C
:10680000F7BED14517B5010013054595C9B721C19C
:10681000411126C206C622C4AE848DC52A849700C3
:106820000000E780E06697E7FF1F83C7A7A099CB2A
:1068300022852244B240A6859244410117330000CC
:106840006700633FB24022449244410182808280CB
:1068500001114AC806CE22CC26CA4EC693F71500AF
:106860002E899DCBAD67371700409387A7AA1CC31D
:10687000B7E70400BC4F13060019854517D5FF1F65
:10688000034585B6829713451900F2406244D2440D
:106890004249B2490561828093F72500638A071C4B
:1068A00017F7FF1F035787E9954763F9E70C014482
:1068B00017F6FF1F130686D89306300513055004FC
:1068C000130810049308B0041303900593076400A1
:1068D0006374F7043A84FD5997F4FF1F83C404D608
:1068E00097F7FF1F83C797D5A204DD8CAD67938709
:1068F000B755638BF41463E3970AA9679387A75589
:10690000638EF414A28517F5FF1F130525D3970096
:106910000000E78000F031A2B307860083C50700BE
:10692000639AD50483C517006396A50483C5270021
:106930006392050583C53700639ED50283C5470072
:10694000639A150383C7570063966702A2890DE80F
:1069500097F5FF1F83D585DEB3853541C20517F551
:10696000FF1F1305A5CDC1814E9597000000E7805C
:1069700040EAE1A005044204418089BF3A84FD5900
:106980008547E3EB87F45DC4854517F5FF1F1305C5
:10699000E5CA97000000E780C0E769A8B167938760
:1069A000C7556380F404B5679387D755E39CF4F427
:1069B000A28517F5FF1F130565C897300000E78013
:1069C00080278947630FF4049305E4FFC205C18162
:1069D00017F5FF1F1305A5C697000000E780404B81
:1069E00089A097200000E780801197000000E780D1
:1069F000804911C9A28517F5FF1F130525C497000B
:106A00000000E780E0480546A28517F5FF1F130543
:106A1000E5C297F0FFFFE780005F97200000E78066
:106A2000000EA68517B5010013054580978001006B
:106A3000E7804040FD57E39DF9F097F7FF1F239F44
:106A400007CE1345290091B5A28517F5FF1F130541
:106A5000E5BE97F0FFFFE780A06CE1B7A28517F5D0
:106A6000FF1F1305A5BD97F0FFFFE780206D55BF01
:106A700093F745000145E38A07E017A501001305D8
:106A8000257C97800100E780C05297300000E780A6
:106A9000204813454900D5BB411122C437E4040006
:106AA0005C5C06C6354697A501009385A51E17B503
:106AB000010013056500829711E917A50100130570
:106AC000E57897800100E780C04E01A08327041C71
:106AD00082972A84054597C00000E78000029770DE
:106AE0000100E780208797600100E780205C97B075
:106AF0000000E78080132285B24022444101828059
:106B00004111054506C622C426C297C0FFFFE78093
:106B100080421305A00497B0FF1FE78040597575A8
:106B200085457D1597C0FFFFE780202C7D75854545
:106B30001305F53697C0FFFFE78080353714004016
:106B40008327840A8D451305002093E7072023241B
:106B5000F40A97C0FFFFE7804029B7E4040097C01C
:106B6000FFFFE780606EC85897800100E7806044AF
:106B700017B50100130545F497800100E7806043D5
:106B80008327840C8545414593E707082324F40CAB
:106B900097C0FFFFE780C02F8D451305000897C001
:106BA000FFFFE780E02E97C0FFFFE780C05B37A5BF
:106BB00007001305051297C0FFFFE78060570145E6
:106BC00097C0FFFFE780805D95450545894717F72A
:106BD000FF1F2307F7B697C0FFFFE780C05DB7E749
:106BE00000E013070006238DE7403707000423A0C9
:106BF000E71097D0FFFFE78040DF97D0FFFFE780E7
:106C000040F197000000E78060E997000000E7800E
:106C1000609097000000E78020B897E0FFFFE780D2
:106C200020E697000000E780E02797000000E7805B
:106C3000E01083A70408170500001305A5C182977B
:106C400097C7FF1F2382A77ABC4C130600648545B3
:106C5000829797B0FF1FE780A079014582807D77FA
:106C6000B377E500AA9563E9F5048566FD16AE964F
:106C700041119D8E06C622C426C2F98E91E2856618
:106C80002D67371600401307A7AA18C237E400E0A3
:106C9000B704400023209418010001000146BE857E
:106CA000254597C0FF1FE780C0B3B2402320941052
:106CB00022449244410182807D5582804111B286F6
:106CC0002E86AA852D4506C697C0FF1FE78060B1B6
:106CD000B2400145410182809307000463ECC70480
:106CE0001D71A2CC2A840808A6CACAC886CE32C69C
:106CF00097800100E780A008AD67371700409387B1
:106D0000A7AA1CC3B7E400E03709400023A0241958
:106D100001000100B2461008A285294597C0FF1F57
:106D2000E78020ACF640664423A02411D6444649AF
:106D3000256182803955828041110D658D4506C6D9
:106D400097C0FFFFE780600AB71700408D6623A653
:106D5000D70A17F5FF1F1305E59E1387C70A938708
:106D6000870A1CC15CC5856689675CC958C114C5A2
:106D700018C9B7E70400B24003A3871E410102838C
:106D80008145B307B5008387070089E71723000013
:106D9000670083DD8505C205C181E5B797A70100BE
:106DA0009387876C1357C5003E970347070001116F
:106DB00006CE2304E100135785003D8B3E97034721
:106DC000070023060100A304E100135745003D8B93
:106DD0003D893E97AA970347070083C7070028000D
:106DE0002305E100A305F10097000000E78080F98A
:106DF000F24005618280411126C2E97797F4FF1FB6
:106E00009384C4A422C49387A7552E842381B400FD
:106E10002E86AA8517F5FF1F130585A306C62390A6
:106E2000F400A381040097800100E78040F59305FA
:106E30002400C205C18117F5FF1F130545A1970066
:106E40000000E7804084B38784002382A70021816B
:106E5000A382A700930564002244B2402685924491
:106E6000C205C1814101172300006700E3CF09C9B2
:106E70009307800263E6B700170300006700E3F79B
:106E8000828017F5FF1F0345658D828097F7FF1FEE
:106E900083C7879B89E7172300006700E3CC8280C4
:106EA00097F7FF1F83C7679D99EF411106C697208B
:106EB0000000E78040C3B240854717F7FF1F230E4D
:106EC000F79A4101828082806302056463800564D1
:106ED0005D71A2C4A6C286C6CAC04EDE52DC56DAB6
:106EE0005AD85ED662D466D26AD0B9472A84AE84B4
:106EF00063F9B706394697A501009385653E9780EB
:106F00000100E78060E531ED8347E40013071003DB
:106F10006394E702854717F7FF1F2307F79217A52A
:106F200001001305E53C97F7FF1F239E079097008C
:106F30000000E78020E571A01307000317A50100FA
:106F40001305053EE395E7FE97F7FF1F238E078E97
:106F500097F7FF1F2399078E17A501001305C53A60
:106F6000F9B797F7FF1F83C7278E63890722BD6A8A
:106F7000B96B938CFA55014A17EBFF1F130B4B7E2D
:106F8000138CEB65938AFA6605A8B307440183C6A0
:106F9000070097F7FF1F83D7078BB1E39307A0057F
:106FA000639BF600854717F7FF1F231EF78897E7B7
:106FB000FF1F2387D77A050A93170A01C183E3E6E7
:106FC00097FCB640264496440649F259625AD25A72
:106FD000425BB25B225C925C025D61618280054D26
:106FE000639BA7039307500A639EF600894717F730
:106FF000FF1F231AF784930750FA17E7FF1FA30117
:10700000F77655BF9307A005E387F6FA97F7FF1FBA
:10701000239B07824DB7138717004207DA974183F6
:107020002380D70017F6FF1F231FE6808D47E3F468
:10703000E7F817E9FF1F0349D97297E7FF1F83C7D6
:10704000477222093369F9009307F9FFC207C18328
:107050009306F00DE3ECF6FA93076900C207C183CB
:10706000E31BF7F493052900C205C18117E5FF1F53
:107070001305256F97F0FFFFE780E06033072B01D2
:107080008347570003474700A207D98F17E7FF1F21
:10709000231B077A6319F50E8149630DA90197E94E
:1070A000FF1F83C9296CA20997E7FF1F83C7976B4E
:1070B000B3E9F900170500001305A5DB97F0FFFF02
:1070C000E78020F263878907636D3C039387EB5564
:1070D0006382F90497E7FF1F83C7C7680547638981
:1070E000E70681CB1387A7051377F70F8D4663F269
:1070F000E6081307F0072300E100A300F10089452B
:107100009DA063829905E39759FD97F0FFFFE78003
:10711000801F11A8CA8517E5FF1F1305A56497F006
:10712000FFFFE780A002014597F0FFFFE78060EBDB
:1071300059B5CA8517E5FF1F1305C56297F0FFFF14
:10714000E780600CCDB797F0FFFFE7808015E1BFC7
:10715000930710F8130511002300F10097F0FFFFCB
:10716000E7802021FD450A8597000000E780E0C800
:107170005DBFCA8517E5FF1F1305C55E97F0FFFFCA
:10718000E780C0BC4DB79307F00789450A852310F7
:10719000F10097000000E78040C631BDBD4763F0B5
:1071A0009724414697A501009385C51922859780AC
:1071B0000100E78060BA6316052217A501001305D8
:1071C000A51997000000E780E0BB17E5FF1F0355F6
:1071D000055797000000E780A0BC97E7FF1F83C713
:1071E000A74517A501001305250D89E717A501007F
:1071F0001305050D97000000E780C0B817A5010032
:107200001305051797000000E780C0B717C5FF1FDB
:107210000355451B97000000E78080B8054597504F
:107220000100E78040A02A8417A501001305C509C5
:1072300009E417A501001305E50997000000E780A0
:1072400060B4630504188347640003457400A20713
:107250005D8D97000000E780A0B48347840003455C
:107260009400A2075D8D97000000E78060B317A52A
:1072700001001305E51097000000E780A0B017C5D6
:10728000FF1F0355851697000000E78060B117A522
:1072900001001305650F97000000E780A0AE17D529
:1072A000FF1F035545E297000000E78060AF17A578
:1072B00001001305E50D97000000E780A0AC17D58D
:1072C000FF1F035505E097000000E78060AD17A59C
:1072D00001001305650C97000000E780A0AA17D5F0
:1072E000FF1F035525DE97000000E78060AB17A560
:1072F00001001305A50A97000000E780A0A89740A9
:107300000000E780E062418197000000E78040A92B
:1073100097400000E780C06142054181970000006E
:10732000E78000A817A501001305C5079700000016
:10733000E78040A597400000E780406041819700CA
:107340000000E780E0A597400000E780205F42054D
:10735000418197000000E780A0A417A50100130554
:10736000E50497000000E780E0A117C5FF1F035563
:1073700025F597000000E780A0A217A501001305DE
:10738000650397000000E780E09F97C7FF1F83C752
:10739000E700A20717C5FF1F034555005D8D970045
:1073A0000000E780E09F97C7FF1F83C747FFA20742
:1073B00017C5FF1F0345B5FE5D8D97000000E780F0
:1073C000209E179501001305256195B617A50100AC
:1073D000130545FA97000000E780C09A49BD639005
:1073E000F4123D4697A50100938505FD22859780FF
:1073F0000100E78060964DE5C514C2041306F40051
:10740000C1804D0481470D45254895456379950018
:10741000631C86001397070141876348E00417A5A2
:107420000100130565FA21B603470600930607FD20
:1074300093F6F60F637CD8009306F7FB93F6F60FEE
:1074400063ECD500130797FC9376F70F9207D58F5F
:10745000C207C18305065DBF9306F7F993F6F60FE1
:10746000E3EFD5FA130797FAC5B717C7FF1F0357FE
:10747000C7F7630AF70017C7FF1F2318F7F697D05F
:10748000FFFFE780602E17A50100130525F6970082
:107490000000E780208F17C5FF1F035505F531BF9A
:1074A000C14763FE9704414697A50100938545F5C2
:1074B000228597800100E780208A31E1834704011B
:1074C00013071003639CE700854717E7FF1F230797
:1074D000F72817A501001305E5F391BC1307000376
:1074E00017A50100130505F6E393E7A497E7FF1F2F
:1074F0002386072617A50100130545F30DBCA685B5
:10750000228597C0FFFFE780A0CD65BC8280411136
:1075100026C2AE848D4522C406C62A8497C0FFFFCA
:10752000E7800097B717004099C803A5C70C418DA5
:1075300023A6A70CB240224492444101828003A5B5
:10754000870C418D23A4A70CF5B78347050003479B
:107550001500A207D98FC2076177C18713072720BB
:10756000639AE700834525003705040017030000F0
:10757000670023FA828017E6FF1F130666308147F3
:10758000B2861303F00FA9483308F6000348080039
:1075900013F7F70F6307A80C630668008507E395E8
:1075A00017FF2947B387E6002380A70097E7FF1F4F
:1075B0009387C72D5DA8411113D7650013471700A6
:1075C00006C693F63500058B954791CA054699473F
:1075D0006387C60009469D476383C600A14713F62B
:1075E00045003336C00093F68503050685C2A145E4
:1075F000638BB604E145638AB60493058002638811
:10760000B604930580036393B600914697E5FF1F88
:107610002383F54E97E5FF1F238EC54C97E5FF1F8B
:10762000A38AD54CBE8517A501001305E5E7978011
:107630000100E7802080B240854717E7FF1FA30CB9
:10764000F74A410182808546D1B78946C1B78D4648
:1076500075BF17A501001305A5E7177301006700A3
:10766000637D17E7FF1F13076722BA972380B700D0
:10767000E147E302F5F493077002E30CF5FC828026
:107680002A8723800500814717E5FF1F1305451F43
:107690001308F00F2946B306F50083C6060063966B
:1076A000E60297E6FF1F9386661EB69783C707001C
:1076B00005452380F5009947636EF7029D4763FDFA
:1076C000E700E147630DF7008280638506018507C7
:1076D000E393C7FC0145C5B7238005008280B73717
:1076E000004003C7370083C7050093F70704D98F0D
:1076F0002380F50082805D7152DC56DA5ED6716AB5
:1077000097EBFF1F938B4B508D6AA6C24EDE62D45F
:1077100086C6A2C4CAC05AD866D26AD06ECEC14943
:107720005E8C97E4FF1F93842417130A0A20938A20
:107730007ADC17E9FF1F03492950B3872B0183C760
:10774000070093F7F70FC9EFB787004003C767003B
:10775000058BE310077C03C76700118BE30D077EE1
:1077600083C75700918B99E36F10200317E7FF1F22
:107770000347A74C85476304F7006F10400197E764
:10778000FF1FA38AE73697E7FF1F2387071C97E7AA
:10779000FF1F2385072897E7FF1F2383073497E7F9
:1077A000FF1F2380073497E7FF1FA387071A97E778
:1077B000FF1FA385072697E7FF1FA383073297E7DD
:1077C000FF1FA380073297E7FF1FA387073297E7C2
:1077D000FF1FA3840746B787004011476F007077EB
:1077E0009307190093F7F70F3D476364F70617E710
:1077F000FF1F2303F74497E7FF1F9387E742CA97CA
:1078000083C707001307100293F7F703638EE71E81
:107810006366F70405446385871CE38C07620947A8
:10782000638EE71013070002E384E74EB7E700E03A
:107830003707400023A0E7180100010062992300E8
:107840000900FD1923A0E71093F9F90FE39309EE5E
:10785000E5BD97E7FF1F2381073E71BF1307300285
:107860006388E70C63E8E71613074002638CE70AB6
:1078700013070003E39CE7FA97E7FF1F9387C739D5
:10788000CA9703C70700A1471377F70FE31BF71445
:1078900083C7640097E6FF1F2386F62497E7FF1F40
:1078A00083C7F7FF91C7FD5797E6FF1F238CF6228A
:1078B00097E5FF1F83C555FE97E7FF1FA384B722F7
:1078C00097E7FF1F83C747FD13FB070893060004D4
:1078D00093F70706639FD74C9307A009638DF516AE
:1078E00063EAB7129307F0056386F54A93075009D8
:1078F0006384F52A014497E7FF1F83C7B71E154726
:10790000E392E736B7E700E03707400023A0E71827
:1079100001000100B786004023808602130680FC28
:107920006F00500EFD5717E7FF1F230CF71AFDBD20
:10793000FD5717E7FF1F2305F71ACDBD17A5010057
:10794000130585CA97700100E780A06697E7FF1FBF
:107950009387872CCA9703C40700014B97ECFF1F3E
:10796000938C0C0C1374F40F17AD0100130D4DC85C
:1079700063478B04294597700100E7808050854755
:1079800017E7FF1FA30CF70817E7FF1F2309870856
:1079900017E7FF1F2302F71637E700E0B70640009E
:1079A0002320D71801000100378600408347A60234
:1079B00093F7370F2305F6022320D71085BDB38731
:1079C0006C0183C507006A85050B97700100E7808D
:1079D000604679BF854717E7FF1F2301F704B9B554
:1079E00017E7FF1F130747234A970347070097E648
:1079F000FF1FA383F6F697E6FF1F2380E6F617E73F
:107A0000FF1F230BF70E1DB5854717E7FF1F230543
:107A1000F7F429BD9307400A6389F5349307200BD7
:107A20006384F5369307100AE396F5EC8387240008
:107A30000144E3D207EC97E7FF1F83C717E693F6ED
:107A40003700638A061A0546638AC622094663958B
:107A5000C61A1D4755A217E5FF1F034505E4C94790
:107A600097ECFF1F83CC7CE397E5FF1F83C505E3FD
:107A700017E4FF1F034494E26315F510CD476392AA
:107A8000FC1093077008639CF5021307300FB717BB
:107A90000E006308E4001307900DB7B704006314E9
:107AA000E40817E7FF1F2325F704BE8517A501008B
:107AB000130585B497700100E780C03725BD930793
:107AC0008008639DF500B307804013F4F70FB77784
:107AD0004600938787CDB3D78702E1B79307900815
:107AE000639AF500B307804013F4F70F916793870B
:107AF000C766D5B79307A008639BF500B30780401E
:107B000013F4F70FB7173D0093870790E9B7930772
:107B1000B008639AF500B307804013F4F70F91673C
:107B2000938797D04DBF93F5F5078D47639BF5007D
:107B3000B307804013F4F70FB7975B00938707D81C
:107B400059BF8947639BF500B307804013F4F70FD3
:107B5000B7770B009387071BBDBF8547639AF50076
:107B6000B307804013F4F70FDD67938767E3A5B78A
:107B7000D28785F9B307804093F7F70FB3D7FA029E
:107B80000DB797000000E780409FA28566859700AB
:107B90000000E780809EB9BB9305610017E5FF1FD9
:107BA0000345A5CF17E4FF1F034434CF970000001F
:107BB000E78040AD93057100228597000000E780C3
:107BC00060AC3C0017E7FF1F232EF70283476100DC
:107BD0002304F10083477100A304F100894717E7EC
:107BE000FF1F2301F7F08357810017E7FF1F2315BD
:107BF000F7CA094409B3154793F64700B336D000D6
:107C000093F78703850685C32146638BC7066146C4
:107C1000638AC706130680026388C70613068003BB
:107C20006393C700914717E6FF1F2305D6EC97E63D
:107C3000FF1FA381F6EC97E7FF1F238EE7EA17E704
:107C4000FF1F0347A7C59376070497E7FF1F83C766
:107C5000F7C48DEE1377770C93067008630CD70288
:107C60001377F7078D466312D70CB307F040B7952B
:107C70005B0093F7F70F938505D849A81947ADBF67
:107C8000854755B7894745B78D4771BF930670083B
:107C90006311D7021307300FB7150E006389E7028F
:107CA0001307900DB7B504006383E702130770084C
:107CB00045BF9306800C6311D702B307F040B77538
:107CC000460013F7F70F938785CDB3D5E70297E703
:107CD000FF1F23AFB7E0D9BB9306900C631CD700FE
:107CE000B307F04093F5F70F91679387C766B3D555
:107CF000B702F1BF9306A00C631DD700B307F04095
:107D0000B7153D0093F7F70F93850590B3D5F502AE
:107D10007DBF9306B00CE315D7F4B307F04093F59D
:107D2000F70F9167938797D0D9B78946631BD70020
:107D3000B307F040B7750B0093F7F70F9385051B5A
:107D4000F1B78546631AD700B307F040DD6593F7B6
:107D5000F70F938565E35DBFD28535FBB305F04032
:107D600093F5F50FB3D5BA029DB783C72400C18B35
:107D700099C7854717E7FF1F2309F7D6A5BE97E7E1
:107D8000FF1F238407D6BDB6854717E7FF1FA3044F
:107D9000F7D68DB63C0017E7FF1F2325F7E6094706
:107DA000930700032314F10097E6FF1F238CE6D20C
:107DB0002DBD63940756A94763E5B74217970100A5
:107DC0001307C76B8A05BA959C41BA97828717E457
:107DD000FF1F034494AC894C6306940D63E68C0644
:107DE00085476303F4089307F00F17E7FF1F034766
:107DF00067CF63F6E70017E7FF1F2305F7CE97EC81
:107E0000FF1F83CC2CCE9307000413F4FC0F63F404
:107E100097011304000497E7FF1F9387A7DE03ADC4
:107E2000070022862685EA85B38C8C40229D9770B8
:107E30000100E780C0F497E7FF1F238597CB97E702
:107E4000FF1F23A1A7DD45BC8D47630CF40A9947AA
:107E5000E31BF4F8979701009387C76817E7FF1FA4
:107E60002322F7DAA94751B717E7FF1F0347E7DCDB
:107E700097E7FF1F938707C94946979501009385A8
:107E8000656F63068700979501009385A56A3E8517
:107E900097700100E780A0EE17E7FF1F2324A7D605
:107EA000C947A1B797E6FF1F83C626D9054797E7BD
:107EB000FF1F938727C56394E6023E851306700271
:107EC000979501009385856897700100E78020EB06
:107ED00017E7FF1F2328A7D29307700239B73E8503
:107EE0001306300497950100938585609770010013
:107EF000E780E0E817E7FF1F2326A7D093073004A9
:107F0000EDB597E5FF1F83C545991795010013054A
:107F1000E56F97700100E780E0F1054D97EDFF1FD9
:107F200083CDADD197E5FF1F83C525971795010038
:107F30001305C56D6398AD0B97700100E78080EF66
:107F400097E7FF1F83C76795B5CBE36EF4E81794F7
:107F5000010013046466638CB701179401001304D5
:107F6000246663869701179401001304E466228552
:107F700097700100E78020051375F50F9307150032
:107F8000860717E7FF1F230FF7B68D4717E7FF1F79
:107F9000A30AF7B697E7FF1F9387C7B60147BE86C8
:107FA0001376F70F89076365A60297E7FF1F23ABD8
:107FB000D7C497E7FF1F83C7E7B405BD97970100B4
:107FC0009387875817E7FF1F232EF7C2914731BDCC
:107FD0003306E40003460600A3800700050723805C
:107FE000C7007DBF97700100E780C0E497E7FF1FDF
:107FF00083C7A78AE1D7E368F4DE1794010013046E
:10800000A458638CA7011794010013046458638675
:1080100097011794010013042459228597700100D9
:10802000E78060FA1375F50F93071500860717E7C9
:10803000FF1F2309F7AC8D4717E7FF1FA304F7AC19
:1080400097E7FF1F938707AC0147BE861376F70FAC
:108050008907E37CA6F43306E40003460600A38008
:10806000070005072380C700D5B797E5FF1F83C525
:10807000C582179501001305255A97700100E78006
:1080800060DB97E7FF1F83C7B7A793E7470017E7B2
:10809000FF1FA307F7A683C7240017E7FF1FA30F3F
:1080A000F7A489B81795010013054558977001008A
:1080B000E78020F097E7FF1F938747A483C7070057
:1080C00017D7FF1F230AF77C17E4FF1F034484A17F
:1080D000333480000DB01795010013056556977075
:1080E0000100E78000ED97E7FF1F83C777A193E7C3
:1080F000070117E7FF1FA305F7A083C7240017E7B1
:10810000FF1F230DF79E6FF0EFFE1795010013057B
:10811000655497700100E780C0E903C704007D8BB8
:1081200051EFB787004003C767021377C70B136788
:1081300027002383E70203C7A7021377C70B136740
:1081400027002385E70203C7E7021377C70B1367EE
:1081500027002387E70203C727031377C70B13679B
:1081600027002389E702854717D7FF1F2306F77EDD
:1081700017E7FF1F2304F78A17E7FF1F2302F7966D
:1081800017E7FF1F230FF79497D7FF1FA386077CDE
:1081900097E7FF1FA384078897E7FF1FA382079431
:1081A00097E7FF1FA38F079297E7FF1FA386079408
:1081B00097E7FF1FA38307A86FF0CFF389476312E8
:1081C000F70297D7FF1F83C7676D9146638CD70867
:1081D00063E0F604638EE70C6369F70A0547638082
:1081E000E70EFD5717E7FF1FA30EF78E3707400076
:1081F000B7E700E023A0E71801000100B7860040C0
:108200001306F0FC2381C60223A0E7106FF00FE2F3
:10821000130720086382E7086362F7021307100858
:10822000E391E7FC378700408347670293F7C70B6A
:1082300093E727002303F7026FF0CFEB1307300813
:108240006389E70213074008E39DE7F8378700409A
:108250008347270393F7C70B93E727002309F70208
:108260006FF04FE9378700408347270393F73707BD
:10827000F5B7378700408347E70293F7C70B93E7CB
:1082800027002307F7026FF0EFE6378700408347A8
:10829000E70293F73707F5B7378700408347A70210
:1082A00093F7C70B93E727002305F7026FF08FE4DE
:1082B000378700408347A70293F73707F5B737871B
:1082C00000408347670293F73707ADB71795010062
:1082D0001305453997700100E780A0CD97D7FF1FA0
:1082E000238C075AD5B3179501001305A53897704D
:1082F0000100E78000CC97D7FF1F239F075897D72F
:10830000FF1F9387277E03C40700894763F3870015
:1083100009441374F40F6FF00FDE13070002E392A9
:10832000E7EC631B0B0A638FF5009307200263835E
:10833000F508179501001305653797700100E78070
:1083400060AF45B51795010013058533977001009F
:10835000E78020C60144179D0100130DAD33A14CE9
:10836000B387840083C507006A8505049770010000
:10837000E78040ACE31694FF178501001305C56B39
:1083800097700100E780E0C217D4FF1F0344045137
:1083900001E897D7FF1F2383074E014B6FF0AFD53E
:1083A0008947E310F4E4854717D7FF1F2308F74CEC
:1083B0006FF04FD417D6FF1F0346364E97D5FF1FD9
:1083C00083C5A54D179501001305452D9770010034
:1083D000E78040A66FF00FD26380F5069307100286
:1083E000E399F5F497D5FF1F83C5454B1795010019
:1083F0001305C52C97700100E780C0A397E7FF1F06
:1084000023A2978097D7FF1F9387876E944383D7C4
:10841000470017D7FF1F0347076E17D6FF1F232DEF
:10842000D6461D4497D6FF1F239AF64697D7FF1FBF
:108430002387E7466FF02FCC97D5FF1F83C50546EE
:10844000179501001305052997700100E780809EAC
:1084500097D7FF1F2384074297D7FF1F239E07420A
:108460006FF02FF92547638FE7C89946378700409B
:108470006394D70223008702B7E700E0B706400005
:1084800023A0D71801000100130600FC2301C70236
:1084900023A0D7106FF08FB99306100A639FD700FF
:1084A00023008702B7E700E0B706400023A0D718F3
:1084B00001000100130680FCD1BF9306A009E381EF
:1084C000D7FE9306400AE38DD7FC93062002639DF6
:1084D000D700B7E700E0B706400023A0D718010097
:1084E000010023008702F9B78546E384D7FE93078E
:1084F0000008E300FBFEB7E700E0B706400023A05A
:10850000D71801000100130620FC23008702BDBF1D
:1085100017D7FF1F0347175D6302F71E63E7E702E4
:1085200095476300F7109947630AF704B786004040
:1085300023800602B7E700E03707400023A0E718D2
:10854000010001001306A0FC75B99307F005630A4A
:10855000F700930750096306F70093071002E3172B
:10856000F7FCB7E700E03707400023A0E718010059
:108570000100B7860040130620FC69B117DBFF1F1E
:10858000034B4B56930700045A8D63F46701130D98
:10859000000497D7FF1F9387E76683AC0700137427
:1085A000FD0F2286E685268597600100E780207D05
:1085B000B3078B40669417D7FF1F2305F75297D751
:1085C000FF1F23A18764B7870040630C0B02238041
:1085D000A703B7E600E03706400023A0C618010055
:1085E000010003C72702134707042381E70203C7DB
:1085F00027021377C70F2381E70223A0C6106FF06D
:10860000EFA22380070237E700E0B70640002320EF
:10861000D71801000100130620FC2381C7026FF068
:10862000AFB9378700408347370097D6FF1F83C60F
:10863000F64C93F70708D58FA301F700B706400063
:10864000B7E700E023A0D718010001001306A0FC43
:1086500035BD97D7FF1F9387275CCA9783C707004D
:1086600093F7F70FC1CF97D7FF1F83C7075DD9E7F0
:1086700017D7FF1F03471747930700026310F70838
:1086800083AD040017DDFF1F034D4D2197DCFF1F55
:1086900083CCDC2017DBFF1F034B6B20E6876A8748
:1086A000DA866E8697D5FF1F83C5451D1795010095
:1086B0001305C50397600100E780C07797D7FF1FB8
:1086C00023A8B74397D7FF1F2386A74397D7FF1F3A
:1086D000A382974397D7FF1F238F674197D7FF1F29
:1086E000A38D8718B7E700E03707400023A0E718FD
:1086F00001000100B78600406FF04FA2B7E700E02D
:108700003707400023A0E71801000100B7860040AA
:1087100015BD97D6FF1F83C646520547639CE604E6
:1087200029472381E70209472383E7022385E702DC
:1087300097D7FF1FA382073C97D7FF1FA38F074E32
:10874000B7870040A381070017D7FF1FA308073A88
:1087500005472383E700B640264496440649F2596C
:10876000625AD25A425BB25B225C925C025DF24D6D
:108770006161828029472381E70209472383E70259
:108780002385E7022387E7022389E70255B717D736
:10879000FF1FA304F70E6FE01FFF854717D7FF1FCA
:1087A000230CF71A17D7FF1F230AF72617D7FF1F27
:1087B0002308F73217D7FF1F2305F7326FE0BFFEFC
:1087C000854717D7FF1F2309F71817D7FF1F230760
:1087D000F72417D7FF1F2305F73017D7FF1F2302F2
:1087E000F73017D7FF1FA309071617D7FF1FA307D7
:1087F000072217D7FF1FA305072E97D7FF1FA382B6
:10880000072E8280411106C697000000E78080FB9A
:10881000B787004023800700130740FC2386E7004A
:108820001307C004A386E70017D7FF1F1307C70667
:108830002398E70017D7FF1F1307070A239AE700BB
:1088400017D7FF1F13078715239CE70017D7FF1FB4
:1088500013070721239EE70029472381E7020947E1
:108860002383E7022385E7022387E7022389E702C0
:10887000A3810700930600F8A380D7009306900217
:108880002380D700FD562383D7002381E70093067A
:10889000000537E700E0230BD740B7064000232050
:1088A000D71003C7170013671700A380E700B24073
:1088B00097D7FF1F2394072441018280411106C6E8
:1088C00097000000E78000F0B78700402380070092
:1088D000130700FC2386E7003147A386E70017D77C
:1088E000FF1F130767FB2398E70017D7FF1F130726
:1088F000A7FE239AE70017D7FF1F1307270A239C19
:10890000E70029472381E70209472383E7022385FC
:10891000E702A3810700930600F8A380D70093061F
:1089200090022380D700FD562383D7002381E700E0
:108930009306000537E700E0230BD740B706400059
:108940002320D71003C7170013671700A380E70081
:10895000B24097D7FF1F2393071A41018280F16726
:108960009387072017D7FF1F2324F718854717D7AA
:10897000FF1F2311F718A14717D7FF1F230DF71665
:1089800097D7FF1FA389071697D7FF1F23860716C0
:1089900097D7FF1F238407EE97D7FF1FA38F07ECFE
:1089A000814717D5FF1F1305A5EDFD5517D6FF1FEE
:1089B0001306C6ED2947B306F5002380B600B306BB
:1089C000F600238006008507E397E7FE97D7FF1F91
:1089D000A38B071097D7FF1FA389071097D7FF1FF7
:1089E0002384071097D7FF1F238F070E97D7FF1FEA
:1089F000238E070E97D7FF1FA388070E97D7FF1F59
:108A00002385070E814717D6FF1F1306E61F414730
:108A1000B306F600238006008507E39BE7FE82800D
:108A200017D7FF1F0347672185476316F700170312
:108A300000006700E3E8170300006700E3DC411172
:108A400022C406C617D7FF1F0347271F85472E8658
:108A500013F4F50FAA856317F70417D5FF1F130545
:108A6000E5F797600100E780803197D7FF1F2387E4
:108A700007FAB787004023848702B7E600E037068D
:108A8000400023A0C6180100010003C7A702137706
:108A9000C70F2385E702B240224423A0C610014538
:108AA0004101828017D5FF1F130505E7976001007C
:108AB000E780E02C97D7FF1F238007EAB7870040A5
:108AC00023828702B7E600E03706400023A0C618DD
:108AD0000100010003C767021377C70F2383E70272
:108AE0005DBF411106C697000000E78080E7B240F5
:108AF0004101170300006700E3F2411106C697F039
:108B0000FFFFE78080BF97D7FF1F83C7F7E4A1CBA4
:108B100097D5FF1F83C565E489C917D5FF1F1305C6
:108B2000E5E397E0FFFFE780603A97D7FF1FA38553
:108B300007E297D7FF1F238107FC37E700E0B7065E
:108B400040002320D71801000100378600408347EA
:108B5000660293F7370F2303F6022320D710B240A3
:108B60004101828041C9D9C597D7FF1F83C707F943
:108B7000D1C3011122CC4AC84EC656C25AC006CE35
:108B800026CA52C42E89AA890144930A0004371BBD
:108B9000030063772403B3078940C207C183BE84FF
:108BA00063F4FA0093040004C204C180130A1BD4C6
:108BB00097D7FF1F83C747DA9DE37D1A631C0A001E
:108BC000F2406244D2444249B249224A924A024B9C
:108BD0000561828097F0FFFFE78020B2D1BF338527
:108BE00089002694A685420497000000E78060E58E
:108BF000418045B7828097D7FF1F9387A707184208
:108C00009C4383D645000345070083C5C700035630
:108C100046006396A50083D5E700638DD502011158
:108C200006CE2386A7002397D700B705CF00DC4BDD
:108C30009385757D05077D162EC2230001003AC479
:108C40002316C1002317D10099C30A858297F240E9
:108C5000056182808280DC4DDC4B81CFB7E7040068
:108C6000904503A38705914517D5FF1F0345C50010
:108C7000028382806D713C083EC6B707E50023225F
:108C800091103EC8AA843C083285232611103ECAA2
:108C900023248110232021112E8997300000E780A2
:108CA000C0632A84979501009385C5A717750100B5
:108CB0001305857797600100E780C017A285179597
:108CC00001001305A5B697600100E780A0162945AD
:108CD00097600100E780E01AB705CB009385757DAA
:108CE000680097100000E780206CA285680097302C
:108CF0000000E780E050014781467000CA85268564
:108D000097200000E780A08F05CD2A849795010069
:108D1000938545A117750100130505719760010042
:108D2000E7804011A285179501001305E5B0976013
:108D30000100E7802010294597600100E78060145A
:108D40008320C110032481108324411003290110C2
:108D50005161828097D7FF1F9387C7F118429C43C8
:108D6000797122D406D60348070083C807012A84F4
:108D700083D64500035546006396080183D8270132
:108D8000638DD8022388070105072399D700370888
:108D9000CC00DC4B1308787D3ACC1307F5FF42CAB0
:108DA00023080100231EE100231FD10099C70808F2
:108DB00032C62EC482973246A24522859700000013
:108DC000E78080EBB2502254456182806D713C088F
:108DD0003EC0B707E5003EC23C083EC42326111042
:108DE000232481102322911023170100231801004E
:108DF00023190100231A0100231B010097A7FF1F5D
:108E000083D7076199E3C167FD172316F10097A780
:108E1000FF1F83D7076091EB97D7FF1F938787E5E5
:108E20009C439C43DC4783D7070017A4FF1F130410
:108E3000245E584C2317F10083574400484B2318F5
:108E4000F10031E1979501009385C59417750100F4
:108E50001305855D97600100E780C0FD179501004F
:108E60001305859497600100E780C0FC2945976051
:108E70000100E78000018320C110032481108324B6
:108E800041105161828097A7FF1F83C7D75889EB94
:108E9000B7E70400BC5782975C4C23AA0700E1BFE8
:108EA000FD1797A6FF1FA388F656035607018347B1
:108EB00004014C470A85230BF10097300000E7803E
:108EC000403197D7FF1F9387E7DA9C4301478146DC
:108ED00088430A866C0097100000E7804072AA84DD
:108EE00029C1979501009385E58A1775010013053F
:108EF000A55397600100E780E0F3A6851795010070
:108F00001305458B97600100E780C0F22945976003
:108F10000100E78000F7584CB7E70400BC57484B06
:108F20009DBF97A7FF1F83C7174FF5D7B7E704006B
:108F3000BC4F1044854517D5FF1F0345E5D38297E5
:108F40001DBF5C4EDC4BB9CFB1CD411122C41775AA
:108F500001001305654D2E84979501009385C58109
:108F600006C697600100E780E0ECA2851795010036
:108F70001305058797600100E780C0EB29459760DE
:108F80000100E78000F0B7E704002244B24003A3E9
:108F9000870517D5FF1F034525CE130640069145CB
:108FA000410102838280411122C417A4FF1F1304D0
:108FB000E4431C4C06C689C7DC4399C34C488297DE
:108FC000584CB7E70400BC57484B82975C4CB24002
:108FD000224423AA07004101828017A7FF1F13071D
:108FE000E742834707009306F00B850793F7F70FD7
:108FF00063E9F60097A6FF1F238AF64003450700A2
:109000008280930700F8FDB78357450063860710F9
:1090100001114AC817A9FF1F1309893F52C4032A27
:10902000C90106CE22CC03274A0126CA4EC656C223
:10903000F15735E31307D00DFD57636EC704B7E949
:10904000040083A709072A8413058600420541818D
:10905000B284AE8A8297232AAA000325C9015C49FB
:10906000A9E7978501009385256F17750100130502
:10907000A53B97600100E780E0DB17850100130541
:10908000657E97600100E780E0DA2945976001007E
:10909000E78020DFDD57F2406244D2444249B249C2
:1090A000224A924A3E850561828093874400B70533
:1090B000CF002319F5009385757D310597100000C9
:1090C000E780802E0325C901834564003105973070
:1090D0000000E780E0120325C9012686D685310508
:1090E00097300000E780E00E7146A2854A859760C0
:1090F0000100E780C0C8504419CA83A78905854587
:1091000017D5FF1F034545B78297814769B7970079
:109110000000E780E0CBD5BFFD573E85828041113E
:1091200026C297A4FF1F9384A42ED84C22C437E4F0
:1091300004003C54484B06C68297DC4C0323C4050C
:109140002244B240924423AA070017D5FF1F0345CB
:10915000A5B2854541010283411126C297D4FF1F64
:10916000938444B19C4006C622C44AC0D5C3DC43A4
:10917000C5C35CC12300B5002A849785010093858F
:10918000E558177501001305252A97600100E7804F
:1091900060CA294597600100E780A0CE9C4023A4C7
:1091A000070023A2070097A7FF1F93872724DC4F00
:1091B000DC4B91C7295597000000E78000DF97A797
:1091C000FF1F9387E724DC4FDC4B89C79700000023
:1091D000E78020F537E904008327C905894517D5BD
:1091E000FF1F034565A982978327C905914517D5B8
:1091F000FF1F034565A882979C4003A347016309AD
:10920000030022852244B240924402494101028374
:10921000B2402244924402494101828001113285C8
:1092200006CE22CC26CA2E8497300000E780E00AC2
:10923000AA84978501009385A55017750100130531
:10924000A51E97600100E780E0BE03078400035677
:10925000640083554400A686178501001305455A0E
:1092600097600100E78000BD294597600100E78015
:1092700040C197A7FF1F83C7C717639D970001458C
:1092800097000000E78060D281450A8597000000C2
:10929000E780C0ECF2406244D244056182806D7187
:1092A00023248110232611102322911093F74500C7
:1092B0002E84638707143C083EC0B707E5003EC212
:1092C0003C083EC4231701002318010023190100A4
:1092D000231A0100231B010097A7FF1F83D7071143
:1092E00099E3C167FD172316F10097A7FF1F83D7E6
:1092F000071091EB97D7FF1F9387C7979C439C4319
:10930000DC4783D7070017A7FF1F1307270E231774
:10931000F100544F835747002318F100DC4AA1E7BE
:109320009785010093850546177501001305C50F44
:1093300097600100E78000B0178501001305C5465E
:1093400097600100E78000AF294597600100E78042
:1093500040B3134544008320C110032481108324AB
:1093600041105161828097A7FF1F83C79708255539
:10937000D9C3FD1717A6FF1FA30DF60603D60601D6
:1093800083470701CC460A85230BF1009730000084
:10939000E78020E497D7FF1F9387C78D9C4317A7CB
:1093A000FF1F1307A704978601009386E6428843B0
:1093B0000A866C0097100000E7806024AA8451D9C7
:1093C000978501009385053C177501001305C505B8
:1093D00097600100E78000A6A685178501001305A8
:1093E000653D97600100E780E0A429459760010092
:1093F000E78020A9268597000000E78000BB91BF89
:1094000093F725009DC7B7E70400BC474146814557
:1094100028088297255597000000E78000B92808A2
:109420009305F00F97000000E78040D31345240018
:109430001DB793F71500014599DF97000000E780FD
:1094400020991345140001BF5C4D411106C688C325
:1094500017D7FF1F2320F782B7E7040083A7070869
:10946000170500001305E5E38297B24097D7FF1F69
:109470002384A78001454101828001113335A0007A
:10948000A307A100B7E7040083A7471706CE13067A
:10949000F1008545130550308297F24005618280C6
:1094A0008280411122C406C697C7FF1F83C7477E2B
:1094B000014489EF97B7FF1F83C7D7D7054499E7C2
:1094C00017B4FF1F034404D71344140022859700E8
:1094D0000000E780C0FA178501001305A54309E4E1
:1094E00017850100130505442244B240410117636A
:1094F000010067002394797122D4A30F010037E49F
:1095000004008327841726D24AD006D6AA842E893F
:10951000130550309305F10132C6829732468347D6
:10952000F10193150601C18185CB01452EC6970037
:109530000000E780C0F483274417B2454A86268599
:109540008297054597000000E78060F3B2502254EF
:109550009254025945618280832744174A862685A2
:109560008297EDB741119397050122C406C626C222
:10957000C1872E8463D40702B7E40400FC5417A506
:10958000FF1F0345E5EB829719C1BC548297216503
:10959000218DB240224492444101828093F715000C
:1095A0008DC7B7E7040083A7471A17A6FF1F130646
:1095B00026E897C5FF1F9385E56C17A5FF1F034598
:1095C00025E8829713451400E9B793F7250099CF52
:1095D000B7E70400BC4F13060064894517A5FF1FB9
:1095E000034505E682971345240065B793F7850088
:1095F00085CF97C7FF1F83C7676A85E7B7E7040072
:1096000003A8871A1307401F97A7FF1F83C747E3C5
:10961000814613064006994517C5FF1F0355856708
:10962000029813458400B5B793F745000145B5D3BB
:10963000B7E4040083A7041817C5FF1F0355856509
:109640008297BC4C13060064914517A5FF1F034584
:1096500025DF8297134544002DBF97C7FF1F83D78F
:1096600067636398A70217C7FF1F2316B76217C760
:10967000FF1F2313C76217C7FF1F2310D7622E8651
:109680001785010013058530BE851753010067005B
:10969000637A178501001305E53017630100670041
:1096A00043910357450097C7FF1F83D7A75E631EEB
:1096B000F704C1674111F91722C417C7FF1F232BF5
:1096C000F75C37E4040097C7FF1F23A7075C97C721
:1096D000FF1FA38F075A97C7FF1F2381075C7C4C8E
:1096E00006C6894517A5FF1F034585D582977C4C83
:1096F000914517A5FF1F0345A5D482972244B24088
:10970000410117030000670003DA17850100130504
:109710006529176301006700C3897D15954763E2DA
:10972000A71C178701001307671D0A053A951C41FE
:10973000011122CC06CEBA972E84828717850100AC
:109740001305C52697600100E780A086A1A203C784
:10975000250099476311F7022E8597000000E780E6
:1097600080F4834564001785010013052525975073
:109770000100E780206C97B7FF1F238D07AA17858C
:109780000100130565257DBF03C7250095476319B3
:10979000F702C16717C7FF1F0357C74FF91703D554
:1097A000A5006309F702B7E7040083A7C7178297EC
:1097B000178501001305452397500100E780607F5E
:1097C000854717B7FF1F2307F7A617850100130565
:1097D00025248DBF97C7FF1F239EA74A83D7E50087
:1097E00097C6FF1F2399F64A83D7050197C6FF1F27
:1097F0002394F64A83D7250197C6FF1F239FF64877
:1098000097C7FF1FA3860748631BE502B7E704005D
:10981000BC4F096613060690A14517A5FF1F034517
:1098200025C282970356E4008355A40017850100E2
:109830001305C51C97500100E780C05F51B793071F
:10984000700F2316F100B7E7040083A7870D17A652
:10985000FF1F0346E6BE6C0082974DF9854717C788
:10986000FF1FA307F7425DB7178501001305051B0E
:10987000D1BD83C5250091476392F502178501008C
:109880001305451B97500100E780A0729700000068
:10989000E78060C1F240624405618280994763922B
:1098A000F502228597000000E780E0DF8345640031
:1098B000178501001305851097500100E780805738
:1098C000D1BF9547639AF50083471400E1F31785EC
:1098D000010013056518BDB517850100130545186E
:1098E000E1BF82800111B7F5070030008146E10534
:1098F000194506CE9790FF1FE780A0EE8347C10071
:109900000347D100B7562D47A207D98F938676D546
:1099100017A7FF1F130707B414C3B736302D93865C
:10992000360354C313D6C700978601009386C60238
:1099300036960345060013D687003D8A3696834542
:10994000060013D647003D8ABD8B3696B69783C670
:1099500007000346060097A7FF1F938727B123043C
:10996000A700A304B7002305C700A305D70023065B
:1099700007002385A700A385B7002386C700A38619
:10998000D700F24005618280411106C697000000B1
:10999000E78080F5B7E7040083A7871417A6FF1FA9
:1099A000130646ABD54501458297B2405D4697A563
:1099B000FF1F9385A5AB130570304101170300000D
:1099C0006700A3B361712324811A37E4040083275D
:1099D00004082326111A2322911A2320211B232E47
:1099E000311917050000130525B8829717A9FF1F25
:1099F000130909A5994785442300A900231CF100F8
:109A000097850100938545F493074006177501007B
:109A1000130585A1231CF1082308910097C9FF1F96
:109A20009389E9D197500100E780C04083D50900B0
:109A300017850100130545F097500100E780803F2E
:109A4000294597500100E780C04303D50900896983
:109A500097000000E78040E98327441710088545F8
:109A60001305503082978327441717A6FF1F13064C
:109A7000E69FDD451305703082978327441717A6AC
:109A8000FF1F1306269CB545130560308297832778
:109A900044173008894513051031829783274417EE
:109AA0003009894513052031829783274415938512
:109AB00009900D4582978327441593850990114598
:109AC0008297A30591002306910002CD230801008F
:109AD000230C01008327841630099145130570403B
:109AE0008297832784161306B1008545130500402D
:109AF000829783278416700085451305104082974E
:109B000083278416300885451305204082978327D4
:109B10008416100885451305504082978327041545
:109B20007D558297832744137D5582977D5597A055
:109B3000FFFFE78080B58327440C829797A0FFFF43
:109B4000E780E0908327841417A6FF1F13068690F2
:109B5000D5450145829789471306700F814528092D
:109B60002306F1009780FFFFE780605A8D471306B8
:109B7000000881452808230CF1089780FFFFE78043
:109B800000599147230CF100976701009387477BA9
:109B9000984383C747003AC8230AF10097D0FFFFD4
:109BA000E780C08770008545054597A0FFFFE780E7
:109BB000E0B430099305700F094597A0FFFFE780D7
:109BC000E0B33008930500080D4597A0FFFFE7803C
:109BD000E0B210089545114597A0FFFFE78000B25D
:109BE000C16717C7FF1F1307E70AF9171CC3232212
:109BF000070017A5FF1F1305658497A0FFFFE780E7
:109C0000C0AE8327C41D17C5FF1F13052507829704
:109C10003C4803450900854582978320C11A0324E7
:109C2000811A8324411A0329011A8329C1195D610C
:109C30008280C16717C8FF1F0358C805F917630161
:109C4000F8083DCDB5CD011126CAB7E4040083A7BD
:109C5000841222CC2E862315B10006CE2A84014719
:109C60008146ED45428582972AC611ED1785010090
:109C70001305C5CF97500100E780A033F24062443E
:109C8000D24405618280FC440356A100A2858297DC
:109C90002C0017C5FF1F0355E5FF97A0FFFFE780C6
:109CA00080B169DD17850100130585CD975001004E
:109CB000E780203083A7C412ED45280082977DBF3E
:109CC00082800DC585471797FF1FA302F7789797E6
:109CD000FF1F238F077635469795FF1F938585765F
:109CE0001305603017030000670023819797FF1F5B
:109CF000A38F0774E9BF97C7FF1F83C727FAA9EF90
:109D0000C16717C7FF1F0357E7F8F9176306F70482
:109D10004111854722C417C7FF1F2301F7F837E415
:109D200004007C4C06C6A1451795FF1F03454571ED
:109D300082970323841A2244B2409797FF1F83C758
:109D4000277017C5FF1F0355E5F41307401F814611
:109D5000314699454101028382806D71232481102F
:109D60002326111023229110328401CD8947630AE2
:109D7000F5028320C1100324811083244110516116
:109D8000828017850100130565CEAE8497500100CF
:109D9000E7802022A285268597C0FFFFE780008705
:109DA000C9BFB7E70400FC47280082971785010068
:109DB000130585CC97500100E780A01F83478100E1
:109DC00039C41307000B6380E7021387A7051377D5
:109DD000F70F8D4663EDE602A285280097C0FFFFCE
:109DE000E780C0F679B78547E3F587F883459100AA
:109DF000177501001305C592B335B00097A7FF1F73
:109E00002380B72C97500100E780C0029DB703471D
:109E10009100A207D98F35671307D7556385E708E7
:109E20006368F7022D671307B7556387E706316745
:109E30001307C755638AE70429671307A755639477
:109E4000E702A285280097C0FFFFE780202F15B703
:109E500039679306E7656381D70863E9F60013075E
:109E6000E7556384E706A28528003DB73D67930662
:109E7000F755638AD7061307F766E396E7FE97C0A0
:109E8000FFFFE7804048F5B50146A285280097C04E
:109E9000FFFFE7804017F1BDA285280097C0FFFFB4
:109EA000E7800028F9B58947E3F587EC97000000C3
:109EB000E780A0E49305E4FFC205C1811305A1007A
:109EC0009790FFFFE780C0316DB5A285280097C04D
:109ED000FFFFE780A02771BDA285280097C0FFFF84
:109EE000E780603279B597C0FFFFE780803B51B5CE
:109EF000C16717C5FF1F0355E5D9F9176307F500BB
:109F0000B7E7040003A3C71702838280854717C7FA
:109F1000FF1F230FF7D6014517F3FFFF67002356F6
:109F20001783FFFFE702031A2A8408452E89B289A6
:109F300019C900C1971500009385A5866105973062
:109F40000100E780400281447D5A97100000E780BD
:109F5000E03963C7A404814497100000E780003A09
:109F600063C8A40497C7FF1F938787D39C43DC472C
:109F7000B307F94091872302F40063830904832720
:109F8000C900B307F4409587A302F4001C4C89C7AD
:109F90009C4799C3228582971783FFFF6700C315EB
:109FA0005C44139714008504BA972390470171BF4E
:109FB0001C48139714008504BA972390070069BFC3
:109FC000832789000547B307F4409587A302F4006F
:109FD00083570400638EE7028DC309476384E70457
:109FE0000D47E395E7FA978701009387A7FB1CCC01
:109FF00097870100938707FC11A897870100938733
:10A00000E7C11CCC97870100938747C25CC8BDBFDE
:10A0100097870100938787AD1CCC978701009387B2
:10A02000E7ADEDB797870100938787FC1CCC978736
:10A0300001009387E7FCD9BF95E51783FFFFE7028F
:10A04000030A004618448347940075839D8B631769
:10A05000F70097100000E78060B448C41783FFFF43
:10A060006700230A82801783FFFFE702A305138995
:10A070003500C16442094111AA890144F114135900
:10A080000901054A2EC697100000E7802026B24538
:10A090006348A400014541011783FFFF6700C30522
:10A0A00083A7090013171400BA9783D707006388A2
:10A0B000B7006394970063742A010504E1B705456E
:10A0C000D9BF1783FFFFE70203FFAA892E89328BCE
:10A0D000B6843A8ABE8A97A00000E780E0FB71C987
:10A0E000268597200000E780E0098D4763E7A700F9
:10A0F0007D551783FFFF670083FF83DB44009710C4
:10A100000000E780A0242A8497100000E780402503
:10A110009307740031443305850263CDA70297107D
:10A120000000E780A02297100000E78020222A8408
:10A1300097100000E780C022930774003144330574
:10A14000850263C3A70497100000E78020209307CF
:10A15000450029A897100000E7808020330585027C
:10A160001307F0179307C017E35FA7FA2D55E3C253
:10A1700077F963040B02D6865286A6854A85972016
:10A180000100E780E0BAB5B797100000E780401DF6
:10A19000330585029307C5FFD1BF83274900138587
:10A1A000C90083D5270097000000E78000EC61F527
:10A1B00081B769553DBF97C7FF1F2395A7AE97C7C6
:10A1C000FF1F9387E7AD904381470C463307F500A7
:10A1D000420741836393B700828054461398470037
:10A1E0008507C2962390E600D5B797C7FF1F9387D0
:10A1F00027AB9C4303C58700828017C5FF1F03550B
:10A2000065AA82801783FFFFE70263EDC1671387AA
:10A21000D7FF630BE502636AA700F1176300F5023D
:10A2200001451783FFFF6700C3ED1387E7FF630254
:10A23000E502FD171D8D13351500E5B79750000099
:10A24000E78080277D15C5BF97500000E78000FCA0
:10A25000D5BF97500000E78020FAEDB71783FFFFC6
:10A26000E702E3E74111AA8401442EC697100000DB
:10A27000E780C008B2456348A40001454101178347
:10A28000FFFF670003E89C48131514003E958357B1
:10A290000500E385B7FE0504C9BF034855008146A4
:10A2A00093F7F60F63E5070181473E8582805845A5
:10A2B00093975600BA9703D727006316B70003D7C2
:10A2C0000700E304C7FE8506E1BF8346450001475A
:10A2D0009377F70F63E4D700814711A81C45131645
:10A2E00057000507B29703D60700E313B6FE3E8575
:10A2F00082801783FFFFE702E3DC93170501C18724
:10A3000097CAFF1F938ACA99635BF00883A70A0064
:10A31000C0479C4703570400198D4205418163687B
:10A32000F500014422851783FFFF6700E3DC120577
:10A330002A94CDBFDC4713944900014A3E948347D9
:10A3400044006341FA02014A834754006349FA0218
:10A350008509C20993D9090183A70A009847E3EB4D
:10A36000E9FCC1B71C4413195A00A6853E994A85D9
:10A3700097000000E780C0EE05E1050AC9B75C441C
:10A3800013195A00A6853E994A8597000000E78078
:10A3900020ED19E1050A4DBFE30C09FA61B7AA8463
:10A3A00081495DBF1783FFFFE70263D31C452A8401
:10A3B00081E79307C5001CC51C44231204001CC080
:10A3C0009307F00F63EDB70093F5F50F2285972003
:10A3D0000000E780E0E21783FFFF670083D29394D9
:10A3E0000501C167C18063F9F500A6852285972024
:10A3F0000000E78000E6C5B7C18193F5F50F22851F
:10A4000097200000E780C0DFA68522859720000006
:10A41000E78000E1C9B797C7FF1F93876788884324
:10A4200082801C4599C797C7FF1F23ABA7860145AC
:10A4300082807D55828097C7FF1F938767869843E8
:10A4400083474500484792073E9582801783FFFF68
:10A45000E702E3C8617100451C183EC6B7078001DA
:10A460003EC81C183ECA8357440002CE02D002CC1C
:10A47000231EF100834784002A8902D22301F102BE
:10A480003C083ED402D697000000E78000FB8357CB
:10A4900005002316F10297500000E78020C523072E
:10A4A000A1025C4003556400F18313F71700834752
:10A4B000F10252055181F99BD98FA307F102971040
:10A4C0000100E780407639CDAA840355050097A0A6
:10A4D0000000E78040BD83D704002AD26800231C17
:10A4E000F10083D72400231DF1001C4803D6470048
:10A4F0008C4397200000E780C0CD8347B400CA8614
:10A5000017760100130606588117A305F4006C00A6
:10A51000481097200100E780A0815D611783FFFF4D
:10A52000670023BE2155D5BF1C45B1CF03C5A70089
:10A53000894613576500630BD7028D46630ED70219
:10A5400085466300D702130740063305E50203C7BB
:10A55000B700418B15CB83C7B700BD8B3355F54092
:10A5600082801375F5031307803EC5B7096713751D
:10A57000F50313070771D1BF372709001375F503DA
:10A580001307077CD9B7014582801783FFFFE702D5
:10A5900003B503A98500630C09048347B900AE84A1
:10A5A00093F7070E85C303459900930520030D819A
:10A5B0000505B305B5028844610597300100E780C1
:10A5C000A0AA35A02E8597000000E78020F62A84F7
:10A5D00019CD97000000E780605C8325C900B307B0
:10A5E000B54063FA87002E94B305A440E9F51783BC
:10A5F000FFFF670003B185457DBF1783FFFFE702BB
:10A6000003AE2A8403D50500011132C636C43AC20E
:10A610002EC002CA02CC02CE97A00000E780A0A8FC
:10A6200082452ACA22852ECC97000000E780E0E010
:10A6300003570500231EE10097500000E78000ABA0
:10A64000A24632469247230FA10036874C08B286B5
:10A650002285014697000000E780E0A60561178388
:10A66000FFFF670003AA1783FFFFE70243A761719B
:10A670001C183EC6B70780013EC81C183ECA3C08DD
:10A6800000453ED4AA8402CC02CE02D002D202D629
:10A6900097000000E78060DA8357050035592316DC
:10A6A000F10297500000E78060A42307A10209C4CB
:10A6B0008357440081EB21594A855D611783FFFF71
:10A6C000670023A4035564005205518197100100CF
:10A6D000E78060552A8965D18347B40093F7070E58
:10A6E00099C71305840197300100E780209A8357AA
:10A6F0004400231EF100834784002301F1025C40E3
:10A7000003550900D98313F7070883471102231C57
:10A71000A10093F7F707D98FA300F102835729000F
:10A72000231DF1005C40F18313F717008347F1020A
:10A73000F99BD98FA307F10297A00000E780A096AC
:10A740002AD235D98347940068001397570083476E
:10A75000B400FD8BD98FA305F4001C4803D6470035
:10A760008C4397200000E780C0A6A68717770100DA
:10A7700013074731740005464C10268597000000EA
:10A78000E78060942A890DD98347B400A685FD8BA4
:10A79000A305F40097000000E78060DF31BF178356
:10A7A000FFFFE702C393832485FE2A844111268597
:10A7B00097000000E78080D7834734FF93F7070EA8
:10A7C0008DCB2AC6268597000000E78060C809CD9A
:10A7D000834734FFB245FD8BA309F4FE91C5228562
:10A7E00097300100E780408841011783FFFF670031
:10A7F00043917DD98327C4FF2685829775F58347CA
:10A8000034FF93F7070E91C7228597300100E78048
:10A81000E087032584FE97000000E78000E5E9B7A4
:10A820001783FFFFE702A3889C4141112A8903C7D0
:10A83000070089472E84935667006380F6040D460F
:10A840006388C6049307F0076304F7022E859720F8
:10A850000000E78080A8AA848149C16B130C4900DD
:10A8600097B7FF1F9387C7439C43984763E4E90466
:10A8700041011783FFFF6700438703D745008547E2
:10A88000E3F8E7FE2E8597200000E78060AAE1B795
:10A8900003D74500E3FEE7FC2E8597200000E78004
:10A8A000C0A3AA84228597200000E78020A5C204C7
:10A8B000C98C5DB7DC470355A900139A49003E9A3D
:10A8C00093170501C187635DF00083570A00639702
:10A8D000A70263E774038327CA00034D5A002DA023
:10A8E000A1672167A98F1307F7EFE374F7FE63975A
:10A8F000090097000000E780209161FD85098DB770
:10A9000083278A00034D4A00835DA900035769002D
:10A91000216A138BC7003AC6814A33CA4D01631EB0
:10A920005D0197B7FF1F938727389C43E1DBA28621
:10A930006286814526858297D1B7A1679387F7EF15
:10A94000930C4BFF63F24703B2455A8597F0FFFF24
:10A95000E780A0710DC103278B00104709CE10437B
:10A960006382C4023107D5BFEE856685970000007B
:10A97000E780008F71F993861A0093FAF60F130B94
:10A980000B0271BF835644005C43E3E9F6F622856F
:10A990003AC697100000E780407EA1679387D704EE
:10A9A0002A8A035D4400324763E897008347D90051
:10A9B00093E707F8A306F9001C4766852286E2851F
:10A9C0008297C1670844FD17337AFA00529508C090
:10A9D0002312A40125B797B7FF1F9387672C9843CD
:10A9E000814715C31447814763FFD50093974500FE
:10A9F0004C47BE9519C903C7550081476375E600EA
:10AA0000DC451606B2973E85828003C74500814724
:10AA1000E37BE6FE16069C45F5B71773FFFFE702DA
:10AA2000636AAA892E8A814497BAFF1F938A4A27AC
:10AA300083A70A00984763E6E4001773FFFF6700E7
:10AA4000A36BDC471394440001493E9413BB1400EC
:10AA500083474400634BF900014913BB140083474B
:10AA60005400634FF9008504E1B708449317590077
:10AA70005287DA860146A2853E9582990509C9BFAB
:10AA80004844931759005287DA860546A2853E95B9
:10AA900082990509E9B71773FFFFE702436481450F
:10AAA00017F5FFFF1305054897B7FF1F239C071EE7
:10AAB00097000000E780A0F61773FFFF670063644C
:10AAC00097B7FF1F9387C71D9C4395C31773FFFF5D
:10AAD000E702E360814517F5FFFF1305A5449700E2
:10AAE0000000E780C0F31773FFFF67008361828077
:10AAF0001773FFFFE702035D37E404008327841226
:10AB000041112315E100AE893289368A3A868146A1
:10AB10000147ED45AA8482972AC621C90356A100A0
:10AB2000D28597400100E78080258327C413CE8516
:10AB300026858297058905C98327440D23142101A1
:10AB400001462C00268582972A8401C9B7E70400B4
:10AB500083A7C712ED45280082972285410117730C
:10AB6000FFFF670063594944D5B76554FDB75C41A1
:10AB7000FD175CC182801773FFFFE7024356B7E7FA
:10AB80000400FC5F829795473305F50281450D81EE
:10AB90001773FFFF6700E3561773FFFFE7022354A5
:10ABA000B7E70400FC5F829795473305F5020D81F6
:10ABB0001773FFFF6700E3541773FFFFE702235289
:10ABC000B7E7040083A7870B035505008297177327
:10ABD000FFFF670003531773FFFFE702435003555E
:10ABE00005003287AE861796FF1F0356868E97B5EF
:10ABF000FF1F9385A50B97000000E780A0EF177358
:10AC0000FFFF670003501773FFFFE702434DB7E7ED
:10AC1000040083A7C71782971773FFFF6700634E6F
:10AC20001773FFFFE702A34BB7E7040083A787135F
:10AC300097B5FF1F93858507829701451773FFFF1F
:10AC40006700234C1773FFFFE7026349B7E704006F
:10AC500083A7C71F81451795FF1F035585838297DB
:10AC60001773FFFF6700E3491773FFFFE7022347EE
:10AC7000B7E7040083A7871397B5FF1F93850504E3
:10AC8000829701451773FFFF6700A3471773FFFF04
:10AC9000E702E344B7E7040083A7C71F8145179580
:10ACA000FF1F0355058582971773FFFF67006345F4
:10ACB0001773FFFFE702A3422E8597800000E7800D
:10ACC000A0B097800000E780A0ED1773FFFF67003A
:10ACD00043431773FFFFE702834097800000E7803C
:10ACE000A0F71773FFFF6700C3415C49E1175CC918
:10ACF0005CC583572501A1072319F500835705017A
:10AD0000A1072318F5008280F1473305F50297B7B4
:10AD1000FF1F9387A7FC9C433E9582808D47631558
:10AD2000F60803D74600854763F0E7081773FFFF6F
:10AD3000E702E33A368536842E8997100000E780D3
:10AD4000C05929C98357440093140501C18063E3A6
:10AD50009704228597100000E7802058FD142312E5
:10AD600094009307A0026300F5029307B002630703
:10AD7000F50293079002631FF500228597000100FA
:10AD8000E780808601A80146CA85228597A0000039
:10AD9000E78020B11773FFFF6700A3362285971065
:10ADA0000000E7808004FDB7828097B6FF1F93867E
:10ADB00026F39C42014599CF9843D44217B6FF1F12
:10ADC0002320E6F26396D70097B6FF1F23ACE6F088
:10ADD0001385C7FE82801773FFFFE7024330970099
:10ADE0000000E780A04B71443305850291459790A0
:10ADF0000000E780E0E911E565551773FFFF670084
:10AE0000433097B7FF1F23A9A7EC97000000E78006
:10AE1000E04833058502914597900000E78040E7C0
:10AE200061DD97B7FF1F23ABA7EA97000000E7801B
:10AE3000E04697B7FF1F239BA7E897000000E78035
:10AE4000E04597B7FF1F2394A7E897770100938702
:10AE5000A7C817B7FF1F232FF7E6970700009387B0
:10AE600007E917B7FF1F2325F7E6014579B71773E1
:10AE7000FFFFE702C326AA8517B5FF1F130505E5E7
:10AE800097100000E780805C1773FFFF670063275F
:10AE90001773FFFFE702A32497000000E78060FD1F
:10AEA00097100000E780005C97B7FF1F938747E388
:10AEB0009C4391CF1387C7FE19CB83D5C7FF17B526
:10AEC000FF1F130565E297200100E780E019177363
:10AED000FFFF670003231773FFFFE702432097007C
:10AEE0000000E780C0EC09CD834785002A8493F7F2
:10AEF000070499EB0355E50097000000E78080F90F
:10AF00001773FFFF6700E31F8347C50093044501E4
:10AF100017B9FF1F1309C9DC85E3832709005CC942
:10AF200097B7FF1F23AE97DA83274900F1FB97B746
:10AF3000FF1F23A997DAE9B7FD172306F50061057E
:10AF400097800000E78080D78307840063CB0704E5
:10AF50008347840093E707F82304F400B7E704006D
:10AF60009C5F82974205A94741813375F50283476B
:10AF7000840093F707FCC98F2304F4008347D400AF
:10AF80003E951C402318A40089CF984319CB8347D2
:10AF9000C4005040814585073305F50242054181D3
:10AFA0000297832709005CC897B7FF1F23AA97D28F
:10AFB0008327490089E797B7FF1F23A597D28347C7
:10AFC000C4009DDF8355040117B5FF1F1305C5D1CC
:10AFD00097200100E780400925B71773FFFFE702BC
:10AFE000031097B7FF1F938767F59C47014485833C
:10AFF000858B85E3AE84B2853A8697100000E780A2
:10B00000404C2A8419C597100000E7808042829442
:10B0100008CC22851773FFFF6700A30E1773FFFF8D
:10B02000E702430A41112E8932C6AA89970000001F
:10B03000E780C031324713060502CA869705000033
:10B040009385C5CC17B5FF1F130545C897000000B1
:10B05000E780E0F82A8425C99304C5009700000022
:10B06000E780E0411946AA85268597100000E78011
:10B0700040168545268597100000E7802012177539
:10B080000100130525A34E958345050026859710DD
:10B090000000E780E0165C4831468145A1075CC8A6
:10B0A0005CC483572401E1172319F400835704017A
:10B0B000E1172318F4001C4C3E859770FFFFE780D2
:10B0C0000005A3042501228541011773FFFF6700D6
:10B0D000A3021773FFFFE70283004111AA842EC663
:10B0E00032C497100000E7802037004DB245224659
:10B0F000834784000CC050C093F7F70393E707041D
:10B100002304F40023180400268597100000E7802C
:10B11000403283479400A9462317A40013D7370071
:10B1200005073307D7029D8B85072306F400A30686
:10B13000E40083C70401D8488507230FF7FE17B73B
:10B14000FF1F1307E7B95843232A0400930744015C
:10B1500029E317B7FF1F2327F7B817B7FF1F2321CE
:10B16000F7B817B4FF1F130424B8228597200100F5
:10B17000E780C0E11C44858B5D8D19E58145228502
:10B1800097200100E78040EE41011773FFFF670041
:10B1900043F71CC317B7FF1F2326F7B4D9B717739C
:10B1A000FFFFE702C3F397050000938565B70145EC
:10B1B00097000000E78000B001451773FFFF6700AC
:10B1C00043F41773FFFFE70283F197000000E78065
:10B1D00080B01773FFFF6700C3F28347C500A5E384
:10B1E0001773FFFFE702A3EF2A840355E5009700DA
:10B1F0000000E78000C821C18347840093F7F7FB74
:10B200002304F4001C4091C7DC4381C74C40014536
:10B21000829797000000E78080B917B5FF1F1305DC
:10B22000A5AC97200100E78060E60355E400970095
:10B230000000E78020C61773FFFF670083EC828061
:10B240001773FFFFE702A3E997B7FF1F938747A98B
:10B2500097050000938565C817B5FF1F1305C5A89E
:10B2600023A0070023A2070097200100E780A0CFBA
:10B270001773FFFF6700E3E81C4D91CFDC4381CFDC
:10B280001773FFFFE702A3E5834507008297177353
:10B29000FFFF670003E7828097B7FF1F938707A729
:10B2A0009C4303C50700828097B7FF1F938707A6BB
:10B2B0009C4303C51700828097B7FF1F938707A59C
:10B2C0009C4303C52700828097B7FF1F938707A47D
:10B2D0009C4303C54700828097B7FF1F938707A34E
:10B2E0009C4303C53700828097B7FF1F938707A24F
:10B2F0009C4303C55700828097B7FF1F938707A120
:10B300009C4303C56700828097B7FF1F938707A000
:10B310009C4303C57700828097B7FF1F9387079FE1
:10B320009C4303C58700828097B7FF1F9387079EC2
:10B330009C4303C59700828097B7FF1F9387079DA3
:10B340009C4303C5A700828097B7FF1F9387079C84
:10B350009C4303C5B70011E11D45828097B7FF1FCD
:10B360009387C79A9C4303C5C700828097B7FF1F86
:10B370009387C7999C4303C5D700828097B7FF1F67
:10B380009387C7989C4303C5E700828097B7FF1F48
:10B390009387C7979C4303D50701828097B7FF1F08
:10B3A0009387C7969C4303C52701828097B7FF1FE9
:10B3B0009387C7959C4303D54701828097B7FF1FAA
:10B3C0009387C7949C4303D56701828097B7FF1F7B
:10B3D0009387C7939C4303D58701828097B7FF1F4C
:10B3E0009387C7929C4303C5A701828097B7FF1F2D
:10B3F0009387C7919C4303C5B701828097B7FF1F0E
:10B400009387C7909C4303C5C701828097B7FF1FEE
:10B410009387C78F9C4303C5D701828097B7FF1FCF
:10B420009387C78E9C438857828097B7FF1F938767
:10B43000E78D9C4303D5C702828097B7FF1F938790
:10B44000E78C9C4303D5E70219E11305800C828049
:10B4500097B7FF1F9387878B9C4303C507038280A1
:10B4600097B7FF1F9387878A9C43C85B828097B7F3
:10B47000FF1F938727898843828097B7FF1F938791
:10B48000A7888843828019E17D558280F5DE984245
:10B4900065DFFDD917B7FF1F130747AA1847AA870B
:10B4A0007155058B631D072403C507001547E37D10
:10B4B000A7FC03C737001305F0057D171377F70FB7
:10B4C000E364E5FC03C35700E30003FC83C86700A3
:10B4D000E38C08FA03C77700494579171377F70F0C
:10B4E000E364E5FA03C7A70011481305F7FF1375D6
:10B4F000F50FE36BA8F803CE97000D481305FEFF88
:10B500001375F50FE362A8F803C8B70063090800D4
:10B5100065181378F80F1305600DE36705F703C589
:10B52000C700794879151375F50FE36FA8F403C8C0
:10B53000D7000D457D181378F80FE36705F503D89C
:10B540000701930E40175118420813580801E3ED04
:10B550000EF303C8E7007D181378F80FE36605F3D0
:10B5600003C827017D181378F80FE36F05F103C8AE
:10B570008700C54E75181378F80FE3E70EF103D86E
:10B580006701856E938EBEE06D184208135808015E
:10B59000E3EC0EEF03D847016D1842081358080179
:10B5A000E3E40EEF03D88701791842081358080125
:10B5B000E36C05ED03C8A7017D181378F80FE36568
:10B5C00005ED03C5B7011D487D151375F50FE36D36
:10B5D000A8EA03C5D701714879151375F50FE3651E
:10B5E000A8EA03D5E7011308E00F7D154205418164
:10B5F000E36CA8E803C50702494879151375F50FF0
:10B60000E364A8E8C85301C937C8340059151308C2
:10B6100058BFE36BA8E603A8870237C534001305BB
:10B6200055BF5918E36205E717A5FF1F232EC56C08
:10B6300003C6050117A5FF1F232AF56C0545E37511
:10B64000C5E403D82501D04933760603E31E06E29C
:10B6500003C61501E30A06E217A6FF1F2324B66AF4
:10B6600083C5270001466387A50003C61700F1457F
:10B670003306B60283C707039305C00272971A0701
:10B680001307C70516031A9796084697B387B7029C
:10B6900041553E973297420741836362E80617732C
:10B6A000FFFFE702C3A3368597800000E78060694B
:10B6B00097000100E780E0482A8497A00000E78017
:10B6C000405B2A9497F00000E78020272A94979007
:10B6D0000000E78060822A9497F0FFFFE780E06F28
:10B6E0002A9497400000E78020942A9497700000E5
:10B6F000E780609D22951773FFFF670083A082801B
:10B700001773FFFFE702A39D4111A307A10097A0B4
:10B710000000E78060C69305F100170500001305DF
:10B72000E5B597F0FFFFE780802F014541011773D2
:10B73000FFFF6700039D1773FFFFE702C39717A47E
:10B74000FF1F1304A47F032884007959936818000D
:10B7500097A4FF1F23A8147F137818006310080212
:10B76000BA84BE89368B328A2E89AA8A97F0FFFF67
:10B77000E780E0A77D15269519E531594A851773AD
:10B78000FFFF6700C39697F0FFFFE78040A67D1597
:10B790002695A167E353F5FE97B7FF1F938707B17F
:10B7A00098433E8C814B01CB014597F00000E78028
:10B7B000E044933B15004A85DA865686D2859790F9
:10B7C0000000E780804E2A8911CD1C44F99B17A701
:10B7D000FF1F2329F77683270C00CDD3E3800BFAD4
:10B7E000829769BF268597A7FF1F23AB077497F041
:10B7F000FFFFE780809C4146CE8517A5FF1F1305FC
:10B80000657D97300100E780805797D00000E78082
:10B81000009A0325040B97D00000E780C09D0545E2
:10B8200097D00000E780C0A4054597000000E7809E
:10B8300060EDA9B797A7FF1F938747709C47858B3B
:10B84000EDC71773FFFFE702838917A5FF1F1305D5
:10B85000A57697A7FF1F23A3076E97A7FF1F23A116
:10B86000076E97A7FF1F23AF076C97200100E780A3
:10B87000E08197500000E780A0F697100100E78074
:10B88000604D97100100E780605397A7FF1F9387D3
:10B8900067699C4391C7054597800000E7800021B8
:10B8A00097A7FF1F9387C7519C4399C741657D1593
:10B8B00097700000E78000A397F00000E780A03EAB
:10B8C00097D00000E780409097A7FF1F9387077CE1
:10B8D0009C43139717016356070097F00000E78019
:10B8E000C0AD97A7FF1F23A7076E97A7FF1F23A52C
:10B8F000076E97A7FF1F23A3076E97A7FF1F23A11C
:10B90000076E97000000E780008C97000000E7803A
:10B91000C07297F0FFFFE780401897F00000E780C3
:10B9200000D71763FFFF6700C37D828097A7FF1FC3
:10B930009387C7608843828097A7FF1F938707601C
:10B94000C84382801763FFFFE70263799780000096
:10B95000E780607597800000E780C0771763FFFF7E
:10B960006700237A1763FFFFE702C3752A849304F5
:10B97000140201112E85B289A685214636C63A8960
:10B9800097300100E780403D0DE9B2463808268631
:10B99000CE851305940497500000E780604121464E
:10B9A0002C084A8597300100E780003B13351500CD
:10B9B00005611763FFFF670023740145D5BF176357
:10B9C000FFFFE702C3719305450617A5FF1F130587
:10B9D000253497100100E78020691763FFFF670097
:10B9E00043721763FFFFE702836F41112EC697F082
:10B9F000FFFFE780A01AB24588C141011763FFFF2E
:10BA0000670023701763FFFFE702C36BAA842E84CD
:10BA100097800000E780006CAA8985452285970001
:10BA20000000E780E07D83C7E4011389940899E36F
:10BA300013890403CE85228597000000E780407CAF
:10BA4000214693051902228597000000E78060785F
:10BA500097A7FF1F9387874E8C432285971000007E
:10BA6000E780C082214693858402228597000000EA
:10BA7000E78020761763FFFF670003681763FFFF07
:10BA8000E7026363397197F00000E780E0B4930543
:10BA9000400661E997800000E780006063020514BA
:10BAA00097A7FF1F83C7872813B7170097A6FF1F05
:10BAB000238EE626014499CFC16417A9FF1F1309FD
:10BAC000E9479309400EFD1497000000E7800086C7
:10BAD0006342A40A97F0FFFFE780400C4169B72951
:10BAE0000900096AFD7A2A8B81447D199389F97BC3
:10BAF000130A0A71938A8AC797000000E7800083BF
:10BB000063D7A4041304400EB387840217A7FF1F52
:10BB10001307C7420324070B3E948357C401638273
:10BB2000270B18403307EB4063EAE90083474400E2
:10BB30008507B3874703D6976365F70801468145B4
:10BB4000094597F0FFFFE780A04DAA8B29E59740B4
:10BB50000000E780808385476317F5068965938534
:10BB6000057117A5FF1F1305A51A97100100E7809F
:10BB7000A04F95A0B30734030327090BBA9703D747
:10BB8000C7016308970003C75700A38207002382F9
:10BB9000E700050415BF9305C50022859700000046
:10BBA000E78080E65E852286976501009385C5F172
:10BBB00097F0FFFFE78020525E8597100000E78036
:10BBC000608A850415BF97A7FF1F938727379C4777
:10BBD0008D83858BC1F721611763FFFF67002351B8
:10BBE00001468545094502D002D202D402D697F01B
:10BBF000FFFFE780E042AA8479DD97F00000E7804C
:10BC0000E09C1389C4002A8481454A85970000007E
:10BC1000E780005F0C4041464A8597000000E780BE
:10BC2000405B832944006385090C4E8502D802DA03
:10BC300002DC02DE97300100E780E0382ACE1410E3
:10BC400005462C0808184ECC97500000E780E00A03
:10BC50001375F50F51ED8355840093E525004A8552
:10BC600097000000E780E05E11460C104A859700BF
:10BC70000000E7800056014697650100938545E581
:10BC8000268597F0FFFFE780004526859700000096
:10BC9000E780407D5C40A1D3014685450D4597F086
:10BCA000FFFFE780E037AA841DD548401389C40010
:10BCB00097300100E78020312AC64A8597000000AE
:10BCC000E780404C3246636FC5004C404A85970080
:10BCD0000000E780005001468145268597F0FFFF70
:10BCE000E780603F268597000000E780A077E5B5F4
:10BCF00083558400ADB71763FFFFE702433E97A764
:10BD0000FF1F9387A7239C471DC193E7870017A5B3
:10BD1000FF1F1305E5FF17A7FF1F2325F722971025
:10BD20000100E78040321763FFFF6700833DDD9B22
:10BD300017A7FF1F2328F72097300000E780E06453
:10BD40007DF117A5FF1F1305A5FC97100100E780E3
:10BD5000E033D1BF1763FFFFE702E3354169AA89EA
:10BD60002E8AB28A368BBA8B814417ACFF1F130C14
:10BD7000EC1C930C400E7D1997F0FFFFE780005BF1
:10BD800063C4A40001443DA03384940383270C0BB7
:10BD90003E948357C401638627055A87D686528608
:10BDA000CE851305040397000000E780E0BB01C9BE
:10BDB00023800B0022851763FFFF6700433383470F
:10BDC000F40185C35A87D6865286CE85130594081A
:10BDD00097000000E78040B909C585472380FB0034
:10BDE000D1BF850451BF835745006380071E176389
:10BDF000FFFFE702232D01112A8497000000E7804E
:10BE0000C04D09C985476309F50605611763FFFF42
:10BE10006700832E97E00000E780007C7DF5835764
:10BE200044004947ED9BE392E7FEC1452285970018
:10BE30000000E7804033AA84228597000000E78055
:10BE4000204F0357440002CE91472A89631AF70016
:10BE5000228597000000E780A0513C082ACC3ECE06
:10BE600097E00000E78080765C55C5D374084A8669
:10BE7000A6850545829751BF03574400D147E3F695
:10BE8000E7F8032A0400C169014997AAFF1F938AB2
:10BE9000EA0A130B400EFD1997F0FFFFE7800049F7
:10BEA000634FA90E2285032A040097000000E78053
:10BEB000C042A1452A89228597000000E780A02A78
:10BEC000AA84228597000000E780804A14402A86D1
:10BED000AA8978082685CA8597000000E780C0E710
:10BEE000AA8405D503C7F40189476315F700834782
:10BEF000C10181DF5546D28513856400973001006A
:10BF0000E780E0E7014597800000E780C01901C5A0
:10BF100083D7C401A5E797A7FF1F938727029C47F4
:10BF200093551900858913D73700058B01CF898375
:10BF3000858B6399B70001452EC697000000E78006
:10BF4000C0DBB2454E8597800000E780601F034646
:10BF5000C1012A8493751900268597900000E78017
:10BF6000E03935C1268597800000E780E0182685F6
:10BF700011C0014597800000E780004C9730000019
:10BF8000E780A0408547E312F5E883C75400130714
:10BF9000F00FE38CE7E68507A382F400BDB5B30498
:10BFA000690383A70A0BBE9483D7C401638B37014F
:10BFB0005546D2851385640097300100E780C0D9CB
:10BFC00055DD0509D1BD5DD86DB782801763FFFFD0
:10BFD000E702430F97800000E780000C05C1C164B1
:10BFE000014417A9FF1F130969F59309400EFD14B9
:10BFF00097F0FFFFE7808033634EA40017A5FF1F73
:10C00000130505D197100100E780E0031763FFFFD8
:10C010006700830E330534038327090B3E9583574E
:10C02000C501638897002312050097800000E78010
:10C03000A00C050475BF97A7FF1F938727F09C47A7
:10C040008D83858B8DE31763FFFFE702430917A5F7
:10C05000FF1F1305E5CB97100100E780200317634E
:10C06000FFFF6700030A82801763FFFFE7022307D1
:10C07000970500009385C5A017A5FF1F130545C9A7
:10C0800097100100E78020EE1763FFFF670063074A
:10C090001763FFFFE702A3048841B7E70400BC5B16
:10C0A000050542054181829709C585472300F500B2
:10C0B00005051763FFFF6700C30483C7F5FF2E85DF
:10C0C0008507A38FF5FE828083C7F5FFFD1793F7E1
:10C0D000F70FA38FF5FE99EF1763FFFFE702230029
:10C0E000B7E70400BC571385F5FF82971763FFFF7E
:10C0F0006700230182801C41035745008D8FBA954C
:10C100001CC12312B5003E85828093D78500A2050D
:10C110001441DD8D835745001387E6FF18C1890759
:10C120002312F50013D685004111238FB6FEA38F8D
:10C13000C6FE4101828018419307F7FF1CC1835757
:10C14000450085072312F500A30FB7FE82808357B1
:10C1500045008D8F2312F5001C41BE950CC12E8524
:10C160008280AA8703D7470008410D8FAA952392A2
:10C17000E7008CC38280184108453305A7408280C0
:10C1800083574500035765001D8F1C4108453385C3
:10C19000A7403305A74082801763FFFFE70223F41F
:10C1A00041112EC62A8497000000E780A0FDB24509
:10C1B0006373B50001A0835744000840BE95231265
:10C1C000B4003E9541011763FFFF670083F31763D7
:10C1D000FFFFE702C3F041112E84B28532C69700FB
:10C1E0000000E780A0FB3246A28597300100E7807F
:10C1F00000B941011763FFFF6700A3F01763FFFF5A
:10C20000E702E3ED2E84854597000000E78000F902
:10C21000230085001763FFFF6700A3EE1763FFFF8E
:10C22000E702E3EB41112317B100894597000000B5
:10C23000E780C0F68347E1002300F5008347F10063
:10C24000A300F50041011763FFFF670083EB17634D
:10C25000FFFFE702C3E893D78500A2054111DD8DFA
:10C260002317B100894597000000E78020F383473A
:10C27000E1002300F5008347F100A300F500410130
:10C280001763FFFF6700E3E71763FFFFE70223E59C
:10C290001397850193D78501C166938606F0D98FE0
:10C2A00013D78500758FD98FA2053707FF00F98D49
:10C2B0004111DD8D2EC6914597000000E78000EE0C
:10C2C0006C00114697300100E78060AB41011763B5
:10C2D000FFFF670003E31763FFFFE70243E01C4132
:10C2E000854503C4070097000000E78080E62285AB
:10C2F0001763FFFF6700E3E01763FFFFE70223DE3A
:10C300001C414111894503C7070083C71700230754
:10C31000E100A307F10097000000E78080E30355E8
:10C32000E10041011763FFFF6700A3DD1763FFFF13
:10C33000E702E3DA1C414111894503C7070083C7BF
:10C3400017002307E100A307F10097000000E78032
:10C3500040E08357E100410113D58700A2075D8DBE
:10C36000420541811763FFFF6700A3D91763FFFFF1
:10C37000E702E3D60C4141112A8411466800973048
:10C380000100E780C09F9145228597000000E7806B
:10C3900040DCB247C166938606F01397870113D538
:10C3A0008701598D13D78700758F598DA2073707DD
:10C3B000FF00F98F5D8D41011763FFFF670063D4B4
:10C3C0001C45BE950CC18280AE87944391E65841CE
:10C3D00001EF0CC15CC1828003C7570013671700CF
:10C3E000A382E700B687D5B70CC3EDB7AA8708418B
:10C3F00019CD1841D44398C36313D500D8C32A87F5
:10C40000034657009376160081E6232007008280BA
:10C41000944381CA8C4203A847008CC363930601EE
:10C42000CCC3799A14C3A302C7003687D1BF1C4579
:10C43000DC471D8DB777DBB6938777DB098533053E
:10C44000F502420541818280F147B385F5024845F6
:10C450002E9582808347450085072302F500828060
:10C460001763FFFFE702A3C72A8409E41763FFFFEE
:10C47000670023C983474400F5DBFD1793F7F70FE7
:10C480002302F400E5F71C4403D727000507239196
:10C49000E700DC4399C3228582974C4889CD8347C6
:10C4A0005400898B99E71C4422859C479C439C47F8
:10C4B0008297232A04000040232004007DB71763DD
:10C4C000FFFFE702C3C18357250041112EC681EB50
:10C4D0000144228541011763FFFF670083C20357B0
:10C4E00005008147F146E305F7FEB385D7024045D5
:10C4F00085072E948345440008C4F5F5B247AA8405
:10C5000081E7232A040009A81C456C0022859C436E
:10C510009C43829748C84DDD85472312F400B247FB
:10C5200023200400231804002319F4005C485CC491
:10C5300083D72400FD172391F40061BF1763FFFF29
:10C54000E702E3B99797FF1F9387877E88432326E7
:10C55000050023240500410597100100E78000B382
:10C560001763FFFF6700E3B91763FFFFE70223B715
:10C570001794FF1F1304C47B1C40411199CF9C47A3
:10C580002300B5002AC65CC197000000E78040FB8D
:10C590001C40DC4399C33245829741011763FFFF7A
:10C5A000670023B60347450029E3584DAA877D5508
:10C5B0001DCF1763FFFFE70283B21CC3DC479796CA
:10C5C000FF1F23A7E676F156130507012390D70036
:10C5D000970500009385050297100100E780A09859
:10C5E00001451763FFFF6700C3B17D5582808280DC
:10C5F0001763FFFFE702A3AE0111614681452800E2
:10C600009760FFFFE780A0B09797FF1F938747725F
:10C610009C4328009305F00FDC473EC697000000BE
:10C62000E780C0F405611763FFFF670083AD97974C
:10C63000FF1F9387E76F9C43D847A1679387C70283
:10C64000631EF70A397106DE22DC26DA80004AD83A
:10C650004ED652D456D23285B28497000000E7807D
:10C66000C0C7AA89268597000000E78020C9231843
:10C67000A4FC268597000000E78040C82319A4FC8D
:10C68000268597000000E78060C783D744000A8AA8
:10C69000231AA4FC858393F7F70F230EF4FC860777
:10C6A000BD0793F7073F3301F1408A8A0149834769
:10C6B000C4FD6367F902CE85130584FC232C54FD69
:10C6C00097000000E78080EA5281130104FCF250D9
:10C6D0006254D2544259B259225A925A21618280EC
:10C6E000268597000000E78060C193171900D69750
:10C6F00005092390A7001379F90F55BF82809797FA
:10C70000FF1F9387E7629C43D847A1679387A702DF
:10C71000631AF70A397106DE22DC26DA80004AD86D
:10C720004ED652D456D23285B28497000000E780AC
:10C73000C0BAAA89268597000000E78020BCFD5773
:10C740002318A4FC26852319F4FC97000000E78039
:10C75000E0BA83D744000A8A231AA4FC858393F79E
:10C76000F70F230EF4FC8607BD0793F7073F33014D
:10C77000F1408A8A01498347C4FD6367F902CE8587
:10C78000130584FC232C54FD97000000E78000DE95
:10C790005281130104FCF2506254D2544259B259EE
:10C7A000225A925A21618280268597000000E780F4
:10C7B000E0B493171900D69705092390A7001379C1
:10C7C000F90F55BF82809797FF1F938767569C4349
:10C7D000D847A16789076310F70A397106DE22DCA2
:10C7E00026DA80004AD84ED652D456D232853289C3
:10C7F00097000000E78060AEAA894A859700000094
:10C80000E780C0AF835749000A8A2318A4FC8583B8
:10C8100093F7F70F230CF4FC8607BD0793F7073F48
:10C820003301F1408A8A8144834784FD63E7F4023F
:10C83000CE85130584FC232A54FD97000000E78071
:10C84000E0D25281130104FCF2506254D254425996
:10C85000B259225A925A216182804A85970000007B
:10C86000E780C0A993971400D69785042390A7006A
:10C8700093F4F40F55BF82809797FF1F9387474B20
:10C880009C43D847A1679387E704631EF70A397171
:10C8900006DE22DC26DA80004AD84ED652D456D2A2
:10C8A0003285B28497000000E78020A3AA892685FC
:10C8B00097000000E78080A42318A4FC2685970039
:10C8C0000000E780A0A3231AA4FC2685970000009F
:10C8D000E780C0A283D744000A8A2319A4FC858379
:10C8E00093F7F70F230EF4FC8607BD0793F7073F76
:10C8F0003301F1408A8A01498347C4FD6367F90225
:10C90000CE85130584FC232C54FD97000000E7809E
:10C91000E0C55281130104FCF2506254D2544259D2
:10C92000B259225A925A21618280268597000000CE
:10C93000E780C09C93171900D69705092390A7009C
:10C940001379F90F55BF82809797FF1F9387473E52
:10C950009C43D847A1679387C704631AF70A3971C4
:10C9600006DE22DC26DA80004AD84ED652D456D2D1
:10C970003285B28497000000E7802096AA89268538
:10C9800097000000E7808097FD572318A4FC2685B8
:10C99000231AF4FC97000000E780409683D74400F8
:10C9A0000A8A2319A4FC858393F7F70F230EF4FC5E
:10C9B0008607BD0793F7073F3301F1408A8A014993
:10C9C0008347C4FD6367F902CE85130584FC232CDD
:10C9D00054FD97000000E78060B95281130104FC08
:10C9E000F2506254D2544259B259225A925A216199
:10C9F0008280268597000000E780409093171900F9
:10CA0000D69705092390A7001379F90F55BF8280A7
:10CA10009797FF1F9387C7319C43D847A167DD07CE
:10CA20006317F7041753FFFFE702636B79713285D1
:10CA3000328497000000E780408A2AC6228597004A
:10CA40000000E780A08B2311A1022285970000003F
:10CA5000E780A088B2452300A102280897000000C3
:10CA6000E780C0B045611753FFFF6700836982808C
:10CA70009797FF1F9387C72B9C43D847A16793873E
:10CA800087046317F7041753FFFFE70243657971C3
:10CA90003285328497000000E78020842AC62285F0
:10CAA00097000000E78080852311A102228597006E
:10CAB0000000E7808082B2452300A1022808970089
:10CAC0000000E780A0AA45611753FFFF670063637A
:10CAD00082809797FF1F9387A7259C43D847A1671C
:10CAE0009387A7046312F7021753FFFFE702235F40
:10CAF00001112800814597000000E78020A705610B
:10CB00001753FFFF6700E35F82809797FF1F9387AC
:10CB100027229C43D847A167938757026319F702DE
:10CB20001753FFFFE702A35B0111328597F0FFFF68
:10CB3000E780A07A2308A100814528009700000023
:10CB4000E780C0A205611753FFFF6700835B828007
:10CB50009797FF1F9387C71D9C43D847A16793876B
:10CB6000E702631BF7041753FFFFE7024357011166
:10CB70003285328497F0FFFFE7804078AA842285CF
:10CB800097F0FFFFE7808077854709E9228597F0D6
:10CB9000FFFFE78080744205B337A000280081457D
:10CBA000231891003ECA97000000E780209C056191
:10CBB0001753FFFF6700E35482809797FF1F938707
:10CBC00027179C43D84799476313F7081753FFFF6C
:10CBD000E702E35079713285328497F0FFFFE780F6
:10CBE000C06F2AC6228597F0FFFFE78020712310CF
:10CBF000A102228597F0FFFFE780206E2301A102AA
:10CC0000228597F0FFFFE780406DA301A1022285F6
:10CC100097F0FFFFE780606C2302A102228597F066
:10CC2000FFFFE780806B2313A102228597F0FFFFAF
:10CC3000E780A06AB2452314A102280897000000EB
:10CC4000E780C09245611753FFFF6700834B8280E6
:10CC50009797FF1F9387C70D9C43D847A16793877A
:10CC6000C7036313F7081753FFFFE70243477971C0
:10CC70003285328497F0FFFFE78020662AC622853E
:10CC800097F0FFFFE78080672310A102228597F0CD
:10CC9000FFFFE780A0662311A102228597F0FFFF26
:10CCA000E780A0632302A102228597F0FFFFE780BF
:10CCB000C062A302A102228597F0FFFFE780E06136
:10CCC0002303A102228597F0FFFFE7800061B245B0
:10CCD000A303A102280897000000E780208945618E
:10CCE0001753FFFF6700E34182801753FFFFE702FE
:10CCF000033F01112A8497F0FFFFE780005EAA84BA
:10CD0000228597F0FFFFE780605F228597F0FFFFA5
:10CD1000E780C05E035744008D4763F7E700228534
:10CD200097F0FFFFE780805D228597F0FFFFE780A7
:10CD3000E05C2800A68597000000E780208305615D
:10CD40001753FFFF6700E33B9797FF1F938747FE4B
:10CD50009C43D847A167FD07631FF7001753FFFFE8
:10CD6000E702E337328597000000E78040F8175369
:10CD7000FFFF6700033982809797FF1F938747FB68
:10CD80009C43D847A167E5076315F7081753FFFFD2
:10CD9000E702E33479713285328497F0FFFFE78050
:10CDA000C0532AC6228597F0FFFFE78020552285D1
:10CDB00097F0FFFFE78080542310A102228597F0AF
:10CDC000FFFFE780A053520551812311A102228564
:10CDD0002302010297F0FFFFE7802050A302A10287
:10CDE000228597F0FFFFE780404F2303A1022285B1
:10CDF00097F0FFFFE780604EB245A303A102280829
:10CE000097F0FFFFE780807645611753FFFF6700CB
:10CE1000432F82809797FF1F938787F19C43D847C2
:10CE2000A1679387E703631FF7001753FFFFE7022C
:10CE3000032B328597000000E78060EB1753FFFF5C
:10CE40006700232C82809797FF1F938767EE9C4390
:10CE5000D847A16793874704631EF7021753FFFF64
:10CE6000E702E32779713285328497F0FFFFE7808C
:10CE7000C0462AC6228597F0FFFFE7802048B245CA
:10CE8000280897F0FFFFE780606E45611753FFFFAA
:10CE90006700232782809797FF1F938767E99C434A
:10CEA000D847A167938787026310F7041753FFFFE2
:10CEB000E702E32279713285328497F0FFFFE78041
:10CEC000C0412AC6228597F0FFFFE7800041B245A6
:10CED0002300A102280897F0FFFFE7802069456141
:10CEE0001753FFFF6700E32182801753FFFFE7021C
:10CEF000031F011197F0FFFFE780203EAA8528005D
:10CF000097F0FFFFE780806605611753FFFF67001A
:10CF1000431F9797FF1F9387A7E19C43D847A167BB
:10CF2000D107631FF7001753FFFFE702431B32854A
:10CF300097000000E780A0FB1753FFFF6700631C0A
:10CF400082809797FF1F9387A7DE9C43D847A167EE
:10CF5000C507631FF7001753FFFFE7024318328529
:10CF600097000000E780A0F81753FFFF67006319E0
:10CF700082809797FF1F9387A7DB9C43D847A167C1
:10CF8000B907631FF7001753FFFFE7024315328508
:10CF900097000000E780A0F51753FFFF67006316B6
:10CFA00082809797FF1F9387A7D89C43D847A16794
:10CFB000AD07631FF7001753FFFFE70243123285E7
:10CFC00097000000E780A0F21753FFFF670063138C
:10CFD00082809797FF1F9387A7D59C43D84789479F
:10CFE0006318F7021753FFFFE702630F0111328541
:10CFF00032C897F0FFFFE780402EAA85280097F0FF
:10D00000FFFFE780A05605611753FFFF6700630F1E
:10D0100082809797FF1F9387A7D19C43D847A1672A
:10D020008D076311F7041753FFFFE702430B01114C
:10D030003285328497F0FFFFE780202A13066100D3
:10D04000AA844C00228597300000E780C023280086
:10D05000A68597F0FFFFE780605105611753FFFF3A
:10D060006700230A82809797FF1F9387A7CC9C4372
:10D0700081CFDC4391CB1753FFFFE7024306829732
:10D080001753FFFF6700E30782801753FFFFE70294
:10D09000030579713C08AE843ED2A165B7070A004A
:10D0A0002A843ED448103C08DD053ED636C432C63C
:10D0B0003AC297D0FFFFE780202F12474810BA8569
:10D0C00097F0FFFFE780C01332464810B28597F013
:10D0D000FFFFE780E014A2464810B68597F0FFFFF7
:10D0E000E7800012501001478146A685228597D01F
:10D0F000FFFFE780C05045611753FFFF67006300E3
:10D100001753FFFFE702A3FD01117C000329C501AE
:10D11000AE843ECAA165B70707002A843ECC480802
:10D120007C00C5053ECE97D0FFFFE780E027834512
:10D13000D900480897F0FFFFE780800C50080147AE
:10D140008146A685228597D0FFFFE780404B056189
:10D150001753FFFF6700E3FA1753FFFFE70223F8B7
:10D1600083C7950093F7F707A384F50097000000A5
:10D17000E78040F91753FFFF6700A3F81753FFFF3D
:10D18000E702E3F579713C08AE843ED2A165B707AA
:10D1900009002A843ED448103C08938545043ED6B5
:10D1A00032C636C497D0FFFFE7800020A246481061
:10D1B000B68597F0FFFFE780A00432464810B2859D
:10D1C00097F0FFFFE780C005501001478146A68514
:10D1D000228597D0FFFFE780804245611753FFFF0C
:10D1E000670023F21753FFFFE70263EF83C7950041
:10D1F00041112A8493F7F707A384F50032852EC6E0
:10D2000097F0FFFFE780800F85672AC46370F502FF
:10D2100097700000E78020E92246B24509ED1147EA
:10D220008146228597000000E78060E641011753A0
:10D23000FFFF670003ED01478346F501DDB7175394
:10D24000FFFFE70223E801113C003ECAB7070A00CE
:10D250003ECC3C003ECE83C79500AA89328593F729
:10D26000F707A384F5002E8497F0FFFFE7800009FD
:10D270008567637DF504A165AA84938585044808C4
:10D2800097D0FFFFE7804012268597700000E78067
:10D2900080E12A8929E19145480897F0FFFFE7805E
:10D2A00020F6A685480897F0FFFFE78060F7CA855B
:10D2B000480897F0FFFFE780A0F401478146500837
:10D2C000A2854E8597D0FFFFE78060330561175335
:10D2D000FFFF670063E28145480897F0FFFFE780A2
:10D2E00020F20349090275BF1753FFFFE70283DDF0
:10D2F00079711C103ECAB7070F003ECC404D1C1080
:10D30000AA84AE894808994532C636893ECE97D060
:10D31000FFFFE780600932464808B28597F0FFFFBB
:10D32000E78000EE630C0902A545480897F0FFFF6F
:10D33000E780C0E62546CA8597200100E78020A443
:10D34000500801478146CE85268597D0FFFFE780AC
:10D35000002B45611753FFFF670003DA8355C402B2
:10D36000480897F0FFFFE780A0EB0355E4028145F2
:10D3700005C5854785456301F502C167FD1793051E
:10D38000F00F630BF5007D1597700000E780208E8D
:10D390009305150093F5F50F480897F0FFFFE78018
:10D3A00020E683450403480897F0FFFFE78040E547
:10D3B00083451403480897F0FFFFE78060E4835536
:10D3C0002403480897F0FFFFE78080E58355440376
:10D3D000480897F0FFFFE780A0E49DB71753FFFFD1
:10D3E000E702E3CF83C795008146014693F7F7072D
:10D3F000A384F50097000000E78040EF1753FFFF7C
:10D40000670023D01753FFFFE70263CD79713E8495
:10D410001C103ECA2E89B7070F00A1653ECCFD0542
:10D420001C10AA84480842C03AC23ECE36C432C656
:10D4300097D0FFFFE78040F732464808B28597F063
:10D44000FFFFE780E0DBA2464808B68597F0FFFFC4
:10D45000E78000DD12474808BA8597F0FFFFE780B4
:10D4600020DC0248630C08029145480897F0FFFF52
:10D47000E780C0D21146A28597200100E780209066
:10D48000500801478146CA85268597D0FFFFE7806F
:10D49000001745611753FFFF6700A3C68945480879
:10D4A00097F0FFFFE78080CF834704002300F5005B
:10D4B00083471400A300F500E1B71753FFFFE7020D
:10D4C00063C083C7950001112A8A93F7F707A384E5
:10D4D000F5003285AE8432C697F0FFFFE78000E2A8
:10D4E00032462A89328597F0FFFFE78000DF8567A3
:10D4F0006373F902AA894A8597700000E780A0BA91
:10D500002A8419ED114781464A86A68552859700DF
:10D510000000E780C0B705611753FFFF6700C3BD78
:10D520009387E9FF93F7F70F0547E366F7FE834715
:10D53000F50195EB8947E380F9FE8346F4015285B6
:10D5400001474A86A68597000000E78040B4A1679E
:10D55000D90748083ECC230A010002CE97000000FC
:10D56000E780A0B04DBF639EE7008947639EF90046
:10D5700093071020231FF50097700000E780C0B7C5
:10D580006DBF0947E39BE7FA8D47E398F9FA2285D7
:10D5900097700000E78080DF9797FF1F9387879839
:10D5A0009C4399E79797FF1F938787819C4399C76F
:10D5B00003D5040097800000E780A0CE231F04005D
:10D5C00022855DBF1753FFFFE70263B101113C00E5
:10D5D0003ECAB7070B003ECC3C003ECE83C7950049
:10D5E0002A89328593F7F707A384F500AE8497F074
:10D5F000FFFFE780A0D093170501C187635AF006AB
:10D60000A1652A849385E502480897D0FFFFE7804B
:10D61000A0D9A285480897F0FFFFE78060C09787F0
:10D62000FF1F9387E7799C43A9EB01449375F40F9F
:10D63000480897F0FFFFE780A0BC9355844093F51E
:10D64000F50F480897F0FFFFE78080BB9355044132
:10D6500093F5F50F480897F0FFFFE78060BA0147A0
:10D6600081465008A6854A8597D0FFFFE78020F9BC
:10D6700005611753FFFF6700C3A84165854605464E
:10D68000A2857D1597500000E78060BD59DD5105EA
:10D6900097000100E780808F130440063344850221
:10D6A00071B71753FFFFE70283A30111B707060005
:10D6B0003EC683C7950021642A8993F7F707A384A0
:10D6C000F500AE8428009305A4040AC40AC897D0C4
:10D6D000FFFFE78060CD300001478146A6854A857F
:10D6E00097D0FFFFE780A0F197E0FFFFE780C0142D
:10D6F00013049404480822CC230A010002CE9700A8
:10D700000000E780809605611753FFFF6700639F65
:10D710001753FFFFE702039BC1642A8901449799CD
:10D72000FF1F9389A981130A8002FD1497E0FFFF70
:10D73000E780C0C06347A40001451753FFFF67009F
:10D74000A39BB307440303A7C90ABA9703D70700EB
:10D750006306970083D72700638427010504F9B780
:10D760000545E1BF1753FFFFE702C3952A8A2E89BB
:10D7700099C123A0050081498144978AFF1F938A9C
:10D78000AA5B614B97E0FFFFE78080C163C7A400FD
:10D790004E851753FFFF670023963384640383A7E6
:10D7A0000A003E948357040099E76304090023208C
:10D7B00089008504C1BF4146D285130544009710F6
:10D7C0000100E780605975F5A289E5B71753FFFF9F
:10D7D000E702438F39717C083ED4B7070A003ED672
:10D7E0007C083ED883C795002A8A328593F7F707CD
:10D7F000A384F5002E8932C697F0FFFFE78000B0C2
:10D8000085676373F5083246AA84328597F0FFFF77
:10D81000E780A0AC8547AA8963E8A706A165938540
:10D820008504281097D0FFFFE78000B82685977001
:10D830000000E78040872A8429ED9145281097F061
:10D84000FFFFE780E09BA685281097F0FFFFE780A9
:10D85000209DCE85281097F0FFFFE780609A014752
:10D8600081463010CA85528597D0FFFFE78020D9C6
:10D87000A1679387770448183EDC230A010202DE81
:10D8800097F0FFFFE780607E21611753FFFF67007D
:10D89000A3868145281097F0FFFFE7806096A68554
:10D8A000281097F0FFFFE780A0979797FF1F9387B7
:10D8B000A79F9C4381CB22856389090097D00000F4
:10D8C000E78040248345040271B797D00000E780C9
:10D8D000C022CDBF1743FFFFE702C37E83C7950079
:10D8E0004111AA8993F7F707A384F5003285AE8426
:10D8F000328A97F0FFFFE78060A08567637FF502BB
:10D900002A8997600000E780007A2A84914631C511
:10D910008347F50105476387E70291C70D476366B3
:10D92000F704AD461DA89305050303250A004146EB
:10D9300097100100E78040420DE941011743FFFFC6
:10D940006700837B9305950803250A0041469710DD
:10D950000100E7806040814669F54A86A6854E85CC
:10D9600097000000E780C081C9BF83250A00130526
:10D97000940897700000E780A02919C1C146F1BF43
:10D980009787FF1F9387075A9C4399E79787FF1F45
:10D99000938707439C4399C7228597800000E780BF
:10D9A000208A69FD8547A30FF400228597B0000007
:10D9B000E7806084228597600000E780E0734E85F1
:10D9C00081464A86A68597F0FFFFE780607BA167C6
:10D9D0009387570448003EC42302010002C697F013
:10D9E000FFFFE780806891BF1743FFFFE702A36C4A
:10D9F00083C795004111AA8993F7F707A384F5001F
:10DA000032852E89B28A97F0FFFFE780208F8567E5
:10DA10006374F50EAA8497600000E780C0682A84CA
:10DA20000DED416B014A978BFF1F938B2B51130C0C
:10DA3000400E7D1B19A833048A0383A70B0B3E9469
:10DA40008357C40163836705050A97E0FFFFE780FA
:10DA5000E08DE342AAFE95460DA08357C50163966B
:10DA600097029305050303A50A004146971001009C
:10DA7000E780802E994611E181462686CA854E852B
:10DA800097F0FFFFE780C06F85A883A50A00130504
:10DA9000040397700000E780A017C14679FD228536
:10DAA000231E940097A00000E780E0742285976011
:10DAB0000000E78060649787FF1F9387E77E9C43A1
:10DAC000A9C323000402228597D00000E78040F01C
:10DAD0004E8581462686CA8597F0FFFFE780406A1B
:10DAE000A1679387070448003EC42302010002C6D1
:10DAF00097F0FFFFE780605741011743FFFF670082
:10DB0000035F89472300F402E1B7397106DE22DCA6
:10DB10004AD8800052D456D25AD026DA4ED65ECE9B
:10DB20002E8A32892A8B97D0FFFFE780207D060559
:10DB3000710541998A8A3301A140232224FC2314D0
:10DB400004FC97D0FFFFE780607B83479A000605BF
:10DB5000350593F7F7072315A4FCA304FA004A85BB
:10DB6000232624FC97E0FFFFE78040799317050107
:10DB7000C1876340F0025681130104FCF2506254E5
:10DB8000D2544259B259225A925A025BF24B216145
:10DB90008280AA844A8597E0FFFFE7802076AA89E1
:10DBA0004A8597E0FFFFE7806075A1659385C50210
:10DBB0002A89130544FC97C0FFFFE780E07E268595
:10DBC00097C0FFFFE7802073854511C94A86CE853F
:10DBD00097C0FFFFE780A06CAA8B21E98945130558
:10DBE00044FC97E0FFFFE780A061A685130544FC95
:10DBF00097E0FFFFE780C062CE85130544FC97E005
:10DC0000FFFFE780E061CA85130544FC97E0FFFF52
:10DC1000E780006101478146130644FCD2855A859E
:10DC200097D0FFFFE780A09DB9B78145130544FC5D
:10DC300097E0FFFFE780C05CA685130544FC97E0F2
:10DC4000FFFFE780E05DCE85130544FC97E0FFFF12
:10DC5000E780005DCA85130544FC97E0FFFFE7807D
:10DC6000205C814497D0FFFFE7804069E3D4A4FAA9
:10DC700083A70B0113971400BA9783D5070099C5A2
:10DC8000130544FC97E0FFFFE78080598504D9BF66
:10DC9000797106D622D44AD000184ECE52CC56CA3C
:10DCA00026D25AC8AE893289AA8A97D0FFFFE78068
:10DCB000E0640605690541990A8A3301A140232AD7
:10DCC00024FC231C04FC97D0FFFFE780206383C75C
:10DCD000990006052D0593F7F707231DA4FCA384DF
:10DCE000F9004A85232E24FC97E0FFFFE7800061BE
:10DCF00093170501C187634FF0005281130104FDA2
:10DD0000B250225492540259F249624AD24A424BCA
:10DD100045618280AA844A8597E0FFFFE780005E24
:10DD2000A1659385A5022A89130544FD97C0FFFFCD
:10DD3000E7808067268597C0FFFFE780C05B854549
:10DD400009C9CA8597C0FFFFE78060582A8B29E17F
:10DD50008945130544FD97E0FFFFE780604AA685EB
:10DD6000130544FD97E0FFFFE780804BCA8513054C
:10DD700044FD97E0FFFFE780A04A01478146130674
:10DD800044FDCE85568597D0FFFFE7804087B5B725
:10DD90008145130544FD97E0FFFFE7806046A685B7
:10DDA000130544FD97E0FFFFE7808047CA85130510
:10DDB00044FD97E0FFFFE780A046814497D0FFFF36
:10DDC000E780C053E3DBA4FA83270B011397140009
:10DDD000BA9783D5070099C5130544FD97E0FFFF67
:10DDE000E78000448504D9BF1743FFFFE702232FD4
:10DDF00083474500404DD5EFFD575DC483469400F1
:10DE000009476363D70A0346B400854663EEC60834
:10DE10008306E40063CA06085C45F9562390D700E0
:10DE20009787FF1F83C787F199E3A304E4009787CF
:10DE3000FF1F9387E7F89C4381E78947A306F40017
:10DE40009787FF1F938747469C4381E789472306AF
:10DE5000F4009705000093854506AA841305040184
:10DE600097F00000E7802010FD57231AF402814745
:10DE70001CDC01489787FF1F23AE87EA9787FF1FA7
:10DE8000938787EB232E040304C0804397D0FFFFC2
:10DE9000E780005161463306C502814522859740DF
:10DEA000FFFFE780C02681473E851743FFFF6700DD
:10DEB0004325FD57D5BF1743FFFFE70243222A84BE
:10DEC0000355450297600000E780E01D19E5231E19
:10DED00004001743FFFF6700C3228357E401F5DB0B
:10DEE000930504FF17450100130545F897E000006E
:10DEF000E780E014F9BF1743FFFFE702431E2E89B6
:10DF0000A16541119385E5032A8436C432C6BE84D7
:10DF10003AC297C0FFFFE780204912472285BA85A1
:10DF200097E0FFFFE780C02D32462285B28597E05B
:10DF3000FFFFE780E02EA2462285B68597E0FFFF2F
:10DF4000E780002E630309029145228597E0FFFFD9
:10DF5000E780C0241146A68597100100E78020E2E3
:10DF600041011743FFFF6700C3198945228597E0E8
:10DF7000FFFFE780A02283C704002300F50083C7CA
:10DF80001400A300F500E9BF1743FFFFE7022315C4
:10DF900083C79500444D054793F7F707A384F50021
:10DFA0001C42411183C707006367F7062E842A8944
:10DFB000B1C003C7D400630FF7021787FF1F130711
:10DFC00027E0184305C3A386F40097A00000E7806C
:10DFD000404A83C7D40099E741657D15974000000A
:10DFE000E780403083D72403918B89C797E00000F6
:10DFF000E780C0134A85A28597F0FFFFE780801075
:10E00000A167C10748003EC42302010002C697F081
:10E01000FFFFE780800541011743FFFF6700630EA4
:10E020001743FFFFE702A30B03D745008D47AA84E0
:10E0300041112E8432892E8563E3E70297E0FFFFCA
:10E04000E780C02BAA8523000900268597C0FFFF23
:10E05000E780E02741011743FFFF6700830A97E04D
:10E06000FFFFE780A0292AC6228597E0FFFFE7800F
:10E07000E028B24585472A862300F900268597C007
:10E08000FFFFE780C021F9B7397106DE22DC26DA0E
:10E0900080004ED652D456D24AD85AD05ECEAE89DF
:10E0A000B284AA8A97D0FFFFE780402406051305B3
:10E0B000250241990A8A3301A140232224FC23141A
:10E0C00004FC97D0FFFFE780602283C79900060514
:10E0D0004D0593F7F7072315A4FCA384F9002685C3
:10E0E000232624FC97E0FFFFE780402193170501DA
:10E0F000C1876340F0025281130104FCF250625464
:10E10000D2544259B259225A925A025BF24B2161BF
:10E110008280AA8B03AB040097C0FFFFE780A01D9D
:10E1200051E583D7440001498544F11793B717009F
:10E13000A301F4FC834734FCA165C9C79385E504BA
:10E14000130544FC97C0FFFFE7800026A685130552
:10E1500044FC97E0FFFFE780A00ADE85130544FC3E
:10E1600097E0FFFFE780C00B834734FC114691E343
:10E170000946DA85130544FC97E0FFFFE780600558
:10E180008144630A0900416B7D1B97D0FFFFE78044
:10E19000E01563CCA40201478146130644FCCE85FA
:10E1A000568597C0FFFFE7808045B1B7A685130667
:10E1B00034FC97000000E780E0E6933415002A89DC
:10E1C00086048DBF9385C504A5BF8327C900139717
:10E1D0001400BA9783D5070063886501130544FCD2
:10E1E00097E0FFFFE780C003850445B71743FFFFB3
:10E1F000E70263EC79711C103EC4B7070F003EC6FE
:10E200001C103EC883C79500AA8A328593F7F7078A
:10E21000A384F500AE89328497E0FFFFE780000E0B
:10E2200093170501C187635AF0062A8A228597E071
:10E23000FFFFE780A00C2A895285032B040097C0BA
:10E24000FFFFE780400B39ED8357440081440544CC
:10E25000F11793B71700A303F10083457100DA8724
:10E260002287CA865286280097000000E780E0C80F
:10E27000014781463000CE85568597C0FFFFE78075
:10E280000038A1679387D70348083ECC230A810052
:10E2900026CE97F0FFFFE78040DD45611743FFFF83
:10E2A0006700E3E4A2851306710097000000E78091
:10E2B00060D7AA84094455D13544E30055FB4A850B
:10E2C00097F0FFFFE78000450D4441D9014497D006
:10E2D000FFFFE780A001634DA400C16B0144FD1B5B
:10E2E00097D0FFFFE7808000634EA4001544B5B7C8
:10E2F000DC4413171400BA9783D7070063832703FE
:10E300000504F1B7D84493171400BA9703D7070050
:10E31000631B770123902701268597A00000E780E3
:10E3200080DB01441DBF050465BF1743FFFFE70203
:10E3300063D983C7950041112A8A93F7F707A3840D
:10E34000F50032852E89328497E0FFFFE78000FBDD
:10E3500093170501C1876353F006AA89228597E0C8
:10E36000FFFFE780A0F92311A1004E85832A040056
:10E3700097C0FFFFE78020F839E5835744008544C4
:10E380000144F11793B71700A300F10003481100EF
:10E3900003572100D6875285CE862686CA8597F0F8
:10E3A000FFFFE7806006A167F10748003EC4230233
:10E3B000910022C697F0FFFFE78020CB4101174371
:10E3C000FFFF670063D3A2851306110097000000CA
:10E3D000E78040C52A84894455D9835721001167B5
:10E3E0008544BA97C2071167C1831307F7EFE36F3C
:10E3F000F7F89787FF1F9387E7B29C4381CB85454A
:10E400001305210097500000E780207583552100F7
:10E410002285814497C0FFFFE78080E425D923103F
:10E420000500228597A00000E78040CD85B71743FF
:10E43000FFFFE70243C883C7950041112A8B93F77A
:10E44000F707A384F50032852E8A328497E0FFFF18
:10E45000E780C0EA93170501C1876351F006AA8AD5
:10E46000228597E0FFFFE78060E92A895685832BA4
:10E47000040097C0FFFFE78000E831E583574400C0
:10E4800081440544F11793B71700A301F100034835
:10E490003100DE875A854A87D6862286D28597F054
:10E4A000FFFFE78060F6A167ED0748003EC4230246
:10E4B000810026C697F0FFFFE78020BB410117438C
:10E4C000FFFF6700C3C2A28513063100970000005A
:10E4D000E78040B5AA8409445DD99167CA97C2070D
:10E4E0001167C1831307F7EF0544E362F7FACA85A2
:10E4F00097C0FFFFE780C0D6014451F9814997D00A
:10E50000FFFFE780A0DF63DBA9009848939719001D
:10E51000BA9703D7070005EF2390270197D0FFFF95
:10E52000E780C0DD1544E384A9F6268597A00000A6
:10E53000E780C0BC9787FF1F9387C79E9C43014419
:10E54000B9D74A8597500000E780C05889B7850938
:10E550007DB71743FFFFE702E3B679713E847C087D
:10E560003EC82E8AB7071400A1653ECAE5057C089F
:10E57000AA89080836C4428932C6BA8AC6843ECC03
:10E5800097C0FFFFE78040E2CA85080897E0FFFFD9
:10E59000E78000C732460808B28597E0FFFFE780B2
:10E5A00020C8A246630A09049D45080897E0FFFFBA
:10E5B000E780C0BE1D4681459740FFFFE78020B53C
:10E5C00063890A089145080897E0FFFFE78000BDCE
:10E5D0001146A68597000100E780607A1008014780
:10E5E0008146D2854E8597C0FFFFE7804001456197
:10E5F0001743FFFF670043B0B685080897E0FFFFA9
:10E60000E78000C21C400808D8439355C70185899C
:10E6100012075183B205D98D97E0FFFFE78040C014
:10E620001C40080883C5870097E0FFFFE78040BDD6
:10E630001C40080883C5A70097E0FFFFE78040BCA7
:10E640001C40080883C5970097E0FFFFE78040BBA8
:10E6500085BF8945080897E0FFFFE78020B483C79E
:10E6600004002300F50083C71400A300F500BDB724
:10E670001743FFFFE70203A583C795004111AA894D
:10E6800093F7F707A384F5003285AE84328497E0D0
:10E69000FFFFE780A0C693170501C187635DF00403
:10E6A0002A89032A040097C0FFFFE780C0C419E944
:10E6B000835744000548F11793B71700A307F100EB
:10E6C000814631A81306F100A28597000000E7807B
:10E6D00060951DC51C459DC783D64700014803476B
:10E6E000F10093078500D2884A86A6854E8597005B
:10E6F0000000E78040E641011743FFFF6700C39F2A
:10E7000009487DBF1D486DBF1743FFFFE702839B8C
:10E7100065715C083EC4B7077B013EC65C083EC815
:10E7200083C795002A8A328593F7F707A384F500FB
:10E73000AE8997E0FFFFE78040BA8357E100E1C769
:10E740008945280097C0FFFFE78000C68145280063
:10E7500097E0FFFFE780C0AA97C0FFFFE780E0CB0C
:10E760009787FF1F938747B49C431774FF1F034489
:10E77000E45CAA843334800099C31364240097773F
:10E78000FF1F9387E7639C4399C313644400977703
:10E79000FF1F938727799C4399C31364840083D513
:10E7A00004002800014997E0FFFFE78060A783D5B8
:10E7B0002400280097E0FFFFE78080A683D544006F
:10E7C000280097E0FFFFE780A0A597D0FFFFE78034
:10E7D000E0AD93150501C181280097E0FFFFE780B8
:10E7E00020A4A285280097E0FFFFE78060A39C4457
:10E7F0006360F902014781463000CE85528597C09B
:10E80000FFFFE780C0DF59611743FFFF6700C38E3A
:10E81000DC441314490028003E9497E0FFFFE78092
:10E820006096834744000347540089070607BA9758
:10E830008607E36AF5FC835524002800814A97E0A7
:10E84000FFFFE780E09D83454400280097E0FFFF3D
:10E85000E780009B83455400280097E0FFFFE78096
:10E86000209A8347440063C9FA00814A83475400D1
:10E8700063C1FA020509A5BF1C4413975A0028007A
:10E88000BA9783D50700850A97E0FFFFE780409994
:10E89000C9BF032BC40093975A0028003E9B8355A1
:10E8A0002B00850A97E0FFFFE780809783550B00D8
:10E8B000280097E0FFFFE780A0964DBF1743FFFFBA
:10E8C000E702E3815C4993E717005CC997A0000069
:10E8D000E78020B61743FFFF6700A3821733FFFFCF
:10E8E000E702E37F2E84814597F0FFFFE780C0E7D2
:10E8F00005C583570500FD172310F50009C483578C
:10E9000025002310F40097000000E78060FB01451C
:10E910001733FFFF6700E37E31457DD823100400E5
:10E92000C5BF1733FFFFE702E37983C795004111A5
:10E930002A8A93F7F707A384F50032852E8932845B
:10E9400097E0FFFFE780809B93170501C18763561F
:10E95000F006AA89C145228597E0FFFFE780A080E5
:10E960002A8B4E85832A040097C0FFFFE780A0987A
:10E9700031E983574400231101000544F11793B78F
:10E980001700A300F1008144034811000357210040
:10E99000D6875285CE862286CA8597F0FFFFE7800C
:10E9A000A0A6A1679387170248003EC423028100F6
:10E9B00026C697E0FFFFE780406B41011733FFFF5A
:10E9C0006700837313061100A28597F0FFFFE780AD
:10E9D0006065AA8409E523110100094475B7930510
:10E9E00021005A8597000000E78080EF83572100BF
:10E9F0002A84D9DB9777FF1F9387C7529C4381CB2B
:10EA000085451305210097500000E78000158355C8
:10EA100021002685314497C0FFFFE78060842DD513
:10EA200023100500268597900000E780206D0144A3
:10EA3000A1BF1733FFFFE702836A41112E896C00E3
:10EA4000AA8402C697F0FFFFE78000D20DC10357EA
:10EA5000050005072310E50097000000E78040E669
:10EA600081473E8541011733FFFF670083693247C5
:10EA7000954765DBCA85268597300000E780400D05
:10EA8000C147E34005FE3244854741462310F40068
:10EA900083570900A685130544002311F40097004D
:10EAA0000100E780C02D228545BF1733FFFFE70235
:10EAB000636183C795004111AA8A93F7F707A3847E
:10EAC000F5003285AE89328497E0FFFFE78000834E
:10EAD00093170501C1876356F0062A8AC14522852E
:10EAE00097D0FFFFE7802068AA845285032B04009B
:10EAF00097C0FFFFE780208031E98357440023114E
:10EB000001008544F11793B71700A300F1000144F9
:10EB10000348110003572100DA875685D2862686DE
:10EB2000CE8597F0FFFFE780208EA16793870702CD
:10EB300048003EC42302910022C697E0FFFFE78011
:10EB4000C05241011733FFFF6700035BA285130624
:10EB5000110097F0FFFFE780E04C2A8409E52311BC
:10EB60000100894475B726859305210097000000B0
:10EB7000E78060ECAA8449FD83552100228597B087
:10EB8000FFFFE780E06D49F5014997C0FFFFE7808F
:10EB9000E076635DA900184893171900BA9703D768
:10EBA00007000DEF035721002390E70097C0FFFFF8
:10EBB000E780C074630625039777FF1F9387873626
:10EBC0009C4399C70355210097500000E78080F0CF
:10EBD000228597900000E78060521DBF050975B738
:10EBE00095443DB705C19307F00F630FF500C54786
:10EBF000630CF5009307F5FF05453315F500420555
:10EC0000418182800145828041657D158280B9E91C
:10EC10001733FFFFE702A34C034506033284970036
:10EC20000000E78060FC9305803EB305B502C20595
:10EC3000C18181CD0357E402854763F8E7001305DE
:10EC4000040197E00000E78020428357E402416717
:10EC50007D176385E700FD172317F4021733FFFFC5
:10EC60006700234A82801733FFFFE702C344004254
:10EC700083C79500444D0349140093F7F707A38415
:10EC8000F50083470400220911673369F900A16781
:10EC9000B347F90041112A8BAE8A63ECE70E834734
:10ECA00024001307C00EB91793F7F70F6373F7101B
:10ECB00003473400C14763EEE70E83474400130760
:10ECC000E00793C707086371F70C83498400834703
:10ECD0007400A209B3E9F900856763F7F90A034AEA
:10ECE0006400834754004E85220A336AFA00975025
:10ECF0000000E780403B61C123962403834B34002E
:10ED0000137AFA00239A3403238874032399440363
:10ED100093890401631C090023A6040223980402BA
:10ED20004E8597E00000E78060363DA0034924004F
:10ED30004A8597000000E78020EB2397A4028347D1
:10ED400044004E85A388F402E38D0BFCE30B09FC21
:10ED500097E00000E780202F97900000E780007385
:10ED600081460146D6855A8597E0FFFFE780005827
:10ED7000A167938797033EC423020100480002C69F
:10ED800097E0FFFFE780602E41011733FFFF670028
:10ED900003368544A2862686D6855A8597E0FFFFEE
:10EDA000E780C054A167938797033EC42302910074
:10EDB000F1B7BD44C5B79144F1BF1733FFFFE70278
:10EDC000633001111C08404D3EC2B7070F003EC41E
:10EDD0001C083EC62A89AE8997C0FFFFE780E0D9AC
:10EDE000585C1C5C6346B70E6394E50063E2A70EB3
:10EDF0003385A740B3B7A700B305B7401306803EDD
:10EE000081469D8D97000100E78080B7931405012E
:10EE1000C180A1659385C503480097B0FFFFE780D7
:10EE2000A0588145480097D0FFFFE780603D83559B
:10EE30000404480097D0FFFFE780803E83552404F8
:10EE4000480097D0FFFFE780A03D814589CCC1678E
:10EE5000FD179305F00F6388F40026859750000096
:10EE6000E780E0E0AA85480097D0FFFFE7804039BF
:10EE700003554404814501CDC167FD179305F00F8B
:10EE80006307F50097500000E78060DEAA85480020
:10EE900097D0FFFFE780C03683456404480097D0D1
:10EEA000FFFFE780E03583457404480097D0FFFFFB
:10EEB000E7800035500001478146CE854A8597B0EE
:10EEC000FFFFE780C07305611733FFFF6700C322B0
:10EED000814481B71733FFFFE702632083C79500A2
:10EEE00093F7F707A384F50097000000E78020ED73
:10EEF0001733FFFF6700E3201733FFFFE702831C90
:10EF000083C795004111404D93F7F707A384F5009F
:10EF10002A8A3285B284AE8997D0FFFFE780003E0F
:10EF20002A8B268597D0FFFFE780403D2A892685DA
:10EF300097D0FFFFE780603A93170B0163CA07027F
:10EF4000E177CA97C207C183116763E3E7029307BA
:10EF50000910C207C1831307B00F637BF700931733
:10EF60000901C187AA8A634AF000C54763FE5701B9
:10EF700041011733FFFF6700231897B0FFFFE780B9
:10EF80000028E31725FFD5B763080B0263060902C3
:10EF9000814463890A02B7077F00231064052311A7
:10EFA00024057CC0568597000000E780E0C39304E9
:10EFB000803EB304950239A0B7077F0023200404E4
:10EFC0007CC081440355240497E00000E780A0A39F
:10EFD000A1C497C0FFFFE78040BA269593D7F441BC
:10EFE00033379500AE97BA9708DC5CDCCE85528546
:10EFF00097000000E780A0DC99E023220404A167C9
:10F000009387B70348003EC42302010002C697E07D
:10F01000FFFFE7808005A9BF814701481CDC232E44
:10F020000403E9B71733FFFFE702630B97C0FFFF45
:10F03000E7800037E1473305F5029145975000001E
:10F04000E78000C5E55711C59777FF1F23A6A7CE18
:10F0500081473E851733FFFF6700A30A854717776F
:10F06000FF1F230DF7CC82801733FFFFE702230732
:10F070009777FF1F938707CC80433DC083570404D5
:10F080006390A70683572404639CB7043689B2842F
:10F0900097C0FFFFE78060AE5C5C63C3B704639515
:10F0A000B7001C5C63EEA7028347640463F3F400BB
:10F0B000A6872303F4048347740463F39700A687A9
:10F0C000A303F4048357440441677D176385E70075
:10F0D00085072312F4043C4481C7CA85268582979C
:10F0E0001733FFFF6700E3019777FF1F938787C4FC
:10F0F0009C43014599C303C5870082801733FFFFF6
:10F10000E702E3FD0111B70707003EC683C795007C
:10F11000584D0AC493F7F7070AC8A384F5002A8953
:10F12000AE8411CB1C4283C707002304F7009790DD
:10F130000000E7800034216493055402280097B052
:10F14000FFFFE780602697000000E78020FAAA858D
:10F15000280097D0FFFFE780A00A300001478146D2
:10F16000A6854A8597B0FFFFE780604913044402F3
:10F17000480822CC230A010002CE97E0FFFFE78077
:10F18000C0EE05611733FFFF6700A3F71733FFFFDA
:10F19000E702E3F401117C003ECAB70707003ECC4A
:10F1A0007C003ECE83C795002E84AA8493F7F70790
:10F1B000A384F500A16593855502480897B0FFFF29
:10F1C000E780801E97000000E78040F2AA8548088B
:10F1D00097D0FFFFE780C002500801478146A28513
:10F1E000268597B0FFFFE780804105611733FFFF59
:10F1F000670023F19777FF1F9387C7B39C430945A7
:10F2000099C303C5970082809777FF1F938787B2C2
:10F210009C43094599C303C5D70082809777FF1F98
:10F22000938747B19C43014599C303C5A7008280DA
:10F230001733FFFFE70203E90111B70708003EC6D5
:10F2400083C79500404D0AC493F7F7070AC8A38403
:10F25000F5002A89AE8429C41442854703C70600F5
:10F2600063E0E70A83479400094681496380C70247
:10F27000B307F740A304E400B339F00083C71600D6
:10F280002305F40097900000E780A01E0357240395
:10F29000058B19C76386090097D00000E78000E955
:10F2A000216493058402280097B0FFFFE780C00F18
:10F2B00097000000E78040F4AA85280097D0FFFF60
:10F2C000E78000F497000000E78080F5AA85280019
:10F2D00097D0FFFFE780C0F2014781463000A68546
:10F2E0004A8597B0FFFFE780803113047402480815
:10F2F00022CC230A010002CE97E0FFFFE780E0D690
:10F3000005611733FFFF670023DF1733FFFFE702B5
:10F3100003DD01117C003ECAB70708003ECC7C002B
:10F320003ECE83C795002E84AA8493F7F707A38463
:10F33000F500A16593858502480897B0FFFFE78037
:10F34000A00697000000E78020EBAA85480897D028
:10F35000FFFFE780E0EA97000000E78060ECAA8505
:10F36000480897D0FFFFE780A0E950080147814691
:10F37000A285268597B0FFFFE780602805611733D7
:10F38000FFFF670003D89777FF1F9387A79A9C43D7
:10F39000014599C303C5B70082801733FFFFE70219
:10F3A00003D40111B70707003EC683C79500404D3F
:10F3B0000AC493F7F7070AC8A384F5002A89AE8424
:10F3C00005C81C42054783C707006368F706034763
:10F3D000B400630FF700A305F40097900000E780E6
:10F3E00040098347B400B9CF97D0FFFFE78040BE04
:10F3F00021649305B400280097B0FFFFE780C0FAAE
:10F4000097000000E78060F8AA85280097D0FFFFEA
:10F41000E78000DF014781463000A6854A8597B026
:10F42000FFFFE780C01D2904480822CC230A010001
:10F4300002CE97E0FFFFE78040C305611733FFFF6F
:10F44000670023CC97D0FFFFE78020BF55B7173365
:10F45000FFFFE702C3C801117C003ECAB7070700DF
:10F460003ECC7C003ECE83C795002E84AA8493F7C1
:10F47000F707A384F500A165AD05480897B0FFFF25
:10F48000E78080F297000000E78020F0AA85480816
:10F4900097D0FFFFE780C0D6500801478146A2857C
:10F4A000268597B0FFFFE780801505611733FFFFC2
:10F4B000670023C59777FF1F9387C7879C4309453C
:10F4C00099C303C5C70082801733FFFFE70223C13A
:10F4D00001117C00AE843ECAA165B70707002A84EB
:10F4E0003ECCD1057C0048083ECE97B0FFFFE780B8
:10F4F000A0EB97000000E78020FCAA85480897D081
:10F50000FFFFE780E0CF500801478146A6852285AE
:10F5100097B0FFFFE780A00E05611733FFFF67007C
:10F5200043BE1733FFFFE70283BB83C7950093F702
:10F53000F707A384F50097000000E78020F9173350
:10F54000FFFF670003BC1733FFFFE702A3B783C7C2
:10F5500095000329C501411193F7F707A384F5002E
:10F560001C4283C90700854763E637079777FF1F6B
:10F57000938787D39C432E84AA8485CF970000006D
:10F58000E78080F389476306F50263040902834735
:10F59000C900638037032306390197900000E78094
:10F5A00040ED83572903898B89C797D00000E780F6
:10F5B000E0B72685A28597000000E78020F1A167CB
:10F5C000CD0748003EC42302010002C697E0FFFFBA
:10F5D000E780A0A941011733FFFF6700E3B19767F8
:10F5E000FF1F938727759C431D4599C303C5E700FB
:10F5F00082801733FFFFE70283AE0111B7070700D0
:10F600003EC683C79500584D0AC493F7F7070AC84A
:10F61000A384F5002A89AE8415C71C4283C707005E
:10F6200093968701E18663C4060685466381D70603
:10F630008346E7006388F6002307F70097900000F1
:10F64000E78020E321649305E400280097B0FFFFE2
:10F65000E78080D597000000E780A0F8AA85280001
:10F6600097D0FFFFE780C0B9014781463000A685EB
:10F670004A8597B0FFFFE78080F83504480822CC20
:10F68000230A010002CE97E0FFFFE780009E05619C
:10F690001733FFFF6700E3A61733FFFFE70223A43A
:10F6A00001117C003ECAB70707003ECC7C003ECE6D
:10F6B00083C795002E84AA8493F7F707A384F500E7
:10F6C000A165B905480897B0FFFFE780E0CD970036
:10F6D0000000E78000F1AA85480897D0FFFFE78087
:10F6E00020B2500801478146A285268597B0FFFFCA
:10F6F000E780E0F005611733FFFF670083A0173351
:10F70000FFFFE702239CAA8401441769FF1F130926
:10F71000A962E14997C0FFFFE78080C86344A40065
:10F72000014519A833053403832709003E95835703
:10F7300025006397970011051733FFFF6700C39BF0
:10F740000504C9BF032E8500630A0E121763FF1F4D
:10F750001303437D032303006315030029436390D0
:10F76000061203234E01631503001D43639907101E
:10F770001733FFFFE7022394C689428A3E89BA8A7B
:10F78000B684328BAE8B2A84B5E103554E0019E561
:10F7900001431A851733FFFF67006395A167A98F9F
:10F7A000116763FBE70097000000E78080F5814563
:10F7B00097F0FFFFE780C0120844B70700E0584108
:10F7C000F98F18455CC1B707001FF98F1CC55C494C
:10F7D00091C7610597E00000E780408BE38A09FA52
:10F7E000228597900000E78060C65DB7328597C09C
:10F7F0000000E78040430D4349DD1C44116703D5F9
:10F800004700A167A98F63FBE70097000000E7802E
:10F8100040EF814597F0FFFFE780800C03238400D1
:10F8200093164B01D1828347B3000356630085884A
:10F83000FD8BA305F300FD777D8E558EFD76FD16BD
:10F84000B204F18E83274301C58E23127301231363
:10F85000D3002304530123052301A3044301BDDF87
:10F86000228597B0FFFFE78060CCAA850844B5D118
:10F87000610597D00000E780207F8DB71D431A8572
:10F8800082801733FFFFE702E3830569AA84AE890C
:10F89000328A0144FD5A7D1997C0FFFFE78000A519
:10F8A0006347A40001451733FFFF6700E384D84492
:10F8B00093171400BA9703D70700631F37032390E9
:10F8C000570163070A00268597900000E780A08013
:10F8D0009C449DC383D76700B3F72701639E37011C
:10F8E000D2880148814701478146014681452685E6
:10F8F00097000000E78040E5050479BF1723FFFF6C
:10F90000E702437C79711C103EC4B7070F003EC666
:10F910001C103EC883C79500AA8A328593F7F70763
:10F92000A384F5002E89328497D0FFFFE780009DE5
:10F9300093170501C187635AF006AA89228597D0DB
:10F94000FFFFE780A09B2A8A4E85032B040097B017
:10F95000FFFFE780409A39ED835744008144054416
:10F96000F11793B71700A303F10083457100DA87FD
:10F970002287D2864E86280097E0FFFFE780E05777
:10F98000014781463000CA85568597B0FFFFE78062
:10F9900000C7A1679387F70348083ECC230A81007C
:10F9A00026CE97D0FFFFE780406C45611723FFFF0D
:10F9B00067008374A2851306710097E0FFFFE7805C
:10F9C0006066AA84094455D1528597E0FFFFE7801D
:10F9D00060D40D4459D90546D2852685970000008C
:10F9E000E78060EA2A8451B71723FFFFE702236FFD
:10F9F000835507000346270041112A842E8532C60D
:10FA00002EC497E0FFFFE780E0D001C93246A2454F
:10FA1000228597000000E78000E741011723FFFFE0
:10FA20006700236E1723FFFFE702E36883C7950093
:10FA30004111AA8A93F7F707A384F5003285AE89AE
:10FA4000328497D0FFFFE780608B93170501C18751
:10FA50006357F00AC1452A8A228597C0FFFFE780D5
:10FA600080702A8D228597D0FFFFE78020892A8920
:10FA7000228597D0FFFFE7804086930705F893F72C
:10FA8000F70F1307E007AA8B637BF706228597D051
:10FA9000FFFFE78080842A8C228597D0FFFFE780D4
:10FAA000C083AA8C5285032B040097B0FFFFE78028
:10FAB000808439E983574400231101008144F11700
:10FAC00093B71700A300F1000544034711008356C4
:10FAD0002100938784005685DA8822885286CE8555
:10FAE00097F0FFFFE78020A7A167E90748003EC421
:10FAF0002302810026C697D0FFFFE780005741010F
:10FB00001723FFFF6700A35E13061100A28597E08D
:10FB1000FFFFE7802051AA8409E523110100094471
:10FB20006DB7930521006A8597F0FFFFE780A0F08D
:10FB30002A8441FD835521009356C90013164901BB
:10FB400085486688E2875E87858A51822685970088
:10FB50000000E78060BF2A848DBF1723FFFFE70204
:10FB6000835583C7950041112A8B93F7F707A38428
:10FB7000F5003285AE89328497C0FFFFE7800078B8
:10FB800093170501C1876352F00A2A8A228597C01C
:10FB9000FFFFE780A076AA8A228597C0FFFFE78053
:10FBA000E0752A89228597C0FFFFE78000739307DD
:10FBB00005F893F7F70F1307E0072A8C6377F7062A
:10FBC000228597C0FFFFE7804071AA8C228597C0ED
:10FBD000FFFFE78080702A8D5285832B040097A059
:10FBE000FFFFE780407139E58357440085440144B5
:10FBF000F11793B71700A301F100034731009307F2
:10FC000084005A85DE882688D6865286CE8597F06F
:10FC1000FFFFE78040948D4748003EC423029100D7
:10FC200022C697D0FFFFE780404441011723FFFF22
:10FC30006700E34BA2851306310097E0FFFFE780E2
:10FC4000603E2A84894455D99356C9001316490148
:10FC500085486A88E6876287858A5182D6859700BB
:10FC60000000E78060AEAA8449BF1723FFFFE702C8
:10FC700063452A8981440144617A916A176BFF1FA9
:10FC8000130B4B2A97B0FFFFE780406763C7A400C0
:10FC900022851723FFFF67002346832709009399D6
:10FCA0001400CE9703D5070033074501420741836F
:10FCB0006364570305C103270B0019C785453E85BB
:10FCC00097400000E78060E9832709000504CE978C
:10FCD0002390070085047DB797000000E78060A2AD
:10FCE000832709000504CE972390070065D5814539
:10FCF00097F0FFFFE780C0BEF1BF1723FFFFE702C9
:10FD0000633C83C7950041112A8A93F7F707A384C0
:10FD1000F50032852E89328497C0FFFFE780005EB0
:10FD200093170501C187635AF004AA89832A040046
:10FD300097A0FFFFE780205C31E5835744008544AE
:10FD40000144F11793B71700A301F10003483100F4
:10FD5000D68752850147CE862686CA8597D0FFFF73
:10FD6000E780806AA167F50748003EC4230291003E
:10FD700022C697D0FFFFE780402F41011723FFFFE6
:10FD800067008337A2851306310097E0FFFFE78005
:10FD900060292A8489445DD99767FF1F9387871854
:10FDA0009C4381CF044997B0FFFFE7802055AA8587
:10FDB000268597400000E78040DA1305040197008C
:10FDC0000000E780C0EA228597800000E7800033CA
:10FDD0008144ADBF1723FFFFE702E32D83C79500E2
:10FDE0004111AA8A93F7F707A384F5003285AE89FB
:10FDF00032842311010097C0FFFFE7802050931742
:10FE00000501C1876354F0062A8AC145228597C03F
:10FE1000FFFFE7804035AA8B5285032B040097A093
:10FE2000FFFFE780404D21E98357440085440144AA
:10FE3000F11793B71700A300F1000348110003570F
:10FE40002100DA875685D2862686CE8597D0FFFF99
:10FE5000E780805BA1679387270248003EC42302A6
:10FE6000910022C697D0FFFFE78020204101172391
:10FE7000FFFF6700C327A2851306110097E0FFFF6D
:10FE8000E780401A2A8489444DD99767FF1F9387DA
:10FE9000670998433E8901CF044997B0FFFFE78087
:10FEA000E045AA85268597400000E78000CB130532
:10FEB000040197000000E78080DB97B0FFFFE78038
:10FEC000E04395443DD9930521005E8597F0FFFFFF
:10FED000E78060B6AA8435F11C48035721002285CB
:10FEE0002390E70097800000E780402183270900E6
:10FEF000A9D70355210097400000E780A0BD35BF7A
:10FF00001723FFFFE702231B83C795004111AA8A2D
:10FF100093F7F707A384F5003285AE89328497C042
:10FF2000FFFFE780A03D93170501C1876351F006ED
:10FF30002A8A228597C0FFFFE780403C2A895285A4
:10FF4000032B040097A0FFFFE780E03A31E58357D9
:10FF5000440085440144F11793B71700A301F10051
:10FF600003483100DA8756854A87D2862686CE85B1
:10FF700097D0FFFFE7804049A167F90748003EC4DA
:10FF80002302910022C697D0FFFFE780000E4101B7
:10FF90001723FFFF6700A315A2851306310097E022
:10FFA000FFFFE78020082A8489445DD99167CA97BA
:10FFB000C2071167C1831307F7EF8544E362F7FABD
:10FFC0009767FF1F938707F69843BE8B01CF0449BD
:10FFD00097B0FFFFE7808032AA8526859740000012
:10FFE000E780A0B71305040197000000E78020C850
:10FFF00097B0FFFFE780803095443DD11C482285B3
:020000040001F9
:1000000081442390270197800000E780200F83A779
:100010000B00B9D74A8597400000E780A0AB89B7AD
:100020001723FFFFE702A30B2A844105B284970040
:100030000000E780C0C311C5228597800000E780DB
:10004000E00B81460146A685228597800000E78067
:10005000C04E1C4C89C7DC4799C322858297172361
:10006000FFFF6700030A9767FF1F9387A7CC9C4396
:10007000014599C31385070182809767FF1F938706
:1000800067CB884382801723FFFFE702430593175E
:10009000C600DD8DC2054111C1812A8432C697C0D8
:1000A000FFFFE780E0173246228511829375F60F35
:1000B00097C0FFFFE780C01441011723FFFF6700CF
:1000C00043041723FFFFE702E3FF79713C083ED2A8
:1000D000B7070C003ED43C083ED683C79500AE84DB
:1000E0002A8993F7F707A384F500A1659385350462
:1000F000481097A0FFFFE780202BC165FD15014444
:10010000176AFF1F130A8AE3930A400EAE892E8BEB
:100110002EC697B0FFFFE7806021420593170401C8
:100120004181C183B24563E9A702C167FD176387B7
:10013000F500481097C0FFFFE780800E5010014780
:100140008146A6854A8597A0FFFFE780404B456121
:100150001723FFFF670043FA3307540383270A0B73
:10016000BA9703D6C701630A3601638A350148107E
:1001700097000000E78060F1DA85050451BFB28581
:10018000EDBF1723FFFFE70203F379717C083EC838
:10019000B70711003ECA7C083ECC83C79500AA89E8
:1001A000328593F7F707A384F5002E8997C0FFFFE8
:1001B000E780C01485676378F504A165AA84890582
:1001C000080897A0FFFFE780201E268597400000C3
:1001D000E78060ED133415000A04A285080897C073
:1001E000FFFFE780E001A685080897C0FFFFE780D2
:1001F000200325CC014781461008CA854E8597A06B
:10020000FFFFE780C03F45611723FFFF670023EE34
:10021000B30754030327CA0ABA9703D70700631C1E
:10022000970003D627006380650508089700000043
:10023000E780A0E5DE8505042EC697B0FFFFE780C6
:10024000E00F4205931704014181C183B245E3E108
:10025000A7FCC167FD17E38FF5F8080897C0FFFFFB
:10026000E78000FC41BFB285F9B7C165FD150144C7
:10027000176AFF1F130A8ACC930A80022E8BAE8B5B
:1002800065BF1723FFFFE70283E518418347170087
:1002900083460700A207D58FD207D1832390F500AC
:1002A00083472700034717008D45A207D98F918305
:1002B0002310F60097C0FFFFE780A0E91723FFFF98
:1002C000670023E41723FFFFE702C3DFC164014493
:1002D0001769FF1F130989C693098002FD1497B09F
:1002E000FFFFE780A0056347A40001451723FFFF38
:1002F000670083E0330534038327C90A3E9583579B
:100300000500E38597FE0504D9BF1723FFFFE70229
:1003100063DB2A8AAE89B284B68A97400000E78000
:1003200080D819E591473E851723FFFF6700C3DC9E
:100330002A894E8597C00000E780E08E2A84638E6C
:100340000A048D476DD103570500C547E31D47FDDE
:100350000347F9018546AD47E317D7FC83474500BE
:1003600081CF4146A6855D0597F00000E780C09EDD
:10037000814755D9AD4745BF130965012302E50003
:10038000CA85268597100000E780606231C1A547C5
:10039000E38B0AF82302040079B705C183570500EF
:1003A000E39247F94146A685190597F00000E780DA
:1003B000A09A81472DD99947BDB74E859700000077
:1003C000E78080F02A84954739DD130955004DBF39
:1003D0004146A68523104401231134011305190059
:1003E00097F00000E780A099228597800000E780C1
:1003F000A0EA81470DBF1723FFFFE70243CE7971C3
:100400007C003ECCB7070A003ECE7C003ED083C7BE
:100410009500B2842E8493F7F707A384F5001306A2
:10042000A1002A892C00268597000000E780A0E51E
:10043000A16528088D0597A0FFFFE780E0F69040B2
:100440008355A10003558100854697000000E78091
:1004500000ECAA84AA85280897C0FFFFE78040DA4D
:100460000356A10083558100280897000000E7800B
:10047000C0C1300801478146A2854A8597A0FFFF89
:10048000E780E017854748103ED42302910202D648
:1004900097D0FFFFE78060BD45611723FFFF67002E
:1004A00043C61723FFFFE70283C379717C003ECC6C
:1004B000B7070A003ECE7C003ED083C79500B284C9
:1004C0002E8493F7F707A384F5001306A1002A8969
:1004D0002C00268597000000E780E0DAA165280857
:1004E0008D0597A0FFFFE78020EC90408355A10089
:1004F00003558100814697000000E78040E1AA840F
:10050000AA85280897C0FFFFE78080CF0356A10087
:1005100083558100280897000000E78000B7300865
:1005200001478146A2854A8597A0FFFFE780200DFD
:1005300048102302910202D402D697D0FFFFE78031
:10054000C0B245611723FFFF6700A3BB1723FFFF5E
:10055000E702E3B897000000E78060DB1723FFFFA6
:10056000670023BA9757FF1F9387077D88438280D0
:100570001723FFFFE702A3B6835725004111AE847E
:100580002A842307B10017F5FFFF130525466C00E9
:100590002316F10097A0FFFFE780604891C42285F1
:1005A00097800000E780E0D6FD572310F400130683
:1005B00020028145130554009720FFFFE78020B5F6
:1005C00041011723FFFF6700C3B31723FFFFE702B3
:1005D00063AF79717C003ECCB7070A003ECE7C0049
:1005E0003ED083C79500AA89AE8493F7F70732857A
:1005F000A384F5001306A1002C0097000000E780FB
:1006000080C803558100114497400000E780A0A9ED
:1006100015C50355A100014497B00000E780A06014
:1006200011CD035705008357810045446318F70037
:10063000854597000000E780E0F3014421699305B8
:100640003900280897A0FFFFE78000D6A285280878
:1006500097C0FFFFE780C0BA0356A1008355810011
:10066000280897000000E78040A230080147814633
:10067000A6854E8597A0FFFFE78060F848104AD412
:100680002302810202D697D0FFFFE780009E4561DA
:100690001723FFFF670043A61723FFFFE70283A28C
:1006A0009757FF1F938707692A8488432E8915C5AA
:1006B000035745038357C4016311F702232605023C
:1006C00023180502410597D00000E780209C6306AF
:1006D000090097800000E78060DB81449769FF1F75
:1006E0009389C985130A800297B0FFFFE78000C590
:1006F00063C4A4049757FF1F9387876C9C4399C7D3
:100700000355C40197200000E780C0BD63070900BE
:10071000228597800000E780C0A01306400E814527
:1007200022859720FFFFE780809EFD57231EF4005F
:100730001723FFFF6700439C3385440383A7C90A3F
:100740003E95035705008357C4016317F700CA8518
:1007500097000000E78000E2850479B71723FFFFC8
:10076000E702439683C795004111AA8993F7F707DB
:10077000A384F5003285AE8497C0FFFFE78000B800
:1007800085676378F5042A8997400000E780A09187
:10079000014401CD83D70400314463882701854596
:1007A00097000000E78080EF01444E85A2864A86CC
:1007B000A68597D0FFFFE780A09CA16793871704C9
:1007C00048003EC42302810002C697D0FFFFE780A5
:1007D000C08941011723FFFF670003921723FFFF22
:1007E000E702438E9757FF1F9387C754804329C45E
:1007F000014597C00000E780002181470148C1649E
:100800001CDC232E0403232004041759FF1F1309A3
:10081000E97201449309400EFD1497B0FFFFE78091
:10082000E0B0634FA400814517F5FFFF1305857FF6
:1008300097A0FFFFE780A01E1723FFFF6700C38B71
:10084000330534038327090B3E958357C50163871E
:100850009700854597000000E78040E4050475BFD8
:100860009357050113D78700A380F500931705015F
:10087000C183A1832380E5002381F500A381A50026
:1008800082801723FFFFE70283852300050083C7CB
:100890001500A300F50083C725002301F50083C7D9
:1008A0003500A301F50083C745002302F50083C787
:1008B0005500A302F50083C7650093059500A303C7
:1008C00005002303F500230405003285970000008E
:1008D000E78040F91723FFFF6700A3821713FFFF8C
:1008E000E702437E4111E9540DCD85CD93F9C5FF53
:1008F0002E842A89AA84338AA900B7EA04006318DF
:100900009A020D88854411CCB7E704009C5F82975A
:100910002AC622866C003305390197E00000E78083
:100920000046268541011713FFFF6700E37C83A77C
:100930008A039104829793170501C183A183A38E33
:10094000F4FE93570501238FF4FEA183238EA4FEAA
:10095000A38FF4FE6DB763E6D5021713FFFFE7021E
:100960000378B28741113686BE8536C697E000000F
:10097000E780E040B246410136851713FFFF67006C
:100980004378814636858280838705001387F5008A
:100990003D05FD8793F77708834607007D1586069A
:1009A000B58FA300F5006307B7007D1783471700D5
:1009B0009D83DDB782801713FFFFE7024372B7E71D
:1009C000040083A7070932872A863A858297133560
:1009D00015001713FFFF6700C37215C181478DC152
:1009E0001713FFFFE702A36F414697E00000E7807F
:1009F000003985473E851713FFFF670083708147E5
:100A00003E8582801DCD1713FFFFE702436D4146EF
:100A100081452A849710FFFFE780606F414681453A
:100A2000130504039710FFFFE780606E0147C1675D
:100A30002322040438C87CC805451713FFFF67004C
:100A4000436C0145828081473DCDB5CD1713FFFF33
:100A5000E702E368B2842E891306800581452A8463
:100A60009710FFFFE780A06ACA8524C426859700F7
:100A70000000E780C0F64146814522859710FFFFC0
:100A8000E780E0683044A285228597000000E78077
:100A9000C0F293040401A285268597000000E78038
:100AA000E0EEA6851305040297000000E78000EE43
:100AB000228597000000E78020F585473E851713C3
:100AC000FFFF670003643E8582801713FFFFE70284
:100AD000635F4111E9540DCD85CD93F9C5FF2E8497
:100AE0002A89AA84338AA900B7EA040063984403D8
:100AF0000D88814411CCB7E704009C5F82972AC619
:100B000022866C003305390197E00000E78020273A
:100B1000268541011713FFFF6700035E83A78A0341
:100B20009104829793170501C183A183A38EF4FEDC
:100B300093570501238FF4FEA183238EA4FEA38F78
:100B4000F4FE6DB765CD1713FFFFE702A357B2841C
:100B500011E605451713FFFF6700035A2A842E8903
:100B60000145EDD93C487848B3E6E700E5D69386E1
:100B7000F7FFB3B7F6007D17032A4404BA9734C8C9
:100B80007CC863050A06C14913050A03B3894941B4
:100B90002295637D3601B2862E86A68597000000D9
:100BA000E780A0DB7C40BE9464C065B7CE862E860D
:100BB000CE8597000000E78040DAC114D2944E99A8
:100BC00023220404A2879306040103C7070003C677
:100BD00007038507318FA38FE7FEE398F6FE3044C5
:100BE000A285228597000000E78020DD2699C14973
:100BF0003306994063EC9900A9DCA686A685130507
:100C0000040397000000E78040D579BF8147B30611
:100C1000F4003307F6000347070083C50600850785
:100C20002D8F2380E600E39437FF3044A285228590
:100C300097000000E78060D8C1145DBF0145828045
:100C40000DC11713FFFFE702834913068005814595
:100C50009710FFFFE780A04B05451713FFFF6700C4
:100C6000434A01458280814749C5C1C51713FFFF2B
:100C7000E702E346FC4141462E84AA846399C704F7
:100C800013860501A2878146C14503C7070003C536
:100C900007038507298F3305D60003450500850620
:100CA000298FA38FE7FEE392B6FE3044A285268506
:100CB00097000000E78060D0228597000000E78061
:100CC00060F885473E851713FFFF67008343138550
:100CD00007031D8E814522959710FFFFE780204373
:100CE0007C40130700F813060402A2972388E7024A
:100CF00051BF3E8582801713FFFFE702433E6D71AF
:100D00002E84B284AA8590102800368997000000AE
:100D1000E780A0D309EDD55725A050400C4028000E
:100D200097000000E78040E27DD5FD142104F5F432
:100D30002C004A8597000000E78020F3814761DDA1
:100D40003E8551611713FFFF6700A33B1713FFFF99
:100D5000E702E33841112EC432C62C000546970045
:100D60000000E78080F941011713FFFF6700633936
:100D70001713FFFFE702A33601112A842EC602C80B
:100D800002CA02CC02CE97E00000E780C023B24640
:100D90002A86A285080897000000E78060FB13758B
:100DA000F50F05611713FFFF6700A3351713FFFF4A
:100DB000E702E3327971B2872A8421462308B10021
:100DC00013051101BE853AC436C697E00000E780DE
:100DD00000FBB24693059101368597000000E7803D
:100DE00060A82285141035460C0897000000E780A3
:100DF00020F62A84224701E921460C103A8597E023
:100E00000000E780C0F7228545611713FFFF6700E8
:100E1000432F1713FFFFE702832C7171AE84AA855D
:100E20000A85328497000000E78060BB11C90A86FA
:100E3000A685228597000000E78020B8814711E150
:100E4000C5473E854D611713FFFF6700832B1713BE
:100E5000FFFFE702C3251D712A8AB289BE84354689
:100E60008547130511012E8CB68A3A8BC28C468DAC
:100E70002308F10097E00000E78060F010100C08F4
:100E80005285231F010097000000E780C0F82A84E4
:100E90003DEDA1476313FD089307900591E0E547F9
:100EA0003546E2851305110113990A012308F10063
:100EB0001359090197E00000E78060EC135789009F
:100EC00093978A00D98F90080C085285231FF10050
:100ED00097000000E78020F42A8415E9A1E49387B5
:100EE000FA0091831379F9003EC663130900414962
:100EF000668B8144C14B854DB247639F970C6A86D0
:100F00008C0033855C0197E00000E78040E7228594
:100F100025611713FFFF6700431D93079004C9F075
:100F2000A547BDBF834701050947C14B2308F10011
:100F300083471105A58FA308F100938724008144FE
:100F400063E1FB04014714083386E6008C08B3868E
:100F5000E400BA95DA9683C6060083C50500050746
:100F6000AD8E2300D600E390E7FE4147639CE70483
:100F700090080C08528597000000E780C0E925D151
:100F800081A0B3069B00BA871008B305F60090084D
:100F90003E9603C506000346060085078506298E92
:100FA0002380C500E39277FF998F90080C08528543
:100FB000BE9497000000E78000E68947014749D1C9
:100FC0002A84B1B790083E96034606001408BE96E0
:100FD0002380C600850759BFB247850463879714ED
:100FE00081471808B306F70098083E973386F90042
:100FF00003470700034606008507318F2380E6007C
:10100000E39177FF90080C08528597000000E78075
:1010100080E05DF53546E285130511012308B10135
:1010200097E00000E780A0D51397040141839397D0
:1010300084002183D98F10180C085285231FF100DA
:1010400097000000E78020DD25FD814710183387D9
:10105000F9003E960347070003460600B306FB006F
:101060008507318F2380E600E39277FF65A8180893
:10107000B306F70098083E973386F9000347070048
:10108000034606008507318F2380E600E3E127FF52
:10109000CA87639E770990080C0852859700000064
:1010A000E78060D711FD81479800B306F7009008EC
:1010B00018103E973E960347070003460600850733
:1010C000318F2380E600E39177FF3546E2851305F3
:1010D00011012308B10197E00000E78040CA13978F
:1010E00004014183939784002183D98F10180C0841
:1010F0005285231FF10097000000E780C0D1E31163
:1011000005EC814710183387F9003E960347070026
:1011100003460600B306FB008507318F2380E600F7
:10112000E3E227FFC109410BC1BB814785B79408A2
:10113000BE9683C6060018083E972300D700850791
:1011400089BF638006321713FFFFE70243F6597128
:101150002A84BE89B28B85473546130511022E8B32
:10116000468C4289BA8A368A2300F10297E0000051
:10117000E780E0C010180C102285231701029700A9
:101180000000E78040C963180512A147631FFC06F1
:101190009307900563930900E5473546DA85130503
:1011A000110293140A012300F102C18097E00000AC
:1011B000E780E0BC93178A0013D78400D98F90088A
:1011C0000C1022852317F10297000000E780A0C4CD
:1011D0007DE1639209049307FA00BD88918391E051
:1011E000C144C207C183DE8C814A3EC6414DB2472D
:1011F00063E2FA0E6286B3854B01881097E0000027
:10120000E78080B54DC93D557DA093079004E396D6
:1012100009F8A54759B7834701050947C14C230081
:10122000F10283471105B3C7F900A300F1029387C8
:101230002900814963E1FC04814618103306D70078
:101240008C083387D900B69556970347070083C5A6
:10125000050085062D8F2300E600E390D7FE414769
:101260006390E70690080C10228597000000E78045
:1012700080BA35D189A0B3863A01BA871010B30578
:10128000F60090083E9603C5060003460600850753
:101290008506298E2380C500E39297FF3387EC40B3
:1012A00090080C102285BA9997000000E780A0B63C
:1012B0008947014741D165611713FFFF6700E3E2EA
:1012C00090083E96034606001410BE962380C60082
:1012D000850779B7B247850A93990A01939D8A00D9
:1012E00093D909016391570F85473546DA85130570
:1012F00011022300F10293D9890097E00000E780F2
:1013000000A8B3ED3D0190000C1022852317B10316
:1013100097000000E78020B059FD8147A68963EA65
:10132000970626860C084A8597E00000E78020A5EE
:1013300081471810B306F700100898083E973E96AC
:1013400003470700034606008507318F2380E60028
:10135000E3E197FE639FA90590080C102285970092
:101360000000E78040AB21F981479810B306F700F1
:10137000900818183E973E9603470700034606005C
:101380008507318F2380E600E391A7FF4109C10C57
:10139000B9BD18089000B306F7003E963387FC00ED
:1013A00003470700034606008507318F2380E600C8
:1013B000B5B798084E97034707001C10CE972380B7
:1013C000E700850941BF85473546DA8513051102D7
:1013D0002300F10293D9890097E00000E780209A6A
:1013E000B3ED3D0190000C1022852317B103970047
:1013F0000000E78040A2E31005EC81471808900048
:10140000B306F7003E963387FC0003470700034608
:1014100006008507318F2380E600E391A7FF414650
:101420000C084A8597E00000E78060958147181016
:10143000B306F700100898083E973E96034707004A
:10144000034606008507318F2380E600E391A7FF5E
:1014500090080C10228597000000E780C09B1DD5E6
:1014600099BD7D5582801713FFFFE70243C7011125
:101470002A842E8593055100328902C002C202C41B
:1014800002C69304740097F0FFFFE780A03D1D465D
:10149000A6851305910097E00000E780408E1008B4
:1014A0008A854A8597000000E780E09619ED93074A
:1014B0001400180883C607000346070085070507C0
:1014C000B18EA38FD7FEE397F4FE05611713FFFFDC
:1014D000670023C31713FFFFE702C3BE2E848C41AE
:1014E0004111AA89838715003289914463D307008B
:1014F000A1449757FF1F938727DB9C43A1C7C1CA0D
:101500008D472310F10083C725004A852301F10090
:1015100083C73500A301F10083C745002302F10012
:1015200083C75500A302F10083C7650093059100AE
:10153000A30301002303F1002304010097F0FFFF40
:10154000E78040320C404A860A8597F0FFFFE7802B
:1015500080330328040083564400A6881D08814771
:101560000147E51642868A854E8597000000E78090
:10157000408E2A8919E5A685228597B0FFFFE7806E
:10158000E0C14A8541011713FFFF6700E3B64A86B1
:101590000A8597F0FFFFE780002F6DB71713FFFF55
:1015A000E70243B22E848C414111AA89838715003A
:1015B0003289914463D30700A1449757FF1F938753
:1015C000A7CE9C43A1C7C1C68D472310F10083C796
:1015D00025004A852301F10083C73500A301F100EE
:1015E00083C745002302F10083C75500A302F10021
:1015F00083C7650093059100A30301002303F10055
:101600002304010097F0FFFFE780C0250C404A86C5
:101610000A8597F0FFFFE7800027835644000328E0
:1016200004008A85858EC2061D08C1822312D4005B
:10163000A68881470147E51642864E85970000003F
:10164000E78060B041011713FFFF6700E3AA4A86F5
:101650000A8597F0FFFFE78000234DBF1713FFFFB8
:10166000E702E3A7B335B000011185052A891315F8
:10167000F601336515012308B10093051101368485
:101680003AC632C03EC442C297F0FFFFE780801DD9
:10169000A2471248425593D68700230BF1009305C9
:1016A000910193578800A30AD100A30BF100230CEA
:1016B000010197F0FFFFE780E01A32470246032856
:1016C0000400B337E000835644009207914411C2EE
:1016D000A1444A85A68842860C0897F0FFFFE78060
:1016E00040772A8919E5A685228597B0FFFFE78014
:1016F000E0AA4A8505611713FFFF670083A017134F
:10170000FFFFE702239C01113EC68647B335B000B8
:101710008505AA891315F6015D8D2308B10093058F
:10172000110136843A89B28442C446C297F0FFFF61
:10173000E780401322489248164593578800A30A31
:10174000F1009305910193D78800230B0101A30BAE
:10175000F100230C110197F0FFFFE780A010324742
:10176000104083564400B337E00092070328090075
:10177000914891C0A1480C084E8597000000E78071
:10178000809CAA8401E9835544004A8597B0FFFFF5
:10179000E780C0A0268505611713FFFF6700C3958A
:1017A000AA959307F00F170701001307A76F631798
:1017B000B50013C5F7FF1375F50F82800505834645
:1017C000F5FFB58FBA9783C70700D5B70357450014
:1017D00014419307F00F170601001306A66C369705
:1017E00042074183139506014181631BE500AD8FDC
:1017F000B29703C50700130515F313351500828052
:10180000850603C5F6FFA98FB29783C70700D9BF26
:101810001713FFFFE702A38CB28736842E86BA86A1
:10182000AA853E85BA8497F0FFFFE7806052634F38
:101830000500228597D00000E780E0782A86A686FA
:10184000A285268597F0FFFFE78080501713FFFFE2
:101850006700238B1713FFFFE702C3865D712A8B96
:10186000AE8A17050100130565612C00B284368A23
:10187000BA893E8997F0FFFFE780C04F2A845DE177
:1018800034104146DA85280097F0FFFFE780404C8E
:101890002A8449E98547A303F100A6C29307710092
:1018A0002408BEC4A68685470D462C18281002DCE5
:1018B00002DED6C0BEC697F0FFFFE78000442A8450
:1018C00035E183477102A6860D4693F7F70723009B
:1018D000FA00C1473EDE2C188947281026DCA303F6
:1018E000F10097F0FFFFE78040412A8405ED414673
:1018F000A6854E8597D00000E78060488D47A68674
:101900000D462C182810A303F10097F0FFFFE78085
:10191000C03E2A8401E94146A6854A8597D0000049
:10192000E780E045228561611703FFFF6700C37C04
:101930001703FFFFE702A37A97F700009387C7A07A
:10194000984383C7470079712A89AE84170501003F
:10195000130545530C083AC42306F10097F0FFFF26
:10196000E78040412A8405ED14104146CA850808E5
:1019700097F0FFFFE780C03D2A8415E11408154663
:101980002C00081097F0FFFFE780803C2A8401E9D3
:1019900021462C08268597D00000E780403E22850E
:1019A00045611703FFFF6700C3751703FFFFE702D9
:1019B000037397F70000938727999C477971AA844E
:1019C0002E84170501001305654C0C083EC697F0E0
:1019D000FFFFE780203A0DE914104146A68508086C
:1019E00097F0FFFFE780C03605E1140811466C0050
:1019F000081097F0FFFFE780A03519E58347F10154
:101A000093F7F7032300F40045611703FFFF670016
:101A1000436F1703FFFFE702836C3688A1488147B5
:101A20000147E54697F0FFFFE780A0421703FFFF5D
:101A30006700236D1703FFFFE702636A3688A1483A
:101A400081470147E54697F0FFFFE780C06F170326
:101A5000FFFF6700036B1703FFFFE70243680111F5
:101A60002A842E850C0832C697F0FFFFE78080306D
:101A700009ED3247970601009386C63F1008C1451D
:101A8000228597000000E780E0D805611703FFFF7B
:101A9000670023671703FFFFE70263644111C14733
:101AA0002EC032C48A8509463EC23EC697F0FFFF6B
:101AB000E780A02441011703FFFF67008364170339
:101AC000FFFFE702C3614111AE8613061009AA8524
:101AD0000A8502C002C202C402C697F0FFFFE78077
:101AE000202741011703FFFF6700A3611703FFFFD2
:101AF000E702E35E3287970601009386A6392E86B9
:101B00009305000297000000E780C0D01703FFFF95
:101B10006700235F1703FFFFE702635C7971C1472A
:101B20002ACC2ED032D42C080D4628003ECE3ED2F0
:101B30003ED602C402C602C802CA97F0FFFFE78081
:101B4000C01B45611703FFFF6700A35B1703FFFF7F
:101B5000E702E3580111AA842E841705010013053A
:101B6000E5338A8597F0FFFFE780C02015E514086C
:101B70004146A6850A8597F0FFFFE780601D09EDC5
:101B80008347E1010347F101A207D98FCA07C9833F
:101B90006177D98F2310F40005611703FFFF6700F9
:101BA000435615CD1703FFFFE70263539747FF1F07
:101BB0009387071D90439745FF1F9385A51C1745E5
:101BC000FF1F1305E51797D00000E78000C51745F4
:101BD000FF1F1305E5161703FFFF67008352174524
:101BE000FF1F1305E51582808DCD1703FFFFE70268
:101BF000034F9747FF1F9387A718944301112E8423
:101C00000A869745FF1F9385E51797D00000E78068
:101C100040C60A850294014505611703FFFF67006E
:101C2000434E7D5582801703FFFFE702434B97D059
:101C30000000E78080D19747FF1F23A3A71417F563
:101C4000FFFF1305E5C997B00000E780C0741703D4
:101C5000FFFF6700034B1747FF1F1307A7149317D6
:101C6000150008433E95FD572310F50082801703A9
:101C7000FFFFE702C3462A84084009E51703FFFF78
:101C8000670023481C4158401CC06313E5005CC03A
:101C90008347550023200500F99BA302F50097A078
:101CA000FFFFE780207CC9BF1703FFFFE7028341E6
:101CB0009747FF1F9387071198432A8411CB8347C7
:101CC000350093F7070289C7035505008945029738
:101CD0001305440197B00000E780403B83550400A2
:101CE0000355E40097300000E780A00C485819C560
:101CF00097A0FFFFE7800077232A040213058403DF
:101D000097000000E780E0F68144B1499790FFFF1B
:101D1000E780006D63CBA4028347340023200404D2
:101D200093F727FCA301F40000489790FFFFE7809A
:101D3000206C13161500814522859700FFFFE78070
:101D4000003D1703FFFF6700233BB38734030329DC
:101D5000040385043E994A8597000000E78060F1FE
:101D60002304090065B78347350093F7070299E319
:101D7000014582808357E500E39CB7FEC167FD17EC
:101D80006316F60005458280054599A81703FFFFF5
:101D9000E702E33493170601C187B2842A8401491C
:101DA0006359F002835705009DCB01456367F60038
:101DB000034584003E953325A6001375F50F0DA04D
:101DC0001C4813171900BA9783D70700E38E97FAB8
:101DD00005099790FFFFE780A061E343A9FE014555
:101DE0001703FFFF6700E3311703FFFFE702832DAF
:101DF000AE89AA849790FFFFE78040552A8497D048
:101E0000FFFFE780A02EAA860147130684019705ED
:101E10000000938585E41745FF1F1305E5F89790AB
:101E2000FFFFE780C01B2A8925C98C441304C50025
:101E300022859E0593F5050897A0FFFFE780403CAB
:101E4000CC4083877400E18163DD070493E50508D6
:101E5000228597A0FFFFE780A03A0D4693854400B6
:101E6000228597A0FFFFE780C03683D50400228536
:101E700097A0FFFFE780E03D83D52400228597A04F
:101E8000FFFFE780003D03D6490083A509002285B6
:101E900097A0FFFFE780E0334A851703FFFF670045
:101EA000A32593F5F5076DB71703FFFFE70223237B
:101EB00001112A84328532C697A0FFFFE780E02710
:101EC0009780FFFFE780A033835704001747FF1F69
:101ED0001307C7063246231BF100930700F8A30D32
:101EE000F1001C471843231AA1008983858BB3078F
:101EF000F740B28548083ECE231C0100230D0100A7
:101F000097000000E78080EE05611703FFFF670080
:101F1000431F1703FFFFE702E31A004101453DC4D9
:101F20009304C40026853289AE8997A0FFFFE7801D
:101F3000C02495452A8A2685035B040197A0FFFFEC
:101F4000E7802021268597A0FFFFE780603E8D4532
:101F5000AA8A268597A0FFFFE780A01F268597A065
:101F6000FFFFE780E03C5C48420A135A0A01D2971F
:101F70005CC423186401814763983A0146054D818A
:101F8000330625419337160013F5F70F1703FFFFAC
:101F9000670083161703FFFFE702E31189692A8BA5
:101FA000AE8B328AB68A81440144314CFD19979038
:101FB000FFFFE780E04263CDA4009790FFFFE7803A
:101FC0002045018D33B5AA001703FFFF67002312D8
:101FD0003389840383270B003E9963170A008347E4
:101FE000890085043E94E1B703560A00DE854A85E0
:101FF00033F6C90097000000E780E0F16DD1054598
:10200000E1B71703FFFFE702830D01112A847C006B
:102010000355E5003ECAB70707003ECC7C003ECE24
:1020200097200000E78020082A898545480897A066
:10203000FFFFE78020399945480897A0FFFFE78018
:10204000E015AA844A8597200000E780A008238035
:10205000A4009747FF1F938767EE9C4341661306D2
:1020600006F09396870113D78701558F93D6870083
:10207000F18E558FA207B706FF00F58FD98F114655
:102080002C00138514003EC497D00000E78020CFB9
:102090005008A38204008945228597000000E7804C
:1020A000E0E019C9AA851305840397A0FFFFE78024
:1020B000E0313C4085073CC005611703FFFF670026
:1020C00043041703FFFFE70283019790FFFFE780B8
:1020D00020342A8405049790FFFFE780603233059F
:1020E000A402F14791453305F50297200000E780EF
:1020F00020BA11E565551703FFFF67008300974776
:10210000FF1F23A9A7CA9790FFFFE78060302A84AA
:1021100005049790FFFFE780A02E3305A4028945B0
:10212000060597200000E780A0B669D59747FF1FF6
:1021300023AAA7C69790FFFFE780802D2A84050475
:102140009790FFFFE780C02B3304A4029747FF1F3F
:10215000239C87C49790FFFFE780802B2A84979069
:10216000FFFFE780E029930714003385A702974714
:10217000FF1F239CA7C2970701009387E795174786
:10218000FF1F2327F7C20145BDB71703FFFFE70273
:1021900063F3AA842E8901449749FF1F938909DAC2
:1021A000130A80069790FFFFE78080256347A4000D
:1021B00001451703FFFF670023F43305440383A79A
:1021C00009024A86A6853E9597000000E780E0B99F
:1021D00019E10504C1BF0545E9BF1703FFFFE70289
:1021E00083EDAA8A2E8BB28B368C3A8A81440144C5
:1021F0008149974CFF1F938C6CD4130D80069790E8
:10220000FFFFE780E01F63C9A40011E085494E8508
:102210001703FFFF6700A3ED3389A40383A70C0214
:102220005E86D6853E994A8597000000E780E0B338
:102230001DC19790FFFFE780A01D0544636D450118
:10224000D2866286DA851305090397000000E780CD
:10225000A0D411C1854985045DB71703FFFFE702CC
:1022600063E6C16441112A8901449749FF1F93899C
:10227000E9CC130A8006FD1436C632C42EC29790EC
:10228000FFFFE780E01792452246B2466348A4006C
:10229000014541011703FFFF670003E633054403CF
:1022A00083A709023E9509C683473500C18B9DC7A8
:1022B00091C68347350093F707028DC363069900E3
:1022C0008357E500639C27010357050001CB63E7B3
:1022D000E50083478500BA97E3CDF5FA050469BFA9
:1022E0001703FFFFE70203DEC1642A89014497490F
:1022F000FF1F9389A9C4130A8006FD149790FFFF5E
:10230000E78000106346A4001703FFFF6700C3DEE9
:102310003305440383A709023E958357E500638A8A
:102320009700630499006396270197000000E780F7
:10233000E0970504E1B71703FFFFE70243D7896978
:102340002A8AAE8A328BB68B8144174CFF1F130C3E
:10235000ECBE930C8006314DFD199790FFFFE7808E
:10236000200A63C6A4001703FFFF670003D8338960
:10237000940383270C028355CA015A863E994A85E5
:1023800097000000E780609E31C1814D15A0338425
:10239000AD038327090303D60B00D68533F6C900A6
:1023A0003E94228597000000E780E0B609E9850D9C
:1023B0009790FFFFE780C002E3CBADFC01A8228528
:1023C00097000000E780E08A23040400850471B7C9
:1023D0001703FFFFE70223CE4169AA8A014A174B80
:1023E000FF1F130BABB57D19C14B054C9790FFFF39
:1023F000E78000016346AA001703FFFF670023CFB1
:1024000093098006B3073A0383290B02BE9983D749
:10241000E900638E270163842A01639A570103A4AC
:10242000890301E84E8597000000E780C0BD050ADA
:1024300075BF83570401639977099304C400268507
:1024400097A0FFFFE78060D385452A8D2685835CB2
:10245000040197A0FFFFE780C0CF268597A0FFFF6C
:10246000E780A0E762056185635905048D452685EF
:1024700097A0FFFFE780E0CD8945268597A0FFFF65
:10248000E78020CD8945268597A0FFFFE78060CCB7
:102490008545268597A0FFFFE780E0CC83470500B0
:1024A000094793F7F707639AE7009945268597A0B0
:1024B000FFFFE78040CBA30285014848337D2D0113
:1024C000231894016A9548C40040A1BF1703FFFF79
:1024D000E702E3C037E404008327041D829797478F
:1024E000FF1F83C7A7921715FF1F1305E505A3005C
:1024F000F5008327441C82978327841C814613069A
:10250000F00F8145014582971703FFFF670063BF06
:102510001737FF1F1307877F18439745FF1F83C592
:10252000E58E9747FF1F9387E78C83468703034613
:1025300097036397D5009747FF1F2389C78C828035
:1025400083C587010347A7036317B6009747FF1F9B
:10255000238EE78A828003C687016317C7009747E7
:10256000FF1F2385D78A828083C687011307500205
:102570006319D700930760021747FF1F2308F788E6
:10258000828083C68701130660026315D600930715
:102590007002DDB783C7870155BF9747FF1F938739
:1025A0006785D44B0947638DE6081703FFFFE702F1
:1025B00003B31749FF1F130929813E84834709008C
:1025C000918B9DCFB7E4040083A7041D829783A756
:1025D000441C1735FF1F1305A57F829783A7841C12
:1025E00081461746FF1F0346A68081450145829715
:1025F00021C583470900ED9B1737FF1F2306F77C92
:102600008347040093F7F70F85CB91471737FF1FD8
:10261000232CF77E97000000E78080EB97000000F6
:10262000E78040EFB7E70400BC4F414691451735BE
:10263000FF1F0345A57C82971703FFFF670063AC6C
:1026400082801703FFFFE70283A98D4741116306CC
:10265000F504C5476308F50285476310F50297370F
:10266000FF1F2387A77AB7E70400BC4B9305001030
:102670001735FF1F03458578829741011703FFFF38
:10268000670023A885471737FF1F2303F778B7E7AD
:102690000400BC4B93050020E1BF9737FF1F9387D1
:1026A0006775D44B1147638DE600B7E7040083A735
:1026B000071D8297B7E70400BC4B930500044DBF8C
:1026C00005491737FF1F2321277583C7070032C627
:1026D0002E8493F7F70FD5D3B7E4040083A7041D26
:1026E0007D141374F40F8297E37689FCB245994701
:1026F00003C61500E3F0C7FCFC4409061735FF1FAD
:10270000130545718297BC48930500081735FF1FD4
:102710000345C56E829779BF1703FFFFE702239C2D
:102720001737FF1F1307076D4047184B1C4097369C
:10273000FF1F23A7F66C6316E4001737FF1F232340
:10274000F76C130584FE9790FFFFE78040A90355BF
:1027500064FF9780FFFFE780C07197A0FFFFE780CD
:1027600060D01703FFFF6700C3991703FFFFE7025D
:1027700003979737FF1F9387E767D84BDC4789C7D5
:1027800097000000E78080F985471737FF1F232D4A
:10279000F7669737FF1F938767579C43930500029F
:1027A0001735FF1F0345856583C787031737FF1F4D
:1027B000230EF764B7E70400BC4B82971703FFFFB3
:1027C000670023949737FF1F23A8A762828017030F
:1027D000FFFFE702238F37E404007C4CA145173547
:1027E000FF1F0345A56182977C48A1451735FF1F50
:1027F0000345C5609734FF1F9384C45F8297DC4410
:1028000089EB97000000E78080D91703FFFF67007E
:10281000A38E03D567FF9780FFFFE7808065AA89B5
:102820006DD1D84891476310F7027C4C914517351C
:10283000FF1F0345A55C82977C4891451735FF1F14
:102840000345C55B829703A9490103D40901894760
:10285000B7E904001737FF1F2328F75A83A7091D7C
:1028600021044204829783C784011715FF1F1305B3
:10287000A5CD61191717FF1FA308F7CC83A7491C23
:10288000418082979737FF1F2384075883A7C91C6D
:10289000814609469375F40F4A85829711E9973767
:1028A000FF1F83C7276789C79700FF1FE780803412
:1028B000B7E70400BC4F2146A1451735FF1F03456C
:1028C000E553829799B71703FFFFE702438193F718
:1028D000052001112E8481CF97000000E78020E9B8
:1028E0001345042005611703FFFF6700838193F7F9
:1028F0000510A9CF9734FF1F9384C44FDC4897007D
:102900000000E78020C11737FF1F13072740184337
:1029100083C78401034787036318F700DC4489C732
:1029200097000000E78080DF85471737FF1F232DC2
:10293000F74CB7E70400BC4B930500021735FF1FA7
:102940000345C54B82971345041069BF93F70508EB
:10295000BDC79737FF1F83C7F74BE9171946973550
:10296000FF1F9385454B1305D10093F4F70F1739DB
:10297000FF1F0349294A97C00000E7804040939712
:102980000401C1831737FF1F13074749231DF100B7
:10299000231CF1009737FF1F9387C7453ACE3ACAE9
:1029A000D8432306010009CBDC4393158901540861
:1029B0000D46E185680082971345040825B793F713
:1029C0002500A5C39737FF1F9387C742D84B894778
:1029D0006306F7029737FF1F83C7073F13F72700E8
:1029E00011EF918B99CFB7E70400BC4F1306000A93
:1029F00089451735FF1F034565408297134524001D
:102A0000D5B59737FF1F938767309C4383C78703EC
:102A10001737FF1F230CF73E97000000E78060DBAD
:102A2000F1BF93F7050281CB97000000E78060DAE1
:102A30001345040245BD93F7850081CB9700000044
:102A4000E780E0D21345840071BD93F7150081CB78
:102A500097000000E780A0B41345140061B593F718
:102A6000450081CB97000000E78060B31345440028
:102A700095BD93F7050495C39737FF1F83C7873725
:102A800091CB97000000E780A0A491471737FF1F64
:102A9000232CF73613450404B1B593F7050101451E
:102AA000E38207E49737FF1F9387C734D84B9147DA
:102AB0006310F7049737FF1F938707319C4313D7A1
:102AC00027008583D98F858B91E7B7E7040083A71B
:102AD000071D8297B7E70400FC4F91451735FF1F8C
:102AE0000345C531829785471737FF1F232EF730DF
:102AF00013450401C5BB9737FF1F238DA740828074
:102B000017F3FEFFE702A35D9737FF1F23AA072EE7
:102B10009737FF1F23A8072E85471734FF1F13047D
:102B2000E41E1737FF1F2321F72E1C4083C787039E
:102B30001737FF1F230CF72C9790FFFFE780809239
:102B400029C59717FF1F23A5A7A01C401705000044
:102B50001305A5D783C787031737FF1F2308F72A55
:102B60001717FF1FA302F79E9737FF1FA38407289D
:102B7000B7E7040083A7070882979737FF1F238FC3
:102B8000A72617F3FEFF6700C357B7C7898E938741
:102B900067ED1717FF1F232DF79A45BF1737FF1F44
:102BA00003474725795555E79737FF1F93878724B4
:102BB00003C7170005079736FF1FA38DE62203C73B
:102BC00017008D463377D7029736FF1FA384E6227E
:102BD00083C617001737FF1F13074713184393F6D1
:102BE000F60FA9EE834787031737FF1F2300F7224D
:102BF00085471737FF1F230FF71E9737FF1F938750
